:100000000C94781A0C94A91A0C94A91A0C94A91A95
:100010000C94A91A0C94A91A0C94A91A0C94A91A54
:100020000C94A91A0C94A91A0C94A91A0C94A91A44
:100030000C94A91A0C94A91A0C94A91A0C94A91A34
:100040000C94A91A0C9457D10C94A91A0C94A91ABF
:100050000C94A91A0C94A91A0C9454BE0C94F4A9EB
:100060000C94A91A0C9427560C941D560C94A91A9A
:100070000C94A91A0C94A91A0C94A91A0C94A91AF4
:100080000C9400340C94A91A0C94A91A0C94A91A73
:100090000C94A91A0C94A91A0C94A91A0C94A91AD4
:1000A0000C94A91A0C94A91A0C94D2330C94A91A82
:1000B0000C94A91A0C94A91A0C94A91A0C94A91AB4
:1000C0000C94A91A0C94A91A0C94A91A0C941B3715
:1000D0000C94E5360C94A91A0C94A91A0C94A91A3C
:1000E0000C94A91A084AD73B3BCE016E84BCBFFDD5
:1000F000C12F3D6C74319ABD56833DDA3D00C77FF8
:1001000011BED9E4BB4C3E916BAAAABE0000008090
:100110003F05A84CCDB2D44EB93836A9020C50B91F
:10012000918688083CA6AAAA2ABE000000803F004B
:100130000C9444FC0D942E0B0C9479FC0C9428FC2C
:100140000C94AAFB0C94EBA70C943CFC0C949737F2
:100150000D94C70C0C94D1A90C941EFC0D94030CA7
:100160000C94B9560C9483FC0C945B440C946AFC7C
:100170000D944A0F0C94C1370C94A1FB0C94C6FB50
:100180000C9483FB0D940E090D94B11E0D945E0921
:100190000C94DF370C94D4FB0C94B2560C9407A942
:1001A0000D940C110D941D0F0D94FB040C946342DF
:1001B0000D942C0F0C9414FF0D94040F0D94D40E79
:1001C0000C94C5560D94570B0C94A4FB0C9460FC36
:1001D0000D94570F0D9444010C94D1560D94EC13CB
:1001E0000C94B5370D9495070C94CC370C948DFC7A
:1001F0000C94D7370D94160C0D9449100D942A09C0
:100200000C94BD560D94931E0C9411FC0C94A356A3
:100210000C94AEFB0C9495FB0C94C5370C94B8FB76
:100220000C94CAA70C9494560C94CD560C94D0FB05
:100230000D948E0B0C94CAFB0C9459370C94B13767
:100240000C947EFB0C9497FC0C94B9370D943810E9
:100250000C94C8A80C949DFB0C949C440C9466A42C
:100260000C9414420C9419FC0C94D8560C94A1FCD8
:100270000C94AD370D94C10B0D946B0B0C9435A7FA
:100280000D941A010D94360F0C9465560C94A637F4
:100290000C9499FB0D94C00A0C944CFC0C94ABFC90
:1002A0000C94EB560D94AC020D94FB0E0D94FA09D0
:1002B0000D947D030D94DB080C94BD370D948A0AD0
:1002C0000C94E3560D94A20B0C942FA80C94BCFB39
:1002D0000C942F440C9456FC0C94C2FB0C94E9A48F
:1002E0000C94E8A40C9432FC0C94D4440C94DAA83A
:1002F0000D94010F0C9467420D9435000C94C15677
:100300000C94C9560C94B4FB0C944AA80C9452A7B4
:100310000C9488374E414E494E495459494E46CD6A
:10032000CCCC3D0AD7233C17B7D13877CC2B3295AC
:1003300095E6241FB14F0A000020410000C842008A
:10034000401C4620BCBE4CCA1B0E5AAEC59D740054
:10035000407A10F35A00A0724E18090010A5D4E894
:100360000000E87648170000E40B54020000CA9A27
:100370003B000000E1F50500008096980000004079
:10038000420F000000A086010000001027000000BE
:1003900000E803000000006400000000000A000004
:1003A0000000000100000000002C76D888DC674FB8
:1003B0000823DFC1DFAE59E1B1B796E5E3E453C6E8
:1003C0003AE651997696E8E6C28426EB898C9B62E0
:1003D000ED407C6FFCEFBC9C9F40F2BAA56FA5F48A
:1003E00090055A2AF75C936B6CF9676DC11BFCE0B2
:1003F000E40D47FEF520E6B500D0ED902E03009405
:100400003577050080841E080000204E0A00000099
:10041000C80C333333330F986E12831141EF8D21A3
:1004200014893BE65516CFFEE6DB18D1844B381B0A
:10043000F77C1D901DA4BBE424203284725E2281CF
:1004400000C9F124ECA1E53D27434F4D4D554E49E0
:10045000434154494F4E0044525952554E00455263
:10046000524F525300494E464F004543484F0045B6
:1004700072726F722077726974696E6720746F2070
:10048000454550524F4D210A0053544F505045445A
:100490002E20005072696E7465722073746F7070D4
:1004A00065642064756520746F206572726F727365
:1004B0002E2046697820746865206572726F7220FC
:1004C000616E6420757365204D39393920746F2051
:1004D000726573746172742E202854656D70657234
:1004E00061747572652069732072657365742E205E
:1004F0005365742069742061667465722072657337
:1005000074617274696E67290A004E6F20436865D2
:10051000636B73756D2077697468206C696E6520F4
:100520006E756D6265722C204C617374204C696E1F
:10053000653A20004E6F20436865636B73756D20CC
:1005400077697468206C696E65206E756D6265727E
:100550002C204C617374204C696E653A20006368EE
:1005600065636B73756D206D69736D617463682C61
:10057000204C617374204C696E653A20004C696EA2
:1005800065204E756D626572206973206E6F7420F0
:100590004C617374204C696E65204E756D62657296
:1005A0002B312C204C617374204C696E653A20000D
:1005B0004D3131300053657269616C207374617420
:1005C0007573206D69736D617463680A0077616982
:1005D000740A0053442072656164206572726F7200
:1005E0000A002121204B494C4C20636175736564DE
:1005F00020627920746F6F206D75636820696E6169
:1006000063746976652074696D65202D2063757249
:1006100072656E7420636F6D6D616E643A20004880
:100620006F74656E642049646C652054696D656FF4
:10063000757400486F74656E642049646C6520545D
:10064000696D656F75740A003D3D6F6E46696C613A
:100650006D656E7452756E6F75743D3D0070617599
:100660007365004D363030002066696C616D656ED3
:10067000745F72756E6F7574200066696C616D656C
:100680006E745F72756E6F757420540046696C618C
:100690006D656E7452756E6F75742054002A2A2A27
:1006A000496E6974696E67206361726420697320A2
:1006B0004F4B2A2A2A004D6564696120496E736593
:1006C00072746564004D656469612052656D6F7672
:1006D0006564004D313030305300627573793A20D3
:1006E00070617573656420666F7220696E707574D1
:1006F0000A00627573793A207061757365642066CB
:100700006F7220757365720A00627573793A207092
:10071000726F63657373696E670A002A2A2A6B69B0
:100720006C6C2A2A2A00706F7765726F6666004BC0
:10073000494C4C45442E20005072696E74657220FD
:1007400068616C7465642E206B696C6C2829206369
:10075000616C6C6564210A0053544F505045442E1F
:1007600020005072696E7465722073746F707065CA
:10077000642064756520746F206572726F72732EC9
:100780002046697820746865206572726F722061F6
:100790006E6420757365204D39393920746F20726D
:1007A0006573746172742E202854656D7065726172
:1007B000747572652069732072657365742E205399
:1007C0006574206974206166746572207265737443
:1007D000617274696E67290A006563686F3A004543
:1007E00072726F723A0042696C696E656172204C78
:1007F0006576656C696E6720477269643A0A002104
:10080000212053544F502063616C6C6564206265F5
:100810006361757365206F6620424C546F75636821
:10082000206572726F72202D20726573746172740C
:100830002077697468204D3939390A002121205305
:10084000544F502063616C6C656420626563617510
:100850007365206F6620424C546F75636820657223
:10086000726F72202D2072657374617274207769C3
:100870007468204D3939390A002F2F616374696F0C
:100880006E3A0070726F6D70745F00656E64005335
:10089000656E64204D31303820746F207265737539
:1008A0006D650A00496E736572742066696C616DCE
:1008B000656E7420616E642073656E64204D313006
:1008C000380A005265686561742066696E697368EC
:1008D00065642E0052656865617420446F6E650022
:1008E000526568656174696E672E2E2E00526568C8
:1008F000656174004865617465722054696D656F47
:1009000075740053656E64204D31303820746F204B
:1009100068656174206E6F7A7A6C650A004E6F7A32
:100920007A6C65205061726B656400486F74656E07
:100930006420746F6F20636F6C640A00706175735C
:1009400065640050617573650044697361626C652C
:1009500052756E6F75740050757267654D6F726574
:10096000005061757365640073686F770062757419
:10097000746F6E00626567696E004C6F616420463B
:10098000696C616D656E74004C6F61642046696CC2
:10099000616D656E74205400496E736572742066D3
:1009A000696C616D656E7420616E642073656E6440
:1009B000204D3130380A00726573756D65640052E0
:1009C0006573756D696E670057616974696E67203C
:1009D000666F72206865617475702E0A004C6561DF
:1009E00076696E6720473236003F537065636966EB
:1009F00069656420582C5920636F6F7264696E6159
:100A00007465206F7574206F6620626F756E6473F5
:100A10002E0A003F28522965706561742076616C4A
:100A20007565206E6F7420706C61757369626C659A
:100A30003B206D757374206265206174206C656164
:100A4000737420312E0A003F285229657065617445
:100A5000206D7573742062652073706563696669C3
:100A60006564207768656E206E6F74207573696E9B
:100A70006720616E204C43442E0A003F537065632B
:100A80006966696564206E6F7A7A6C652074656D3D
:100A90007065726174757265206E6F7420706C6120
:100AA000757369626C652E0A003F537065636966F1
:100AB0006965642066696C616D656E742073697A1E
:100AC00065206E6F7420706C61757369626C652E41
:100AD0000A003F53706563696669656420707269D6
:100AE0006D65206C656E677468206E6F7420706C25
:100AF00061757369626C652E0A003F5072696D659D
:100B0000206C656E677468206D7573742062652053
:100B1000737065636966696564207768656E206EC9
:100B20006F74207573696E6720616E204C43442E8C
:100B30000A003F537065636966696564206E6F7A69
:100B40007A6C652073697A65206E6F7420706C61B1
:100B5000757369626C652E0A003F52657472616339
:100B600074696F6E204D756C7469706C6965722064
:100B70006D7573742062652073706563696669655D
:100B8000642E0A003F53706563696669656420528C
:100B9000657472616374696F6E204D756C746970F1
:100BA0006C696572206E6F7420706C617573696218
:100BB0006C652E0A003F5370656369666965642041
:100BC0006C6179657220686569676874206E6F74FE
:100BD00020706C61757369626C652E0A0043292E62
:100BE0000A003F53706563696669656420626564E5
:100BF0002074656D7065726174757265206E6F74B6
:100C000020706C61757369626C65202834302D002A
:100C1000473236207374617274696E672E2E2E0A05
:100C2000004F46460A00466164652048656967686A
:100C3000742000426564204C6576656C696E67209F
:100C4000004661696C656420746F20656E61626C3A
:100C50006520426564204C6576656C696E670A00A4
:100C6000496E76616C6964206D6573682E0A005068
:100C7000726F62696E6720506F696E740025532031
:100C800025692F2569002E0A002F0050726F6269B6
:100C90006E67206D65736820706F696E7420002028
:100CA0002844525952554E29004732392041757413
:100CB0006F20426564204C6576656C696E67003F05
:100CC00020284C2C522C462C4229206F7574206F02
:100CD0006620626F756E64732E0A003F2856296580
:100CE00072626F7365206C6576656C20696D706CDF
:100CF00061757369626C652028302D34292E0A00D5
:100D0000426164205A2076616C75650A004E6F203E
:100D100062696C696E65617220677269640A004479
:100D20006576696174696F6E0025533A20257300FA
:100D300046696E6973686564210A003A207A3A2030
:100D400000206F662000476F696E6720746F3A203D
:100D5000580043570A00206469723A0020616E67A8
:100D60006C653A00537461727420726164697573C2
:100D70003A004D343820506F696E740025533A2084
:100D800025642F256400506F736974696F6E696EF6
:100D900067207468652070726F62652E2E2E0A00BF
:100DA0003F4C656773206F66206D6F76656D656E6D
:100DB0007420696D706C61757369626C6520283090
:100DC0002D3135292E0A003F2028582C5929206F13
:100DD0007574206F6620626F756E64732E0A005002
:100DE000726F6265206F7574206F6620626F756E1A
:100DF0006473003F53616D706C652073697A652080
:100E00006E6F7420706C61757369626C6520283434
:100E10002D3530292E0A004D3438205A2D50726F4E
:100E20006265205265706561746162696C6974798C
:100E300020546573740A003F2856296572626F73E7
:100E400065206C6576656C20696D706C6175736981
:100E5000626C652028302D34292E0A005374616E8F
:100E60006461726420446576696174696F6E3A20CA
:100E7000002052616E67653A2000204D61783A206B
:100E800000204D696E3A2000205369676D613A2059
:100E9000004D65616E3A20005741524E494E472140
:100EA000204C6F77205A204A65726B206D61792043
:100EB0006C65616420746F20756E77616E74656413
:100EC000207061757365732E0A004F4646004F4EC1
:100ED0000020204D61783A2000200020204D696ECE
:100EE0003A2000536F667420656E6473746F70737C
:100EF0003A20003D3D4F6E506F7765724C6F7373B3
:100F0000526573756D653D3D004D32342053256C3F
:100F1000642054256C64004739322E3920452573EE
:100F200000473120462564004739322E39205A25A2
:100F300073004731205A302046323030004731208C
:100F400058257320592573204633303030004D34F6
:100F5000323020532569205A2573004D3130362018
:100F600050256920532569004D32303020442573C7
:100F70000047323852305859004739322E3920450F
:100F800030205A300A47315A2573004D313039200C
:100F9000532569004D31393020532569004D3432D5
:100FA00030205330205A300020496E76616C6964DD
:100FB000206578747275646572200047322F47335C
:100FC0002062616420706172616D65746572730A7C
:100FD00000536C6565702E2E2E005A2050726F6281
:100FE000652050617374204265640A005A20507273
:100FF0006F62652050617374204265640047323827
:101000004C30004D3131372050726F62652066617F
:10101000696C65642E0A4732380A0070726F626527
:101020005F72657769706500473239205265747266
:1010300079696E670050726F62696E6720466169F8
:101040006C6564004D31313720426564206C6576F3
:10105000656C696E67206661696C65642E0A47304D
:10106000205A31300A4D3330302050323520533839
:1010700038300A4D333030205035302053300A4D4F
:101080003330302050323520533838300A4D333029
:1010900030205035302053300A4D3330302050321C
:1010A0003520533838300A4D333030205035302019
:1010B00053300A47342053310070726F62655F66A7
:1010C00061696C6564004D31313720426564206C84
:1010D0006576656C696E6720646F6E652E00205AB8
:1010E0003A200020593A200042656420583A2000F6
:1010F0004D65736820706F696E74206F7574206F12
:10110000662072616E67650A004D302053746F70FF
:10111000004D312053746F7000436F6E74696E75AB
:101120006500436C69636B20746F20526573756D45
:10113000652E2E2E004E6F204D6F76652E00456E6B
:10114000642066696C65206C6973740A0042656787
:10115000696E2066696C65206C6973740A004E6F55
:10116000206D656469610A00526573756D696E670B
:1011700020534400286E6F2066696C652900437512
:101180007272656E742066696C653A2000507269EF
:101190006E742074696D653A20000A53746174732B
:1011A0003A2046696C616D656E7420757365643AAA
:1011B00020002C204C6F6E67657374206A6F623A52
:1011C0002000546F74616C2074696D653A2000537F
:1011D000746174733A20002C204661696C65643A2E
:1011E00020002C2046696E69736865643A200050BF
:1011F00072696E74733A200053746174733A2000FC
:10120000436F6F6C696E672E2E2E0048656174699E
:101210006E672E2E2E0045202553006F6B006F66E3
:1012200066006A0465045E04570449044445425557
:10123000473A004D31313320530042656420436FFB
:101240006F6C696E672E2E2E0042656420486561C2
:1012500074696E672E2E2E00544D33442031305366
:101260002050726F204F46462E002F2F0020520034
:10127000416363656C65726174696F6E3A205000FA
:101280004D32303620580046523A0020466C6F7777
:101290003A20003A200020536572766F2000206FBC
:1012A0007574206F662072616E67650A00536572FF
:1012B000766F200020643A0020693A0020703A00DE
:1012C000496E76616C6964206578747275646572C4
:1012D0000A0020643A0020693A0020703A006469EC
:1012E0007300656E0043290A0061626C6564202802
:1012F0006D696E2074656D702000436F6C642065AD
:101300007874727564657320617265200050494479
:10131000204175746F74756E6500504944204175A5
:10132000746F74756E65206661696C656421204216
:101330006164206865617465722069640A004669A9
:101340006C616D656E742072756E6F757420646962
:101350007374616E636520286D6D293A20004669BB
:101360006C616D656E742072756E6F757420004DC2
:1013700034323120696E636F7272656374207061FC
:1013800072616D657465722075736167650A004DE1
:1013900065736820706F696E74206F7574206F6656
:1013A0002072616E67650A004F666673657473200C
:1013B0004170706C696564004572723A20546F6FB9
:1013C000206661722100546F6F2066617220667220
:1013D0006F6D207265666572656E636520706F69FA
:1013E0006E740A00454550524F4D204F4B0A005035
:1013F0006F7765722D6C6F7373207265636F76659E
:10140000727920004D383400446F6E652070726927
:101410006E74696E672066696C650A004D37370027
:101420004D3331004361703A004D454154504143C2
:101430004B00434F4F4C45525F54454D5045524130
:1014400054555245004348414D4245525F54454D25
:10145000504552415455524500424142595354451A
:101460005050494E470041524353004D4F54494F4D
:101470004E5F4D4F44455300544845524D414C5FDB
:1014800050524F54454354494F4E004C4F4E475FC6
:1014900046494C454E414D45004155544F524550EB
:1014A0004F52545F53445F53544154555300534477
:1014B0005F575249544500524550454154005344EA
:1014C000434152440050524F4D50545F5355505079
:1014D0004F525400454D455247454E43595F504188
:1014E0005253455200434153455F4C494748545F6E
:1014F0004252494748544E45535300544F47474C76
:10150000455F4C494748545300534F465457415246
:10151000455F504F574552004255494C445F504536
:101520005243454E54004C4556454C494E475F4446
:10153000415441005A5F50524F42450052554E4F60
:101540005554004155544F4C4556454C0050524956
:101550004E545F4A4F420050524F4752455353003A
:101560004155544F5245504F52545F54454D5000D1
:10157000564F4C554D455452494300454550524FE6
:101580004D0042494E4152595F46494C455F5452C5
:10159000414E534645520053455249414C5F584FC6
:1015A0004E5F584F4646004649524D574152455F9F
:1015B0004E414D453A4D61726C696E20322E302E8F
:1015C000375F4457372E3320544D33442053534D07
:1015D000444242202841707220323420323032316D
:1015E0002031393A34333A30392920534F55524358
:1015F000455F434F44455F55524C3A68747470736D
:101600003A2F2F6769746875622E636F6D2F496E6C
:1016100073616E6974794175746F6D6174696F6E11
:101620002F4D61726C696E2F747265652F43726500
:10163000616C6974794477696E5F322E3020505244
:101640004F544F434F4C5F56455253494F4E3A31DA
:101650002E30204D414348494E455F545950453A3C
:10166000544D3344203130532050726F204558542C
:1016700052554445525F434F554E543A31205555CB
:1016800049443A63656465326132662D34316132B2
:101690002D343734382D396231322D633535633688
:1016A000326633363766660A0050726F6265204FC5
:1016B0006666736574205A0050726F6265204F66CB
:1016C00066736574205A00290A0020746F20003F59
:1016D0005A206F7574206F662072616E67652028CE
:1016E00000290A0020746F20003F59206F75742074
:1016F0006F662072616E676520282D00290A002020
:10170000746F20003F58206F7574206F66207261DF
:101710006E676520282D0050726F6265204F6666E7
:1017200073657420580043616E6E6F74206F70652E
:101730006E207375626469722000256973002569E3
:101740006D20256973002569682025696D2025694C
:101750007300256964202569682025696D20256945
:101760007300256979202569642025696820256929
:101770006D20256973003D3D4477696E20496E698F
:101780007420436F6D706C6574653D3D002A2A2A94
:101790004E6F7A7A6C6554656D70537461747573AD
:1017A0005B325D203D003D3D48656174696E672098
:1017B000446F6E65204368616E67652046696C61A1
:1017C0006D656E743D3D002020737461727470729B
:1017D0006F677265737320003D3D7761697477614F
:1017E0007920353D3D003D3D776169747761792011
:1017F000343D3D003D3D7761697477617920333D2B
:101800003D003D3D7761697477617920313D3D0050
:101810003D3D6F6E5072696E7454696D657253749C
:101820006F707065643D3D003D3D6F6E4661637451
:101830006F727952657365743D3D00270A0A000096
:10184000272027002027002D006E6F7469666963CA
:101850006174696F6E200063616E63656C00507225
:10186000696E742041626F72746564004469736DBF
:101870006973730055492041626F72746564007228
:101880006573756D65004D3234002A2A2A43506C09
:10189000617920546F6E652A2A2A003D3D6F6E5093
:1018A00072696E7454696D65725061757365643DDB
:1018B0003D00486F6D696E67204661696C65640024
:1018C0006F70656E00545249474745524544003A8F
:1018D000200066696C616D656E74007A5F6D696E7B
:1018E00000795F6D696E00785F6D696E005265709A
:1018F0006F7274696E6720656E6473746F702073A5
:1019000074617475730A0020746F6F206C6F6E675A
:1019100020657874727573696F6E20707265766574
:101920006E7465640A0020636F6C6420657874725D
:101930007573696F6E2070726576656E7465640A82
:1019400000486F6D652025732573257320466972E5
:101950007374005761726E696E673A20486F6D69E3
:101960006E672042756D702044697669736F7220CE
:101970003C20310A000202040000000000000000C8
:101980000000000000809D4300009B430000C8430E
:10199000000000410000004100000040FFFFFF0088
:1019A00000000100000001000080005555550000B6
:1019B00000400033333300AAAA2A004992240000D1
:1019C000002000C7711C0099991900D145170055D6
:1019D0005515003BB11300244912001111110000EC
:1019E0000010000F0F0F00E3380E0043790D00CCFC
:1019F000CC0C00C3300C00E8A20B0064210B00AA41
:101A0000AA0A00703D0A009DD80900427B09009295
:101A1000240900DCD3080088880800104208000070
:101A2000000800F0C10700878707007550070071A4
:101A30001C07003EEB0600A1BC060069900600668C
:101A4000660600703E06006118060017F405007473
:101A5000D105005BB00500B290050062720500552B
:101A600055050078390500B81E0500050505004E2E
:101A7000EC040087D40400A1BD040090A704004931
:101A8000920400C17D0400EE690400C756040044BE
:101A90004404005C320400082104004110040000EA
:101AA0000004003FF00300F8E0030026D20300C367
:101AB000C30300CCB503003AA803000A9B03003817
:101AC0008E0300C08103009F750300D0690300509E
:101AD0005E03001D53030034480300913D030033AF
:101AE00033030016290300381F0300971503003045
:101AF0000C0300030303000BFA020049F10200BAD1
:101B0000E802005CE002002DD802002DD00200594E
:101B1000C80200B0C0020031B90200DAB10200AA66
:101B2000AA0200A0A30200BC9C0200FA9502005C7D
:101B30008F0200DF88020082820200457C020027BB
:101B400076020027700200436A02007C640200D023
:101B50005E02003F590200C8530200FFFDFCFAF884
:101B6000F6F4F2F0EEECEAE9E7E5E3E1E0DEDCDAF8
:101B7000D9D7D5D4D2D0CFCDCBCAC8C7C5C3C2C0A0
:101B8000BFBDBCBAB9B7B6B4B3B2B0AFADACAAA919
:101B9000A8A6A5A4A2A1A09E9D9C9A999897959469
:101BA0009392908F8E8D8B8A898887868483828199
:101BB000807F7E7D7B7A79787776757473727170A9
:101BC0006F6E6D6C6B6A696867666564636261609D
:101BD0005F5E5D5C5B5A5958585756555453525185
:101BE00050504F4E4D4C4B4A4A4948474646454453
:101BF00043424241403F3E3E3D3C3B3B3A39383810
:101C000037363535343332323130302F2E2E2D2CBD
:101C10002B2B2A292928272726252524232322215F
:101C20002120201F1E1E1D1C1C1B1B1A19191818F1
:101C3000171616151514131312121111100F0F0E7B
:101C40000E0D0D0C0C0B0A0A0909080807070606F9
:101C500005050404030302020100003D3D6F6E50C0
:101C600072696E7454696D657253746172746564DF
:101C70003D3D0000809D4300009B430000C84300A1
:101C800000000000000000000000003D3D6F6E53AA
:101C9000746F726553657474696E67733D3D003D82
:101CA0003D6F6E436F6E66696775726174696F6EC2
:101CB00053746F72655772697474656E3D3D00535D
:101CC000657474696E67732053746F726564000A7B
:101CD00020696E6974207A70726F62655F7A6F66D0
:101CE00066736574203D20003D3D6F6E436F6E66E8
:101CF000696775726174696F6E53746F726552654E
:101D000061643D3D00454550524F4D20496E697418
:101D100069616C697A65640A003B20003A0A002018
:101D2000204D363033200020440020204D34313205
:101D300020530046696C616D656E742072756E6F1C
:101D400075742073656E736F723A002055004C00F5
:101D500046696C616D656E74206C6F61642F756E81
:101D60006C6F6164206C656E677468733A00202044
:101D70004D3835312058005A2D50726F6265204F12
:101D800066667365740020204D3431332053005053
:101D90006F7765722D4C6F7373205265636F766534
:101DA00072793A0020440020490020204D3330341D
:101DB00020500020440020490020204D33303120A5
:101DC00050005049442073657474696E67733A001B
:101DD000204A002020473239205720490020204D3A
:101DE0003432302053004175746F20426564204CBA
:101DF0006576656C696E673A0020204D323036207A
:101E00005800486F6D65206F66667365743A0020F0
:101E1000580020530020204D3230352042004164CC
:101E200076616E6365643A20423C6D696E5F7365EE
:101E3000676D656E745F74696D655F75733E205381
:101E40003C6D696E5F66656564726174653E2054C1
:101E50003C6D696E5F74726176656C5F6665656422
:101E6000726174653E20583C6D61785F785F6A6589
:101E7000726B3E20593C6D61785F795F6A65726B69
:101E80003E205A3C6D61785F7A5F6A65726B3E20D6
:101E9000453C6D61785F655F6A65726B3E002054FA
:101EA0000020520020204D32303420500041636326
:101EB000656C65726174696F6E2028756E697473E4
:101EC0002F7332293A20503C7072696E745F6163DF
:101ED00063656C3E20523C726574726163745F612D
:101EE0006363656C3E20543C74726176656C5F611F
:101EF0006363656C3E0020204D3230312058004D28
:101F00006178696D756D20416363656C657261749C
:101F1000696F6E2028756E6974732F7332293A00C9
:101F200020204D3230332058004D6178696D756D39
:101F3000206665656472617465732028756E6974C6
:101F4000732F73293A005374657073207065722083
:101F5000756E69743A0020440020204D32303020E4
:101F600053002044697361626C65640A0046696CC1
:101F7000616D656E742073657474696E67733A0081
:101F800020286D6D29002020473231202020203B61
:101F900020556E69747320696E206D6D003D3D6F34
:101FA0006E4C6F616453657474696E67733D3D0078
:101FB0000000FA430000FA430000204100008C4278
:101FC0000000A0420000A0420000C84300000C43F3
:101FD000EE020000EE020000640000003C00000081
:101FE00024F4D43050C38E20C2A24017828B7011CB
:101FF000127A910D816CD90AA861E108C758660769
:10200000615143061E4B5D05C145A7041A411104E9
:10201000093D9803713931034036DB026533910283
:10202000D4305402802E1D02632CEE01752AC501A6
:10203000B028A001102781018F2564012B244B01BA
:10204000E0223401AC211F018D200D01801FFC0016
:10205000841EED00971DDF00B81CD200E61BC600F1
:10206000201BBC00641AB200B219A8000A19A00013
:102070006A189900D117910040178B00B51684009B
:1020800031167E00B31579003A157300C7146F003E
:1020900058146A00EE1366008813630025135E006F
:1020A000C7125B006C12570015125400C111510089
:1020B00070114F0021114B00D61049008D104700C0
:1020C0004610440002104200C00F4000800F3E0046
:1020D000420F3C00060F3B00CB0E3800930E37003A
:1020E0005C0E3500270E3400F30D3200C10D3100B7
:1020F000900D3000600D2E00320D2D00050D2C00CE
:10210000D90C2B00AE0C2900850C29005C0C270093
:10211000350C27000E0C2600E80B2400C40B24000D
:10212000A00B23007D0B23005A0B2100390B21004B
:10213000180B2000F80A1F00D90A1E00BB0A1E0057
:102140009D0A1D00800A1D00630A1C00470A1B002F
:102150002C0A1B00110A1A00F7091A00DD091900E0
:10216000C4091900AB091900920917007B0918006E
:10217000630917004C0916003609160020091600DD
:102180000A091500F5081500E0081400CC08140031
:10219000B8081400A4081400900813007D08120069
:1021A0006B0813005808120046081200340811008A
:1021B000230811001208110001081100F007100097
:1021C000E0071000D0071000C0071000B0070F0094
:1021D000A107100091070E0083070F0074070F007E
:1021E00065070E0057070E0049070E003B070D005C
:1021F0002E070E0020070D0013070D0006070D0027
:10220000F9060C00ED060D00E0060C00D4060C00EB
:10221000C8060C00BC060C00B0060C00A4060B009F
:1022200099060C008D060B0082060B0077060B004A
:102230006C060B0061060A0057060B004C060A00EC
:1022400042060A0038060A002E060A0024060A0082
:102250001A060A001006090007060A00FD05090013
:10226000F4050900EB050900E2050900D90509009C
:10227000D0050900C7050900BE050900B50508001D
:10228000AD050800A50509009C0508009405080097
:102290008C050800840508007C050800740508000A
:1022A0006C050700650508005D0507005605080078
:1022B0004E050700470507004005080038050700E0
:1022C000310507002A050700230507001C05060045
:1022D000160507000F0507000805060002050700A0
:1022E000FB040600F5040700EE040600E8040600FF
:1022F000E2040700DB040600D5040600CF04060054
:10230000C9040600C3040600BD040600B7040600A5
:10231000B1040500AC040600A6040600A0040500F4
:102320009B04060095040500900406008A0405003D
:1023300085040500800406007A0405007504050084
:10234000700405006B0405006604050061040500C7
:102350005C04050057040500520405004D04050007
:1023600048040500430405003E0404003A04050047
:1023700035040500300404002C0405002704040083
:10238000230405001E0404001A04040016040500BA
:10239000110404000D0404000904050004040400F1
:1023A00000040400FC030400F8030400F403040028
:1023B000F0030400EC030400E8030400E403040059
:1023C000E0030400DC030400D8030400D403040089
:1023D000D0030400CC030400C8030300C5030300BA
:1023E00024F404D9201BC40C5C0E9804C4095F02B9
:1023F00065077101F405F900FB04B3004804870088
:10240000C10369005803550003034500BE023A00AA
:102410008402310053022A00290225000402200010
:10242000E4011C00C8011900AF0117009801140055
:1024300084011300710110006101100051010E00B0
:1024400043010D0036010B002B010B0020010B0096
:10245000150109000C01090003010800FB00080038
:10246000F3000800EB000700E4000600DE000600B1
:10247000D8000600D2000600CC000500C700050009
:10248000C2000500BD000400B9000400B50004004E
:10249000B1000400AD000400A9000400A500030081
:1024A000A20003009F0004009B00030098000300AB
:1024B0009500020093000300900003008D000200CD
:1024C0008B000300880002008600020084000300E5
:1024D000810002007F0002007D0002007B000200FC
:1024E000790002007700010076000200740002000B
:1024F00072000100710002006F0002006D00010017
:102500006C0002006A00010069000200670001001F
:102510006600010065000100640002006200010025
:1025200061000100600001005F0002005D00010029
:102530005C0001005B0001005A000100590001002D
:10254000580001005700010056000100550001002D
:10255000540001005300000053000100520001002C
:1025600051000100500001004F0001004E0000002A
:102570004E0001004D0001004C0001004B00000026
:102580004B0001004A000100490001004800000022
:10259000480001004700010046000000460001001D
:1025A0004500000045000100440001004300000018
:1025B0004300010042000000420001004100000011
:1025C00041000100400001003F0000003F00010009
:1025D0003E0000003E0001003D0000003D00010003
:1025E0003C0000003C0000003C0001003B000000FB
:1025F0003B0001003A0000003A00010039000000F1
:1026000039000100380000003800000038000100E7
:1026100037000000370001003600000036000000DF
:1026200036000100350000003500000035000100D3
:1026300034000000340000003400010033000000CA
:1026400033000000330001003200000032000000BF
:1026500032000100310000003100000031000100B3
:102660003000000030000000300001002F000000AA
:102670002F0000002F0000002F0001002E0000009E
:102680002E0000002E0001002D0000002D00000093
:102690002D0000002D0001002C0000002C00000087
:1026A0002C0000002C0001002B0000002B0000007B
:1026B0002B0000002B0001002A0000002A0000006F
:1026C0002A0000002A000100290000002900000063
:1026D0002900000029000000290001002800000056
:1026E0002800000028000000280000002800010049
:1026F000270000002700000027000000270000003E
:10270000270001002600000026000000260000002F
:102710002600000026000100250000002500000022
:102720002500000025000000250000002500010014
:102730002400000024000000240000002400000009
:1027400024000100230000002300000023000000FB
:1027500023000000230000002300000023000100EC
:1027600022000000220000002200000022000000E1
:1027700022000000220001002100000021000000D2
:1027800021000000210000002100000021000000C5
:1027900021000100200000002000000020000000B7
:1027A00020000000200000002000000020000000A9
:1027B000200001001F0000001F0000001F0000009B
:1027C0001F0000001F0000001F0000001F0001008C
:1027D0001E0000001E0000001E0000001E00000081
:1027E000393000003325000087190000B00F0000C9
:1027F000DB080000BD040000740200003F0100007F
:1028000020436F756E7420583A0023646566696EC4
:10281000652044454641554C545F000062656400A4
:102820004B6420004B6920004B702000504944202D
:102830004175746F74756E652066696E697368653D
:1028400064212050757420746865206C6173742055
:102850004B702C204B6920616E64204B6420636FA9
:102860006E7374616E74732066726F6D2062656C36
:102870006F7720696E746F20436F6E66696775723B
:102880006174696F6E2E680A005049442041757466
:102890006F74756E65206661696C6564212074696A
:1028A0006D656F75740A00504944204175746F74EA
:1028B000756E65206661696C6564212054656D7074
:1028C0006572617475726520746F6F2068696768DE
:1028D0000A00204B643A2000204B693A2000204B2C
:1028E000703A200020436C6173736963205049443F
:1028F000200A00204E6F206F76657273686F6F74C8
:102900000A002054753A2000204B753A2000206DB3
:1029100061783A2000206D696E3A200020643A20E8
:102920000020626961733A20005049442041757467
:102930006F74756E652073746172740A0050494437
:10294000204175746F74756E65206661696C65648D
:10295000212054656D706572617475726520746FA5
:102960006F20686967680A0042656400453100624B
:102970006564002C2073797374656D2073746F70B7
:1029800070656421204865617465725F49443A202E
:102990000048656174696E67204661696C65640012
:1029A00048656174696E67206661696C6564004D95
:1029B0003131322053687574646F776E001000C92E
:1029C0000210012C014001220170011801B0010E1A
:1029D00001F00104015002FA00B002F0003003E6F9
:1029E00000D003DC009004D2007005C800A006BE31
:1029F000000008B400B009AA00D00BA000600E9639
:102A00000060118C000015820020197800C01D6E36
:102A100000A0226400B0275A00902C5000003146DC
:102A200000E0343C0010383200903A2800603C1E30
:102A300000A03D1400803E0A00203F00005448459D
:102A4000524D414C2052554E4157415900546865F2
:102A5000726D616C2052756E61776179004572729A
:102A60003A204D415854454D50004D415854454D24
:102A70005020747269676765726564004572723AC6
:102A8000204D494E54454D50004D494E54454D50F2
:102A90002074726967676572656400202F002042A8
:102AA000403A0020403A0020573A0020573A004967
:102AB0006E76616C69642065787472756465720AFB
:102AC000007C3C3E5E2B3D3F2F5B5D3B2C2A225C15
:102AD0000043616E6E6F74206F70656E2073756257
:102AE0006469722000534420496E6974204661690C
:102AF0006C0053442063617264206F6B0A006F7036
:102B0000656E526F6F74206661696C65640A007649
:102B10006F6C756D652E696E6974206661696C6590
:102B2000640A004E6F20534420636172640A000AF5
:102B30004D3234004D3233202573002E0A006F7061
:102B4000656E206661696C65642C2046696C653A27
:102B5000200046696C652073656C65637465640A62
:102B6000002053697A653A200046696C65206F70D1
:102B7000656E65643A2000454E4420535542524FDD
:102B80005554494E450A002220706F730022207070
:102B90006172656E743A2200535542524F55544942
:102BA0004E452043414C4C207461726765743A2253
:102BB0000053756263616C6C204F766572666C6F52
:102BC00077004578636565646564206D617820539E
:102BD0005542524F5554494E452064657074683AC9
:102BE000002E0A0044656C6574696F6E2066616929
:102BF0006C65642C2046696C653A200046696C65FA
:102C00002064656C657465643A0053442070726991
:102C10006E74696E67206279746520004E6F74204F
:102C20005344207072696E74696E670A0057726946
:102C300074696E6720746F2066696C653A2000665F
:102C40007265736800646F696E67002066696C6501
:102C50003A20004E6F7720002F6175746F25632E28
:102C600067002020506C616E6E6572427566666505
:102C70007242797465733A20002046726565204D72
:102C8000656D6F72793A2000436F6D70696C656491
:102C90003A2041707220323420323032310A002022
:102CA0004C61737420557064617465643A203230ED
:102CB00032312D30342D3138207C20417574686FCD
:102CC000723A2054696E794D616368696E65733339
:102CD000440A00322E302E375F4457372E330A0015
:102CE0004D61726C696E0020536F66747761726516
:102CF0002052657365740A00205761746368646FBD
:102D0000672052657365740A002042726F776E20E7
:102D10006F75742052657365740A00204578746578
:102D2000726E616C2052657365740A00506F77652E
:102D30007255700A0073746172740A004732385811
:102D400059004D31303031006572726F72207772E8
:102D50006974696E6720746F2066696C650A004447
:102D60006F6E6520736176696E672066696C652E8B
:102D70000A004D323900456E6473746F707300251C
:102D80005320256320256320256320256300205AD6
:102D90003A0020593A0020583A00656E6473746F07
:102DA0007073206869743A200070012C019001272B
:102DB00001B0012201C0011D01F001180110021330
:102DC0000130020E016002090190020401C002FFFD
:102DD000000003FA004003F5008003F000D003EB8D
:102DE000002004E6007004E100E004DC004005D7A8
:102DF00000C005D2004006CD00D006C8008007C341
:102E0000003008BE00F008B900C009B400B00AAF35
:102E100000B00BAA00D00CA500000EA000500F9B24
:102E200000C01096005012910000148C00C015874D
:102E300000B0178200B0197D00D01B7800001E730F
:102E40000040206E0090226900F024640040275F5B
:102E50000090295A00E02B5500102E500020304BD6
:102E60000010324600E033410090353C0010373707
:102E70000070383200A0392D00B03A2800A03B2362
:102E800000603C1E00103D1900903D1400103E0FE4
:102E900000703E0A00C03E0500003F0000403FFBBE
:102EA000FF803FF6FFC03FF1FF00000A0B02090C54
:102EB0000D0E0807030401000000000000000000E0
:102EC0000000000000000000000000000000000002
:102ED00000000000001211100000000000000000BF
:102EE0000000000000000000000000000000005092
:102EF000726F62696E67204661696C656400205A72
:102F00003A200020593A200042656420583A2000B7
:102F10003D3D6F6E55736572436F6E6669726D529B
:102F2000657175697265643D3D00220A00556E6BDE
:102F30006E6F776E20636F6D6D616E643A20220054
:102F40002042002050006F6B00204500205A0020D6
:102F50005900204D393220580020453A00205A3A75
:102F60000020593A00583A0020746F6F206C6F6E41
:102F70006720657874727573696F6E2070726576FC
:102F8000656E7465640A0020636F6C6420657874F4
:102F9000727573696F6E2070726576656E746564A4
:102FA0000A0043616E6E6F7420656E7465722073E3
:102FB00075626469723A20004D323520500A4D32F4
:102FC0003400526573756D65005549205061757305
:102FD00065004E6F204D61746368203A005067555C
:102FE00070005067446F776E0049732046696C65C6
:102FF00020004973204469722000476F557044696E
:103000007200486173204D656469610046696C65B2
:103010006E616D652053656C6563746564004D3148
:1030200030303043004D313030300046696C616DD6
:10303000656E7420537461742030202D2033004657
:10304000696C616D656E7420537461742030202D3D
:1030500020320046696C616D656E74205374617432
:103060002030202D2031002046696C616D656E7422
:1030700020526573706F6E7365204E6F00526573DA
:10308000756D652059657320647572696E6720706F
:1030900072696E74000A204E6F2046696C616D651E
:1030A0006E7400496E76616C6964204F7074696F4C
:1030B0006E004D3530300053746F72652053657467
:1030C00074696E67730042656420504944205374EC
:1030D0006172746564004D3939390A4D32383050A7
:1030E000305331363000424C546F7563682052655E
:1030F000736574004D3530320A4D35303000496EFD
:10310000697420454550524F4D00486F74656E6498
:1031100020504944205374617274656400456E67A1
:103120006C69736820416C726561647920536574C1
:10313000004368696E657365204E6F742053757027
:10314000706F7274656400496E4C616E6743686F9E
:10315000696365000A202A2A2A7265636461742EF5
:10316000646174615B305D203D004732380A47314D
:10317000204631303030205A313000556E73757032
:10318000706F72746564204F7074696F6E20536540
:103190006C65637465640047323652323535004DD4
:1031A0003139305335350A4732380A4732390A4DFA
:1031B0003430300A4D313034533231350A473238E9
:1031C0000A4D313039533231350A4D3432305331B2
:1031D0000A4731583130305931303046353030308F
:1031E0000A47315A300A4D3530300A4D31313720D7
:1031F000536574205A204F6666736574004731200A
:103200004631303030205A302E30004732380A47AD
:1032100031204631303030205A302E30004D35309C
:1032200030005A204F6666736574203A202573007B
:103230004D353030005A204F6666736574203A2051
:103240002573004732380A473146313530305A301D
:103250002E30004732385A0A473146313530305A1D
:10326000302E30004D383400473146313030305A3E
:10327000302E30004732380A473146313030305A2C
:10328000302E30004D616E75616C53657454656D00
:1032900070005A204F6666736574203A20257300CB
:1032A00053746F7020547269676765726564005368
:1032B000746F70204E6F0053746F705072696E742B
:1032C0000048616E646C6520446174612041646AE9
:1032D00075737420322053657474696E672053636C
:1032E0007265656E200048616E646C65204461748F
:1032F00061205072696E7446696C65203320536595
:103300007474696E672053637265656E200048614E
:103310006E646C652044617461205072696E7446FD
:10332000696C6520322053657474696E672053633D
:103330007265656E20004D38340048616E646C65BE
:103340002044617461205072696E7446696C652016
:10335000506F73740048616E646C652044617461E1
:10336000205072696E7446696C6520507265004227
:103370006567696E537769746368003D3D204368F3
:1033800065636B6B65793D3D007265636461742EA6
:1033900061646472203D3D007265636461742E64F3
:1033A0006174615B305D203D3D00776169747761D8
:1033B00079203D3D0020202A2A2A2A2A2A2A5254EE
:1033C000535F48616E646C65446174612A2A2A2ADD
:1033D0002A2A2A2A2000526573656E643A2000006A
:1033E000002200250028002B002E003100340002AE
:1033F000010000050108010B010000210024002745
:10340000002A002D003000330001010000040107F4
:10341000010A01050505050705080808080202025A
:10342000020A0A080804040404010101010101015F
:10343000010303030303030303040707070C0C0C36
:103440000C0C0C0C0C02020202060606060606060E
:10345000060B0B0B0B0B0B0B0B01021020200808AB
:1034600010204010204080020102010804020101E6
:1034700002040810204080804020100804020180CF
:103480000402018040201008040201080402010126
:1034900002040810204080010204081020408054DB
:1034A0004D3344203130532050726F205265616497
:1034B000792E005072696E74696E672E2E2E005040
:1034C00072696E7420506175736564006E6F746903
:1034D0006669636174696F6E2000504944205475B9
:1034E0006E652046696E697368656400C4000201F8
:1034F00011241FBECFEFD1E2DEBFCDBF00E00CBF75
:1035000013E0A0E0B2E0E8E4FFE502E00BBF02C098
:1035100007900D92AC3FB107D9F726E1ACEFB3E0CD
:1035200001C01D92A832B207E1F71AE1C7E7DAE15C
:1035300000E006C021970109802FFE010F94D12BD6
:10354000C637D10780E00807A9F70F9448190D94F2
:10355000922F0C9400009F92AF92BF92CF92DF9275
:10356000EF92FF920F931F93CF93DF9300D01F92A0
:103570001F92CDB7DEB7EBE5FBE10027BB27462F57
:10358000572FA82FAA2341F4A52F542FB85FAA23A1
:1035900019F4A52F5527B85FA03138F45295A2959C
:1035A000452F4F70507FA42BBC5FA03428F4550FDB
:1035B000AA1F550FAA1FBE5FA03818F4550FAA1FE7
:1035C000B395550FAA1FEA0FF01F449151E0AA27A7
:1035D000B85081F1C8F0B0FF02C0440F551FB1FFD1
:1035E00004C0440F551F440F551FB2FF06C052952B
:1035F0004295142F1F70407F512BB3FF1BC0A52F86
:10360000542F44270C941A1BB195B0FF02C0559556
:103610004795B1FF04C05595479555954795B2FF1D
:1036200005C05295407F4295452B5F70B3FF02C0A5
:10363000452F5527DD24CC24BB24B2E0649FD0184D
:10364000C108B00AB00B749FC018B108B00B849FBA
:10365000B018B109659FC018B108B00B759FB018BC
:10366000B109859FB0196A9FB018B1097A9FB01946
:103670004D9DA12C99243327992722275D9DA00CCD
:10368000911C301F901F201FAD9D900C311D901F6D
:10369000201F4C9DA00C911C301F901F201F5C9D73
:1036A000900C311D901F201FAC9D300D911D201FCF
:1036B0004B9D900C311D901F201F5B9D300D911D67
:1036C000201FAB9D900D211D4B9F300D911D201F84
:1036D0005B9F900D211DAB9F200DB1E0BB24CC243E
:1036E000DD24639FD018C108B00AB00B739FC018C7
:1036F000B108B00B839FB018B109699FC018B10819
:10370000B00B799FB018B109899FB019629FB018AA
:10371000B109729FB019D61AC70AB80A20F0B1E0F1
:103720003B0F901F201F1124792F632F90E0822FD1
:103730000F900F900F900F900F90DF91CF911F91EE
:103740000F91FF90EF90DF90CF90BF90AF909F9040
:103750000895AF92BF92CF92DF92EF92FF920F93B4
:103760001F93CF93DF93C6E3DCE005EE18E086E419
:10377000A82E8CE0B82EC12CD12C7601C39469916F
:103780007991899199910F940F25288939894A89CE
:103790005B890F9470250F944D2DF80161937193FF
:1037A000819391938F01C616D706E806F90610F4A7
:1037B0006B017C01AC16BD0611F76FEF7FEFCB01FB
:1037C000A70196010F944E2B2093F5083093F6082D
:1037D0004093F7085093F808DF91CF911F910F9114
:1037E000FF90EF90DF90CF90BF90AF900895CF9271
:1037F000DF92EF92FF928091F107882309F457C07E
:10380000C090ED07D090EE07E090EF07F090F00742
:1038100020E030E0A901C701B6010F940A258823F2
:1038200009F445C020E030E040E05FE3C701B601A5
:103830000F9470259B01AC010F9470252BED3FE098
:1038400049E450E40F9470259B01AC0160E070E006
:1038500080E89FE30F94D42C6B017C01C092320C62
:10386000D092330CE092340CF092350C60916502EA
:1038700070916602072E000C880B990B0F9411258E
:103880002AE037ED43E25CE30F947025A70196012F
:103890000F947025609361027093620280936302BB
:1038A00090936402FF90EF90DF90CF900895C12C29
:1038B000D12C80E8E82E8FE3F82ED0CF0F931F9302
:1038C000CF93DF9350E0FC01E40FF51F8081440F9C
:1038D000551F440F551F49565A4FEA01882329F1B5
:1038E00088819981AA81BB81EB01088119812A8194
:1038F0003B810097A105B10569F40C591F4F2F4F6B
:103900003F4FDA010D931D932D933C9313978FEF47
:10391000808306C0081B190B2A0B3B0B37FDF7CF22
:10392000DF91CF911F910F910895188219821A8209
:103930001B82F6CFCF93DF9324E0829FC001112436
:10394000EC01C853D74FFC01E250F84F8E50984F0E
:10395000DC012D913D914D915C916081718182815D
:1039600093810F94DA2B688379838A839B83DF9119
:10397000CF9108958091920590919305A09194051F
:10398000B09195058093410290934202A093430227
:10399000B0934402809190059091910590936802B4
:1039A0008093670208958091410290914202A09114
:1039B0004302B09144028093920590939305A093A3
:1039C0009405B09395058091670290916802909359
:1039D00091058093900584E690E09093680280932F
:1039E000670208958091811290918212891B8770DD
:1039F00089F48091890D81110DC080917E0C909188
:103A00007F0C892B39F481E09091A006911103C0BD
:103A100080E0089581E00895CF93DF93DB01F90101
:103A20009C919130C1F0943080F094509C938830F8
:103A3000D1F480819181009771F001979183808307
:103A4000480F591FEA01188206C08C3539F49C5F73
:103A50009C93943041F4DF91CF9108958B3339F7E3
:103A600081E08C93F8CF20813181B9016F5F7F4F66
:103A700071836083420F531FEA01888380819181A3
:103A80008F3591056CF7E7CF0F931F9381E000917D
:103A90002514109126142091271430912814409158
:103AA000211450912214609123147091241404174E
:103AB00015072607370708F480E01F910F91089536
:103AC00090E080E00895282F9091EC07833021F456
:103AD00095FD0FC094FD0FC0892F90E0B0E0A0E0ED
:103AE00004C0B695A795979587952A95D2F78170CA
:103AF000089581E0089580E00895FC016591759135
:103B00008591949108958F929F92AF92BF92CF9298
:103B1000DF92EF92FF92CF93DF93EC018090C40885
:103B20009090C508A090C608B090C70820E030E08B
:103B3000A901C501B4010F940A25882309F454C0D2
:103B4000C880D980EA80FB80A7019601C501B40135
:103B50000F940A2518160CF04CC02091BC08309127
:103B6000BD084091BE085091BF08C701B6010F942F
:103B70000A25882331F1C092BC08D092BD08E0929A
:103B8000BE08F092BF082091C0083091C108409152
:103B9000C2085091C308688179818A819B810F9402
:103BA00070259B01AC0160E070E080E89FE30F941A
:103BB000D92B60930F02709310028093110290939F
:103BC000120260910F027091100280911102909187
:103BD0001202DF91CF91FF90EF90DF90CF90BF90D6
:103BE000AF909F908F90089560E070E080E89FE331
:103BF000F0CF60E070E0CB01ECCFCF92DF92EF929C
:103C0000FF92CF93DF93EC01CC80DD80EE80FF80CC
:103C100027E137EB41ED58EBC701B6010F943A2E7F
:103C200087FD23C023E030E04BE953E4C701B60130
:103C30000F940A251816CCF0C880D980EA80FB8042
:103C400027E137EB41ED58EBC701B6010F943A2E4F
:103C500087FD0BC0C1E023E030E84DE953E4C70124
:103C6000B6010F940A2518160CF4C0E08C2FDF91D2
:103C7000CF91FF90EF90DF90CF9008952FEB280F1A
:103C80002A3108F047C0E22FF0E080912F05909193
:103C90003005A0913105B091320504C0B695A795C5
:103CA000979587952A95D2F780FD02C08170089577
:103CB000EF5EFA4FE081EE2341F180917E07909113
:103CC0007F07E80FF92FF11D808190ED980F9A3052
:103CD00030F08E3251F4818180538A3098F4F09321
:103CE0000005E093FF0481E008958D3211F08B32DE
:103CF00049F4818190ED980F9A3088F38E3211F457
:103D00008281EACFF0E0E0E0EACF10920005109265
:103D1000FF04E9CF80E008950E943E1E882341F011
:103D200081E02091FF0430910005232B09F480E00D
:103D300008958F929F92AF92BF92CF92DF92EF92AF
:103D4000FF92C090CE05D090CF05E090D005F090C6
:103D5000D10520E030E0A901C701B6010F940A2582
:103D60008823E1F1A701960160E070E080E89FE31D
:103D70000F94D42C6B017C018090D2059090D305D8
:103D8000A090D405B090D50520E030E0A901C50190
:103D9000B4010F940A25882329F1A501940160E05C
:103DA00070E080E89FE30F94D42CC092D804D092A6
:103DB000D904E092DA04F092DB046093DC0470939F
:103DC000DD048093DE049093DF04FF90EF90DF909A
:103DD000CF90BF90AF909F908F900895C12CD12C21
:103DE0007601CACF60E070E0CB01DFCF129A089570
:103DF0005F9A8091300C8E7F8093300C8A9A8091EC
:103E0000300C8D7F8093300C8091080180958170FB
:103E1000809306018091300C8B7F8093300C0C9442
:103E2000F61E269A2E9A08958C3221E0920714F0FD
:103E30008CE291E09093E6118093E5110C94EFFCF5
:103E4000EAE0F6E0108211821282138214820C944E
:103E5000EFFC4F925F926F927F928F929F92AF9200
:103E6000BF92CF92DF92EF92FF920F931F93CF9367
:103E7000DF93EC012091C6053091C7054091C8053C
:103E80005091C905688179818A819B810F94D92BD2
:103E90006B017C012091CA053091CB054091CC0586
:103EA0005091CD056C817D818E819F810F94D92B9E
:103EB0004B015C01A701960160910302709104021D
:103EC00080910502909106020F940A25882309F437
:103ED00050C0C0920302D0920402E0920502F09218
:103EE00006022091D8043091D9044091DA0450910F
:103EF000DB04C701B6010F9470252B013C010F9420
:103F00007C2D6B017C0120E030E0A9010F940A2593
:103F100087FD70C020E030E040E450E4C701B60106
:103F20000F943A2E18162CF4C12CD12CC0E4EC2E90
:103F3000FE2CA7019601C301B2010F94D92B609307
:103F4000D0047093D1048093D2049093D304C7011A
:103F5000B6010F94462D6093CE04062E000C770B0D
:103F60006F5F7F4F6430710514F064E070E0609320
:103F7000CC04D09101021091CE04A501940160916E
:103F80000702709108028091090290910A020F9431
:103F90000A25811133C0D11381C02091B40430911E
:103FA000B5044091B6045091B7046091D00470916B
:103FB000D1048091D2049091D3040F947025209164
:103FC000B8043091B9044091BA045091BB040F94E5
:103FD000DA2BDF91CF911F910F91FF90EF90DF903F
:103FE000CF90BF90AF909F908F907F906F905F9099
:103FF0004F900895C12CD12C76019BCF809207025F
:1040000090920802A0920902B0920A022091DC0468
:104010003091DD044091DE045091DF04C501B4010C
:104020000F9470254B015C010F947C2D6B017C017A
:1040300020E030E0A9010F940A2587FDF3C020E0BD
:1040400030E040E450E4C701B6010F943A2E181650
:104050002CF4C12CD12CB0E4EB2EFE2CA701960140
:10406000C501B4010F94D92B6093D4047093D50487
:104070008093D6049093D704C701B6010F94462DC0
:104080006093CF04062E000C770B6F5F7F4F643078
:10409000710514F064E070E06093CD04C091CF042A
:1040A000D11305C0809102028C1709F470C0809171
:1040B000CE049091CF0490930202809301020C2EC3
:1040C000000CDD0B25E01203C0011124FC01EC0FF4
:1040D000FD1FEE0FFF1FEE0FFF1FE857F84F208167
:1040E0003181428153812093C8043093C9044093A5
:1040F000CA045093CB040091CD04002E000C110B88
:10410000FC01E00FF11FEE0FFF1FEE0FFF1FE8573E
:10411000F84F60817181828193810F94D92B6093D4
:10412000C4047093C5048093C6049093C70420917F
:10413000CC0435E02303F0011124CE0FDF1FCC0F98
:10414000DD1FCC0FDD1FC857D84F288139814A8128
:104150005B812093C0043093C1044093C204509308
:10416000C304E00FF11FEE0FFF1FEE0FFF1FE85714
:10417000F84F60817181828193810F94D92B609374
:10418000BC047093BD048093BE049093BF048090E0
:10419000D4049090D504A090D604B090D704209178
:1041A000C4043091C5044091C6045091C704C501B0
:1041B000B4010F9470252091C8043091C904409136
:1041C000CA045091CB040F94DA2B6B017C01C0928E
:1041D000B804D092B904E092BA04F092BB042091E2
:1041E000BC043091BD044091BE045091BF04C50190
:1041F000B4010F9470252091C0043091C104409106
:10420000C2045091C3040F94DA2BA70196010F94B6
:10421000D92B6093B4047093B5048093B604909343
:10422000B704BBCEC12CD12C760118CFCF92DF9230
:10423000EF92FF92CF93DF93EC0108960E94831DCB
:104240006B017C0120E030E0A9010F940A2520E0F9
:1042500030E0A901882359F0CE010E94291F9B015B
:10426000AC01C701B6010F9470259B01AC016885B4
:1042700079858A859B850F94D92B688779878A876A
:104280009B87DF91CF91FF90EF90DF90CF900895C3
:104290002F923F924F925F926F927F928F929F9256
:1042A000AF92BF92CF92DF92EF92FF920F931F9344
:1042B000CF93DF93D62FC72FFC0180809180A280FF
:1042C000B380C501B40120E831E541E050E00F942E
:1042D0004E2BC9016DE671E00F94BD2B6B017C0183
:1042E000C501B40120E13EE040E050E00F944E2BC8
:1042F000CA01B90128E130E040E050E00F944E2BB4
:10430000362E272E062F172F8CE3482E512C612C8A
:10431000712CC501B401A30192010F944E2BB62E4E
:10432000A72ECA01B901A30192010F944E2BCB0114
:10433000C114D10479F1AF92BF927F936F932F9202
:104340003F92FF92EF92DF92CF9282E697E19F93A6
:104350008F93CF93DF930F94A1248DB79EB70E96C2
:104360000FB6F8949EBF0FBE8DBF8D2F9C2FDF918F
:10437000CF911F910F91FF90EF90DF90CF90BF9062
:10438000AF909F908F907F906F905F904F903F90F5
:104390002F900895E114F104C9F0AF92BF927F937A
:1043A0006F932F923F92FF92EF9282E597E19F9356
:1043B0008F93CF93DF930F94A124EDB7FEB73C9674
:1043C0000FB6F894FEBF0FBEEDBFCFCF012BB9F0F3
:1043D000AF92BF927F936F932F923F9286E497E1C3
:1043E0009F938F93CF93DF930F94A1248DB79EB7A4
:1043F0000A960FB6F8949EBF0FBE8DBFB6CF892B1D
:10440000A9F0AF92BF927F936F938EE397E19F9352
:104410008F93CF93DF930F94A124EDB7FEB7389617
:104420000FB6F894FEBF0FBEEDBF9FCFAF92BF9205
:104430008AE397E19F938F93CF93DF930F94A12407
:104440000F900F900F900F900F900F908ECFEF92D4
:10445000FF920F931F93CF93DF93CDB7DEB78C01FD
:10446000EDB6FEB60F94572401962DB73EB7281B24
:10447000390B0FB6F8943EBF0FBE2DBF8DB79EB758
:104480000196B8010F9450240E9412F90FB6F894C7
:10449000FEBE0FBEEDBEDF91CF911F910F91FF9039
:1044A000EF9008958C38910514F08CE890E090938B
:1044B0007B1180937A110C948CBEAB01BC014093AC
:1044C00025145093261460932714709328148DE8B4
:1044D00095E10C9444AF2F923F924F925F926F926E
:1044E0007F928F929F92AF92BF92CF92DF92EF9284
:1044F000FF920F931F93CF93DF93CDB7DEB76097F3
:104500000FB6F894DEBF0FBECDBF8B876C87042F2C
:10451000122F282F30E03E872D87462F50E05A87F4
:10452000498785E0982E929EC001939E900D11249C
:10453000988B8F87FA01E80FF91FEE0FFF1FEE0F20
:10454000FF1FE857F84F60817181828193819B0141
:10455000AC010F94CC2E882309F445C14B85400F44
:104560006C85610F949EC0011124E985FA85E80FDE
:10457000F91FEE0FFF1FEE0FFF1FE857F84FC08027
:10458000D180E280F380040F909EA0011124E98580
:10459000FA85E40FF51FEE0FFF1FEE0FFF1FE85720
:1045A000F84F0081918082807380262F30E0EF8564
:1045B000F889E20FF31FEE0FFF1FEE0FFF1FE85702
:1045C000F84F20807181798372817A8373817B8334
:1045D000610F70E0EF85F889E60FF71FEE0FFF1F00
:1045E000EE0FFF1FE857F84FF88BEF87F081FC8341
:1045F000EF85F889F181FD83EF85F889F281FE83EB
:10460000EF85F889F381FF83FC01E20FF31FEE0FC2
:10461000FF1FEE0FFF1FE857F84F20812887A1806A
:10462000B2806380FA01E60FF71FEE0FFF1FEE0F57
:10463000FF1FE857F84F4080518032801381202FB0
:10464000392D482D572D602F792D882D972D0F94BA
:10465000CC2E882321F000E0912C812C712C960126
:10466000A701B601C7010F94CC2E882321F0C02EDC
:10467000D92CE82CF72C2C813D814E815F816C81F7
:104680007D818E819F810F94CC2E882321F01C8206
:104690001D821E821F82222D39814A815B81622DFB
:1046A00079818A819B810F94CC2E882339F02C80CC
:1046B0003D8139834E814A835F815B839201432D23
:1046C000512FB201832D912F0F94CC2E882321F0EE
:1046D000412C512C312C10E028853A2D4B2D562D94
:1046E00068857A2D8B2D962D0F94CC2E882321F062
:1046F0004886A52CB32C612E85E02D853E85829FB2
:10470000F001839FF00D112449855A85E40FF51FB0
:10471000EE0FFF1FEE0FFF1FE857F84FFA87E987EC
:104720009601A701B601C7010F94DA2B202F392D6E
:10473000482D572D0F94D92B6B017C01222D3981E7
:104740004A815B81622D79818A819B810F94DA2B6A
:104750002C813D814E815F810F94D92B9B01AC014F
:10476000C701B6010F94DA2B6B017C0128853A2D25
:104770004B2D562D68857A2D8B2D962D0F94DA2B87
:104780009201432D512F0F94D92B9B01AC01C701EE
:10479000B6010F94DA2B20E030E040E450E40F94AF
:1047A000D42CE985FA8560837183828393836C8539
:1047B0008B8560960FB6F894DEBF0FBECDBFDF913C
:1047C000CF911F910F91FF90EF90DF90CF90BF900E
:1047D000AF909F908F907F906F905F904F903F90A1
:1047E0002F900C94A5F760960FB6F894DEBF0FBE1D
:1047F000CDBFDF91CF911F910F91FF90EF90DF9090
:10480000CF90BF90AF909F908F907F906F905F9070
:104810004F903F902F9008958091FF049091000554
:10482000009731F04AE050E070E060E00D942523FD
:1048300060E070E0CB0108958091FF049091000545
:10484000009731F04AE050E070E060E00D94F7210D
:1048500060E070E0CB010895CF93DF93EB010E94FD
:104860008C1E882319F00E941C24EB01CE01DF91DD
:10487000CF9108950E941C2497FD0CC00E941C2417
:104880006F3F71058105910509F034F40E941C24E5
:10489000862F089580E008958FEF0895CF93C62F57
:1048A0000E948C1E882319F0CF910C943A248C2FEF
:1048B000CF9108958091FF0490910005892B41F0DC
:1048C0000E943A2491E0811101C090E0892F08955F
:1048D00091E0FCCFCF93DF93C82FD62F0E948C1E80
:1048E000882321F0DF91CF910C945A248C2F0E94C1
:1048F0003E1E811101C08D2FDF91CF9108950E943E
:104900001C24CB010895CF93DF93EB010E948C1EF2
:10491000882321F0DF91CF910C947F24CE01DF9189
:10492000CF9108950F931F93CF938091FF0490919F
:1049300000050097E9F0FC018F01C1912C2F2F7D1C
:1049400081F0C53411F0C536B9F7F801108270E076
:1049500060E00F949920F801C083CF911F910F91CF
:10496000089570E060E0CF911F910F910D94992010
:1049700060E070E0CB01F1CFCF92DF92EF92FF9237
:104980006A017B010E948C1E882331F0FF90EF901A
:10499000DF90CF900C949224C701B601FF90EF9066
:1049A000DF90CF9008954F925F926F927F928F9297
:1049B0009F92AF92BF92CF92DF92EF92FF921F939E
:1049C000CF93DF9300D01F92CDB7DEB719821A8242
:1049D0001B821C82CE0101964C018CE6C82E87E01A
:1049E000D82E90E2E92E9CE0F92E28ECA22E28E0A9
:1049F000B22E10E088E5810F0E948C1EF401819395
:104A00004F01882309F4E0C00E9492242B013C014D
:104A1000812F0E94631D882309F4CCC0F7012081F7
:104A2000318142815381C301B2010F94DA2BF60127
:104A300060837183828393831F5FF4E0CF0ED11C68
:104A400084E0E80EF11C94E0A90EB11C133091F63D
:104A500085E40E948C1E8C83882309F4C0C00E94C8
:104A600092246B017C0183E00E94631D882371F016
:104A700020912C0C30912D0C40912E0C50912F0C2C
:104A8000C701B6010F94DA2B6B017C01C092780745
:104A9000D0927907E0927A07F0927B078091C50562
:104AA000882359F18091291482FF27C08C818823A3
:104AB00021F18981811103C08A818823F1F02DECD5
:104AC0003CEC4CE45DE36091130870911408809114
:104AD0001508909116080F94DA2B9B01AC01609198
:104AE000280C7091290C80912A0C90912B0C0F941A
:104AF0003A2E181614F40E94EBF640E050E0BA018A
:104B000086E40E94BC2420E030E0A9010F943A2EF4
:104B1000181684F40E94922420E030E040E752E42A
:104B20000F94D42C6093410270934202809343020D
:104B3000909344028091DE0B83FD28C080918B0608
:104B4000882321F120912C0C30912D0C40912E0CBA
:104B500050912F0C609178077091790780917A07B6
:104B600090917B070F94D92B20919806309199064C
:104B700040919A0650919B060F94DA2B6093980609
:104B80007093990680939A0690939B060F900F90CE
:104B90000F900F90DF91CF911F91FF90EF90DF90DA
:104BA000CF90BF90AF909F908F907F906F905F90CD
:104BB0004F900895F5012081318142815381C301D5
:104BC000B2010F94D92B33CFF70180819181A2815B
:104BD000B381F60180839183A283B3832DCF80912B
:104BE0002C0C90912D0CA0912E0CB0912F0C809339
:104BF000780790937907A0937A07B0937B074ECFFD
:104C0000CF92DF92EF92FF926B017C0183E3C81693
:104C1000D104E104F10470F082E3C81AD108E1087C
:104C2000F10862E370E080E090E00E94B0FC0E9436
:104C300006C2ECCFC701B6010E94B0FCFF90EF9016
:104C4000DF90CF900C9406C2CF92DF92EF92FF924A
:104C50000F931F93CF93DF936B017A01EC01CC5636
:104C6000DB4F28813CE0389F8001399F100D1124D3
:104C700027FF24C0FB011182108288818F5F888307
:104C800088819801280F311D87FD3A95C90120912F
:104C90006C12F6012817190629F024F088818C304F
:104CA0000CF43CC080819181049680349C4908F4C6
:104CB00075C0F60180819181049672C08881980147
:104CC000280F311D87FD3A95C90120916C122817D4
:104CD000190699F294F28881A801480F511D87FDA9
:104CE0005A95FA01EE0FFF1FE40FF51FEC5DFD4E24
:104CF000808187FFC2CF8881F801E80FF11D87FD11
:104D0000FA95CF01EE0FFF1FE80FF91FEC5DFD4E86
:104D1000808160E08F770E944EFBAFCF80819181D0
:104D20002881A801420F511D27FD5A959A01FA01C9
:104D3000EE0FFF1FE20FF31FEC5DFD4E218132816C
:104D4000820F931FF7019183808388819801280F38
:104D5000311D87FD3A95F901EE0FFF1FE20FF31F9A
:104D6000EC5DFD4E808187FF20C08881080F111DFA
:104D700087FD1A95F801EE0FFF1FE00FF11FEC5DA4
:104D8000FD4E808161E08F77DF91CF911F910F9170
:104D9000FF90EF90DF90CF900C944EFB80E49CE965
:104DA000F701918380838FEF8883DF91CF911F91EB
:104DB0000F91FF90EF90DF90CF9008950F931F9386
:104DC000CF93DF930AE41CE0CEE5D1E1F801219115
:104DD0003191419151918F0160E070E080E89FE353
:104DE0000F94D42C6993799389939993F1E1CE36FA
:104DF000DF0761F70E942AF5DF91CF911F910F9194
:104E00000C94A91BCF92DF92EF92FF92CF93DF9386
:104E10002091310C222329F1EC0108960E94831D78
:104E20006B017C0120E030E0A9010F940A2520E00D
:104E300030E0A901882359F0CE010E94291F9B016F
:104E4000AC01C701B6010F9470259B01AC016885C8
:104E500079858A859B850F94DA2B688779878A877D
:104E60009B87DF91CF91FF90EF90DF90CF900895D7
:104E70002F923F924F925F926F927F928F929F926A
:104E8000AF92BF92CF92DF92EF92FF920F931F9358
:104E9000CF93DF93CDB7DEB76C970FB6F894DEBF34
:104EA0000FBECDBF8C015B015A834983FC01EA5BD5
:104EB000FF4F208131814281538129873A874B8777
:104EC0005C87CA01B9010F940F256B017C01D501E4
:104ED0002D913D914D915C910F9470250F94B82CBC
:104EE0002B013C01E981FA8120813181428153818A
:104EF000C701B6010F9470250F94B82C4B015C01CB
:104F0000C301B2010F944D2D698B7A8B8B8B9C8BD7
:104F1000683771058105910540F428E730E040E0ED
:104F200050E0298B3A8B4B8B5C8BC501B4010F94FD
:104F30004D2D6D877E878F87988B6837710581052A
:104F4000910540F448E750E060E070E04D875E87EF
:104F50006F87788BF801EE5AFF4F40805180628056
:104F60007380C301B2010F94112569837A838B8307
:104F70009C8369897A898B899C890F940F256D8B15
:104F80007E8B8F8B988F20E030E0A90169817A8138
:104F90008B819C810F940A25882309F4E1C1A70124
:104FA0009601C701B6010F9470254B015C012D8954
:104FB0003E894F89588DCA01B9010F9470259B0114
:104FC000AC01C501B4010F94D92B4B015C012981BF
:104FD0003A814B815C81CA01B9010F94DA2B9B01A4
:104FE000AC01C501B4010F94D42C0F94B82C0F94CC
:104FF0004D2D6D837E838F83988766277727CB011E
:1050000064197509860997090F9411254B015C01F4
:105010006D857E858F8598890F940F252B013C0126
:1050200020E030E0A901C501B4010F940A258823CE
:1050300009F49AC1A3019201C301B2010F94702532
:10504000698F7A8F8B8F9C8FA7019601C701B6015C
:105050000F9470259B01AC01698D7A8D8B8D9C8D91
:105060000F94D92B6B017C01A5019401C501B401FA
:105070000F94DA2B9B01AC01C701B6010F94D42C1D
:105080000F947C2DD80195968D909D90AD90BC90FD
:105090009897750164012D813E814F815885C21A10
:1050A000D30AE40AF50A0F944D2DC61AD70AE80A66
:1050B000F90AF7FE8EC02D893E894F89588DCA01A5
:1050C000B9010F9470256B017C0129813A814B81D4
:1050D0005C81CA01B9010F94DA2B69877A878B87C3
:1050E0009C8720E030E0A90169817A818B819C81D5
:1050F0000F940A25882309F43BC1C501B4010F941C
:105100000F2529853A854B855C850F947025A7016D
:1051100096010F94D92B6D837E838F839887A3018B
:105120009201C301B2010F9470259B01AC016D8106
:105130007E818F8198850F94DA2B2B013C0120E032
:1051400030E040E850E469817A818B819C810F9442
:1051500070259B01AC01C301B2010F94D42C0F94B4
:10516000B82C2B013C0120E030E0A9010F943A2E2D
:1051700018161CF0412C512C3201C301B2010F94BE
:105180004D2D6D837E838F83988786169706A8069C
:10519000B90620F48D829E82AF82B8866D817E81B1
:1051A0008F8198850F940F2529853A854B855C85DD
:1051B0000F947025A70196010F94DA2B0F94882E77
:1051C0000F944D2D69877A878B879C87C12CD12CB2
:1051D000760169857A858B859C8529893A894B89F1
:1051E0005C89621B730B840B950B0F940F2529812F
:1051F0003A814B815C810F94D42C20E034E244EF5F
:1052000059E40F9470250F944D2D4B015C01698575
:105210007A858B859C852D853E854F855889621BB7
:10522000730B840B950B0F940F2529813A814B81C9
:105230005C810F94D42C20E034E244EF59E40F94C5
:1052400070250F944D2D2B013C013FE683169104F0
:10525000A104B10408F090C0F401EE0FFF1FEE0F9F
:10526000FF1FE156F64E85919591A591B4918983E2
:10527000292E3A2EBD8B4FE6441651046104710469
:1052800008F083C0F201EE0FFF1FEE0FFF1FE15683
:10529000F64E45915591659174919A01CB014D81DE
:1052A0005E816F817885D80199964D935D936D935A
:1052B0007C939C974C0D5D1D6E1D7F1DF80145A7CD
:1052C00056A767A770ABE65BFF4F49895A896B8980
:1052D0007C894083518362837383D5968D929D929E
:1052E000AD92BC92D897F80141AE52AE63AE74AEA7
:1052F000FD9649814083218232825D8953833496B1
:10530000208331838283938369857A858B859C850D
:10531000D1966D937D938D939C93D4973D962D85D7
:105320003E854F85588920833183428353836C9611
:105330000FB6F894DEBF0FBECDBFDF91CF911F91A6
:105340000F91FF90EF90DF90CF90BF90AF909F9024
:105350008F907F906F905F904F903F902F90089527
:1053600060E070E0CB0141CE60E070E0CB0188CE20
:1053700060E070E0CB01F3CEC501B4010E94AB1A2E
:105380006983272E382E9D8B76CFC301B2010E94F0
:10539000AB1A9B0184CF8091811290918212891B5C
:1053A000877019F490E080E0089590917E1299231F
:1053B00051F0833030F48FEF890F19F080937E1213
:1053C000F1CF10927E12809182122CE5829FC00153
:1053D00011248250974FFC01208120FDE3CF2091C2
:1053E00082122F5F277020937F12309182122091BA
:1053F0008012321304C020917F12209380120895EE
:1054000090916F0081E091FD02C080E0089590913D
:105410006F009D7F90936F00089580FF04C090916E
:10542000960590FD8E7F81FF05C09091960596951B
:1054300090FD8D7F82FF06C090919605969596957A
:1054400090FD8B7F08958F929F92AF92BF92CF92E3
:10545000DF92EF92FF92CF93DF93209145022223B8
:1054600009F49EC0EC0180919605C82ED12CF12C38
:10547000E12C80FF2CC08090470290904802A090C1
:105480004902B0904A02288139814A815B81C50175
:10549000B4010F943A2E181624F488829982AA82B5
:1054A000BB828090530290905402A0905502B0901D
:1054B0005602288139814A815B81C501B4010F946C
:1054C0000A2587FF04C088829982AA82BB82D701FD
:1054D000C601B695A7959795879580FF2CC08090BB
:1054E0004B0290904C02A0904D02B0904E022C8145
:1054F0003D814E815F81C501B4010F943A2E18168B
:1055000024F48C829D82AE82BF828090570290905C
:105510005802A0905902B0905A022C813D814E81D0
:105520005F81C501B4010F940A2587FF04C08C82F6
:105530009D82AE82BF8282E0F694E794D794C794AE
:105540008A95D1F7C0FE2CC0C0904F02D090500277
:10555000E0905102F0905202288539854A855B859A
:10556000C701B6010F943A2E181624F4C886D986BE
:10557000EA86FB86C0905B02D0905C02E0905D0200
:10558000F0905E02288539854A855B85C701B601A2
:105590000F940A2587FF04C0C886D986EA86FB8651
:1055A000DF91CF91FF90EF90DF90CF90BF90AF90C1
:1055B0009F908F900895CF92DF92EF92FF920F937A
:1055C0001F93C12CD12C76018C012CE23CE048E2E7
:1055D0005CE064E27CE080E29CE00E9426F41F91A3
:1055E0000F91FF90EF90DF90CF9008950C942AF5E3
:1055F00080919D06811105C080917C07882309F464
:1056000063C080918305659B59C081608093830549
:10561000909103018091830591FF52C08260809335
:105620008305809183054B9B4DC0846080938305E7
:105630008091EA0580FF10C080919E0680FF0CC01B
:105640008091830580FF08C08091E006816080938F
:10565000E00680E00E9466C68091EA05869580FF9C
:1056600011C080919E06869580FF0CC080918305B5
:1056700081FF08C08091E00682608093E00681E0AF
:105680000E9466C68091EA058695869580FF1CC0BB
:1056900080919E068695869580FF16C080917C0736
:1056A000882391F08091830582FF0EC08091E006EF
:1056B00084608093E00682E00C9466C68E7FA6CF5D
:1056C0008D7FADCF8B7FB2CF089580919D068111E4
:1056D00004C080917C07882331F062E070E080E0B4
:1056E00090E00C94002608950F931F9380911C1155
:1056F000813019F50E94E3FC00919F051091A005EF
:105700002091A1053091A205601B710B820B930BB8
:1057100028EE33E040E050E00F944E2B6091A3055B
:105720007091A4058091A5059091A605620F731F45
:10573000841F951F1F910F9108956091A705709187
:10574000A8058091A9059091AA05D6CF10921C11A9
:1057500010929F051092A0051092A1051092A2052B
:105760001092A7051092A8051092A9051092AA05FB
:105770001092A3051092A4051092A5051092A605FB
:105780000895CF92DF92EF92FF92CF93DF93C62FCF
:10579000FC01C080D180E280F38020E030E0A901EC
:1057A000C701B6010F940A2520E030E0A90187FD6A
:1057B00014C020E030E048EC52E4C701B6010F9479
:1057C0003A2E24E630E040E050E0181634F0C701ED
:1057D000B6010F94462D9B01AC01C230A0F4D0E07D
:1057E000C750D74FAFEFB0E00F948F2B24E630E0D7
:1057F00040E050E00F94702B2F3F310519F010F06E
:105800002FEF30E02883DF91CF91FF90EF90DF9072
:10581000CF9008958091090180FD06C080912914E0
:1058200083FB882780F9089580E00895CF92DF9266
:10583000EF92FF92FC01C080D180E280F38066305D
:1058400019F510920F061092100610921106109280
:105850001206109213060E948CBE20E030E0A901CF
:10586000C701B6010F940A2587FF1DC0C12CD12C9A
:105870007601C701B6010F94472ECB01FF90EF9040
:10588000DF90CF900C9452220E94201F20E030E045
:10589000A901C701B6010F940A2587FF15C0C12CC5
:1058A000D12C760121C020E030E04CE053E4C70168
:1058B000B6010F943A2E1816E4F6C12CD12C9CE0B8
:1058C000E92E93E4F92ED5CF20E030E046E953E409
:1058D000C701B6010F943A2E181634F4C12CD12CFE
:1058E00086E9E82E83E4F82EC701B6010F94472E0F
:1058F000CB01FF90EF90DF90CF900C94141F90910C
:10590000300C977081E0973009F080E00895209185
:10591000810520FF14C020E83EE3629FA001639F41
:10592000500D729F500D1124CA019695879596953A
:105930008795009731F08A950000E9F708950C9457
:1059400000260895CF93DF931092DF0B1092820C04
:105950001092840C1092830C1092800510927F0597
:10596000CFEFDFEF8091291485FD07C00E94A5AA23
:10597000D093A812C093A712F5CF8FEF9FEF90930B
:10598000A8128093A712DF91CF9108958F929F92D2
:10599000AF92BF92CF92DF92EF92FF920F931F933D
:1059A000CF93DF9310923405109233052FE32093A9
:1059B0002E0510922D0510922C0510922B05109299
:1059C0002F051092300510923105109232059C017E
:1059D000F90190812F5F3F4F9032D1F39E34C9F48B
:1059E000818190ED980F9A3020F08D3211F08B323A
:1059F00081F432969F012F5F3F4F808180538A3020
:105A000008F47BC09F012F5F3F4F8081803209F4F3
:105A100076C0F0937F07E0937E078F010F5F1F4FE3
:105A2000C0816AE270E0C8010F94282F009731F01E
:105A3000FC01319780818032E1F31182CD3429F06D
:105A4000C43519F0C73409F04BC0F80180810F5FED
:105A50001F4F8032D1F380538A3008F041C0C09389
:105A60002E0530E020E04AE0DF011196429FC001A0
:105A7000439F900D11249C01205331098081280FF0
:105A8000311D87FD3A95818190ED980F9A30C8F1CC
:105A900030932D0520932C058E3261F4329690E0E0
:105AA0004AE0DF0131968C9150ED580F5A3058F191
:105AB00090932B05CD01DC0101964C914032D9F336
:105AC000CD3489F52E31310539F018F527313105FE
:105AD00019F02C31310539F5B0933405A093330515
:105AE000DF91CF911F910F91FF90EF90DF90CF90BA
:105AF000BF90AF909F908F900895F9017BCFF901EF
:105B000081CFFD01B1CF949F800D112490ED980FAE
:105B1000C8CF2537310538F027373105E8F2203A6C
:105B200083E03807C9F2D0917E0740E050E0BA0127
:105B300010E000E0C12CD12C7601C394FD01319618
:105B40008C91882309F47FC08132E1F4CD34D1F403
:105B500020323105B9F440932F05509330056093FE
:105B6000310570933205F0933405E093330563E219
:105B700070E0CF010F94282F009709F4B1CFFC01FA
:105B80001082AECF81548A3108F058C0DF019D9158
:105B9000903291F0A0EDA90FAA30E8F09E3271F496
:105BA000918190539A30B8F00115110519F48F01C5
:105BB0000150110990E013C0FD01E8CF9D3211F0B2
:105BC0009B3291F79181A0EDA90FAA3020F09E326F
:105BD00059F79281E6CF9E2F9D1B309759F3A82F3E
:105BE000B0E04601570104C0880C991CAA1CBB1CDC
:105BF0008A95D2F7482959296A297B29AF5EBA4F7D
:105C00009C9380818154DF018A3108F497CFDF01B2
:105C10008191882309F492CF90ED980F9A30B8F3D0
:105C200093ED980F923098F38B3289F3CD01019662
:105C3000EC91E03209F082CFDC01F8CF01151105BB
:105C400001F78D01DECF10933405009333054093A7
:105C50002F0550933005609331057093320540CF86
:105C60004F925F926F927F928F929F92AF92BF926C
:105C7000CF92DF92EF92FF92CF93DF9300D000D0CC
:105C80001F921F92CDB7DEB75C01DB01CD90DD9096
:105C9000ED90FC90E0917C12F0917D12FE83ED83FB
:105CA00084819581A681B78189839A83AB83BC83E4
:105CB0009C01AD01C701B6010F94D92B2B013C010A
:105CC000F50180809180A280B380AD81BE818D91ED
:105CD0009D910D90BC91A02D8D839E83AF83B8873D
:105CE00027E137EB41ED58EBC301B2010F943A2E97
:105CF00087FDD2C023E030E04BE953E4C301B20199
:105D00000F940A2518160CF4C7C02D813E814F81CF
:105D10005885C501B4010F94D92B2B013C0127E113
:105D200037EB41ED58EB0F943A2E87FDB5C023E0D9
:105D300030E84DE953E4C301B2010F940A25181667
:105D40000CF4AAC020E030E0A9016D817E818F8132
:105D500098850F94DA2B2B013C0120E030E040E4E1
:105D600050E40F940A2587FF05C0412C512C30E4E4
:105D7000632E762C27E137EB41ED58E3C301B201E6
:105D80000F94D92B9B01AC01C501B4010F943A2E9D
:105D900087FD82C020E030E84DE953E46D817E81CB
:105DA0008F8198850F94DA2B2B013C0120E030E89D
:105DB00044E953E40F943A2E18163CF4412C20E8A1
:105DC000522E24E9622E23E4722E27E137EB41EDB7
:105DD00058E3C301B2010F94DA2B9B01AC01C5015A
:105DE000B4010F940A2518160CF456C020E030E0D8
:105DF000A90169817A818B819C810F94DA2B4B01F7
:105E00005C0120E030E040E551E40F940A2587FF73
:105E100006C0812C912C90E5A92E91E4B92E27E1A2
:105E200037EB41ED58E3C501B4010F94D92B9B0129
:105E3000AC01C701B6010F943A2E87FD2DC020E0BA
:105E400030E04BE953E469817A818B819C810F9426
:105E5000DA2B4B015C0120E030E84FE853E40F946B
:105E60003A2E18163CF4812C80E8982E8FE8A82E44
:105E700083E4B82E27E137EB41ED58E3C501B401C7
:105E80000F94DA2B9B01AC01B1E0B983C701B601D5
:105E90000F940A2518160CF41982898128960FB6DA
:105EA000F894DEBF0FBECDBFDF91CF91FF90EF9092
:105EB000DF90CF90BF90AF909F908F907F906F902A
:105EC0005F904F900895EAE0F8E082EBDF011D92C9
:105ED0008A95E9F708958091C505811104C00E9453
:105EE000632F0C9406B88091291482FD0C94EBF674
:105EF000089580910A08882361F09091BB08891366
:105F000008C08091291483FF04C088E498E00C94B1
:105F1000D0B680E00895FC01238121110C9405B3D3
:105F20000895EFE6F0E08081826080830895CF924B
:105F3000DF92EF92FF92CF93DF93C82F0E94002A47
:105F400094E0C99FE0011124FE01E850FA4FC0809F
:105F5000D180E280F38081110E94912FC25ADE4EDF
:105F6000C701B6010F941125288139814A815B81CF
:105F70000F947025DF91CF91FF90EF90DF90CF903D
:105F800008958F929F92AF92BF92CF92DF92EF923D
:105F9000FF921F93CF93DF93CDB7DEB760970FB615
:105FA000F894DEBF0FBECDBF182F80E00E94972F60
:105FB0004B015C018092840590928505A092860534
:105FC000B092870581E00E94972F6B017C01C092FF
:105FD0008805D0928905E0928A05F0928B0582E0CF
:105FE0000E94972F60938C0570938D0580938E058A
:105FF00090938F051D861E861F86188A89829A8235
:10600000AB82BC82CD82DE82EF82F88669877A8796
:106010008B879C8783E00E94972F6D877E878F8771
:10602000988B8091310C882321F0CE0101960E943B
:1060300016211E3FD9F480E1FE013196A0E2BCE0BA
:1060400001900D928A95E1F760960FB6F894DEBF45
:106050000FBECDBFDF91CF911F91FF90EF90DF90EA
:10606000CF90BF90AF909F908F90089584E0189F3D
:10607000F0011124DF01A05EB34F81E090E08C0FAE
:106080009D1FE80FF91F40815181628173814D93FB
:106090005D936D937C931397D7CFCF92DF92EF925E
:1060A000FF92CF93DF93C82F0E94002A94E0C99FEC
:1060B000E0011124FE01E451FA4FC080D180E2805A
:1060C000F38081110E94912FC25ADE4EC701B601A2
:1060D0000F941125288139814A815B810F947025A5
:1060E000DF91CF91FF90EF90DF90CF9008950E94C5
:1060F000002A909182129093811290938012909333
:106100007F1294E690937E1220ED33E03093FD08E9
:106110002093FC0881110E94912F81E08093EB0570
:106120000895CF93DF93CDB7DEB72C970FB6F894D1
:10613000DEBF0FBECDBF0E9408F60E94002A9CE081
:10614000E8EFF5E0DE01119601900D929A95E1F7E6
:1061500081110E94912FCE0101960E9446C62C9675
:106160000FB6F894DEBF0FBECDBFDF91CF9108957B
:106170002F923F924F925F926F927F928F929F9257
:10618000AF92BF92CF92DF92EF92FF920F931F9345
:10619000CF93DF9300D0CDB7DEB78090200C9090E6
:1061A000210CA090220CB090230C4090240C509015
:1061B000250C6090260C7090270CC090280CD09075
:1061C000290CE0902A0CF0902B0C0E94A91B0E9435
:1061D000F71B0FE71CE187E492E09B838A8383E748
:1061E000282E8CE1382E198289810E949A1CC801C0
:1061F0000E947D1DEA81FB8161937193819391934C
:10620000FB83EA83C1010E947D1DEA81FB816087D7
:10621000718782879387F981FF5FF9830C5F1F4F36
:1062200084E0280E311CF330F9F686ED95E00E94EB
:106230006DF60E94991E0E94DE26A50194016091D0
:10624000200C7091210C8091220C9091230C0F94C2
:106250000A2581111CC0A30192016091240C709148
:10626000250C8091260C9091270C0F940A25811102
:106270000EC02091280C3091290C40912A0C50918D
:106280002B0CC701B6010F940A258823B9F00F9093
:106290000F900F90DF91CF911F910F91FF90EF9092
:1062A000DF90CF90BF90AF909F908F907F906F9036
:1062B0005F904F903F902F900C9491300F900F90E3
:1062C0000F90DF91CF911F910F91FF90EF90DF9092
:1062D000CF90BF90AF909F908F907F906F905F9086
:1062E0004F903F902F90089580917211909173116B
:1062F000892B79F48091721190917311892B49F453
:10630000209172113091731181E0232B19F480E0F8
:10631000089581E008951092E50480912202909101
:106320002302A0912402B09125028093E20590936C
:10633000E305A093E405B093E505089590918911D4
:1063400010928911923071F0943079F0913099F473
:10635000813089F48091E504882369F01092260247
:106360000C948B3110921F0C089586E898E190935D
:106370007F0C80937E0C08959091291493FB8827BD
:1063800080F993FF06C081E090919015911101C0B2
:1063900080E00895CF93C0918205CF7739F50E94B0
:1063A000BC31882319F18091211490912214A0917D
:1063B0002314B09124140097A105B105B9F0BC01D4
:1063C000CD016D597F4F8F4F9F4F24E630E040E065
:1063D00050E00F944E2B60912514709126148091FB
:1063E0002714909128140F944E2BC22F8C2FCF91ED
:1063F0000895E9EFF8E010821182089581E0089590
:10640000DC01EC918E2F90E0FC01EE0FFF1FE80FF6
:10641000F91FEC5DFD4E80818F77808308958F9208
:106420009F92AF92BF92CF92DF92EF92FF920F9323
:10643000CF93DF931F92CDB7DEB75C017B0149019B
:106440006B01C40ED51EF501808191810F94282B1C
:106450008983002311F0F7018083BE016F5F7F4FB6
:10646000C4010E948BE0F5018081918101969183A6
:106470008083FFEFEF1AFF0AEC14FD0421F780E0A0
:106480000F90DF91CF910F91FF90EF90DF90CF9021
:10649000BF90AF909F908F9008950F93AB010091A4
:1064A000DA0521E002272BED35E0BC018BEB95E00E
:1064B0000E940F320F910895009781F4109290007E
:1064C00082E0809391001092950010929400C19AFE
:1064D000809171008260809371000895019761F44A
:1064E0001092A00082E08093A1001092A50010926B
:1064F000A40089BB8093720008957F928F929F922F
:10650000AF92BF92CF92DF92EF92FF920F931F93C1
:10651000CF93DF93EC017B018881883108F0C3C001
:1065200090E0FC01EE0FFF1FE80FF91FEC5DFD4E40
:1065300080818F770E94D3E619821A8288812CE0AD
:10654000622F0F94B12B829FB001112430E020E024
:10655000AB01420F531FFA01EE0FFF1FE40FF51FAF
:10656000EC5DFD4E908197FD08C02F5F3F4F2C30B2
:10657000310571F790E00E945C327880072D10E0C1
:106580006801CC0CDD1CF601E00FF11FEC5DFD4E47
:1065900080818068808377FC86C080E2E81682E094
:1065A000F8060CF03FC08A8128E532E0281B31094B
:1065B00087FD3395220F331F220F331F032E000C4C
:1065C000440B550B898178E8872E912C881A910805
:1065D00087FD9394880C991C880C991C092C000C3D
:1065E000AA08BB0860E070E0CB01F7FC0AC0B70165
:1065F000653B710514F064EB70E0072E000C880B0E
:10660000990B281939094A095B090F943E2B24EB91
:1066100030E040E050E00F94702B820E931EA41ED9
:10662000B51E740187E18715D8F0298188E890E0CC
:10663000821B910927FD9395880F991F880F991F39
:10664000E816F90604F502972FB7F894E601C00F93
:10665000D11FCC5DDD4E880F991F9A8389832FBF90
:1066600062E370E080E090E0DF91CF911F910F91A5
:10667000FF90EF90DF90CF90BF90AF909F908F9062
:106680007F900C9400262A8188E592E0821B910974
:1066900027FD9395880F991F880F991FE816F90613
:1066A00094F6C701D0CFDF91CF911F910F91FF904A
:1066B000EF90DF90CF90BF90AF909F908F907F90A2
:1066C0000895CF93DF93EB01682F70E08DE692E1A0
:1066D0000E947D32688179818A819B81643F21E0BB
:1066E00072078105910520F464EF71E080E090E08D
:1066F0000E94002689B183FB882780F9DF91CF9122
:106700000895CF93DF9300D01F92CDB7DEB78EEE02
:1067100092E0A0E0B0E089839A83AB83BC83BE01A2
:106720006F5F7F4F8AE50E9461330F900F900F904B
:106730000F90DF91CF910895CF93DF9300D01F92F8
:10674000CDB7DEB78EEE92E0A0E0B0E089839A8309
:10675000AB83BC83BE016F5F7F4F8AE00E946133D1
:106760000F900F900F900F90DF91CF910895CF93DE
:10677000DF9300D01F92CDB7DEB784EF91E0A0E0A9
:10678000B0E089839A83AB83BC83BE016F5F7F4F88
:1067900080EA0E9461330F900F900F900F90DF916D
:1067A000CF9108951F920F920FB60F9211240BB63E
:1067B0000F922F933F934F935F936F937F938F939A
:1067C0009F93AF93BF93EF93FF9348EA50E064EA3F
:1067D00070E081E090E00E942426FF91EF91BF914C
:1067E000AF919F918F917F916F915F914F913F9169
:1067F0002F910F900BBE0F900FBE0F901F9018950A
:106800001F920F920FB60F9211240BB60F922F9377
:106810003F934F935F936F937F938F939F93AF9328
:10682000BF93EF93FF9348E950E064E970E090E094
:1068300080E00E942426FF91EF91BF91AF919F913C
:106840008F917F916F915F914F913F912F910F9019
:106850000BBE0F900FBE0F901F9018959091D10016
:1068600095FD0CC09091D00095FF08C08093D60094
:106870008091D00080648093D0000895209112040C
:106880002F5F2F770FB607FC27C090911304921348
:1068900028C09091D00095FF1EC0909113044091A4
:1068A0001204941306C09091D1009F7D9093D10063
:1068B00012C0E92FF0E0EE5EFB4F32819F5F9F77C1
:1068C0003093D600909313043091D000306430930D
:1068D000D000491741F3D9CF90911304921301C00E
:1068E000FBCFE0911204F0E0EE5EFB4F8283209339
:1068F00012048091D10080628093D10008958F921C
:106900009F92AF92BF92CF92DF92EF92FF920F933E
:106910001F93CF93DF937C0121E5E20EF11CD70199
:106920004C914A3509F0A4C06C01B2E5CB0ED11CE4
:10693000F6013081353A09F09BC0EC01C05BDF4FB6
:106940002881233008F494C08C0100561F4FD801D1
:106950004C93E15BFF4F308331962083EF54F10974
:106960003081E05BFF4F30833038B1F43196AC5466
:10697000B1093C913083E854F109AF5ABF4F50E060
:1069800040E02250330B42175307CCF480813296FB
:106990008D934F5F5F4FF7CF233031F5313809F0DA
:1069A00074C0FC01EC55FF4FDC01AC5ABF4F2C9179
:1069B00020833196885A9F4FDC018C918083480157
:1069C000B12CA12C888190E002968A159B050CF4CD
:1069D0003FC0F40181914F010E942E340E94A1E03A
:1069E000FFEFAF1ABF0AEECF323821F5FC01EC5AA7
:1069F000FF4F30814181E05BFF4F40833196308310
:106A0000DC01AA55BF4F50E040E02350330B421742
:106A10005307ACF6FA01EE7FE45AFF4FE80FF91F77
:106A2000608171817C9311966C9311974E5F5F4FDB
:106A30001296EDCF243019F6333809F6FC01EC5AE2
:106A4000FF4F20813181E05BFF4F30833196B0CF23
:106A500080E5DE011D928A95E9F78AE1F80111923D
:106A60008A95E9F78AE5D7018C9385EAF601808358
:106A7000DF91CF911F910F91FF90EF90DF90CF901A
:106A8000BF90AF909F908F900895323809F097CFC4
:106A9000ADCFAF92BF92CF92DF92EF92FF920F9362
:106AA0001F93CF93DF93EC0184E6C82E80E2D82EAB
:106AB000E12CF12C02E8A12C90E2B92E15E0009314
:106AC000B613C092B713D092B813E092B913F092F4
:106AD000BA13B092C013A092BF131093B31383E6FE
:106AE00093E10E947F348FEFC81AD80AE80AF80AA7
:106AF00088E7C81680E2D806E104F10401F724E62D
:106B000030E240E050E0BE0183E693E1DF91CF91B7
:106B10001F910F91FF90EF90DF90CF90BF90AF90BB
:106B20000C94A6E0CF92DF92EF92FF920F931F9307
:106B3000CF93DF93CDB7DEB77C01CDB6DEB60F9431
:106B4000572401962DB73EB7281B390B0FB6F89482
:106B50003EBF0FBE2DBF0DB71EB70F5F1F4FB70152
:106B6000C8010F945024F80101900020E9F73197F3
:106B7000E01BF10B759720F08BE792E0F801848B16
:106B8000C8010E9449350FB6F894DEBE0FBECDBED7
:106B9000DF91CF911F910F91FF90EF90DF90CF90F9
:106BA00008958F929F92AF92BF92CF92DF92EF9211
:106BB000FF920F931F93CF93DF930E94A22C3AE092
:106BC000C32E30E2D32EE12CF12C15E002E8460171
:106BD0005701CAE0D0E01092C0131092BF13109377
:106BE000B3130093B6138092B7139092B813A09288
:106BF000B913B092BA1383E693E10E947F342197D0
:106C00008FEF881A980AA80AB80A209721F78AE015
:106C1000C80ED11CE11CF11C82EDC81680E2D8061A
:106C2000E104F104A1F6C12C20E2D22EE12CF12CDA
:106C3000D5E0C2E81092C0131092BF13D093B313E3
:106C4000C093B613C092B713D092B813E092B913A1
:106C5000F092BA1383E693E10E947F341092C0133E
:106C60001092BF13D093B313C093B613D701C601CC
:106C70008C529F4FAF4FBF4F8093B7139093B81371
:106C8000A093B913B093BA1383E693E10E947F34C3
:106C90008FEFC81AD80AE80AF80A8AE0C81680E214
:106CA000D806E104F10431F69EEDC92E90E2D92E0A
:106CB000E12CF12CD5E0C2E81092C0131092BF1362
:106CC000D093B313C093B613C092B713D092B81336
:106CD000E092B913F092BA1383E693E10E947F34F5
:106CE0008FEFC81AD80AE80AF80A86EEC81680E2BA
:106CF000D806E104F10401F7CC24C39482E1D82E34
:106D0000E12CF12C0AE010E0D5E0C2E81093C013AA
:106D10000093BF13D093B313C093B613C092B713AD
:106D2000D092B813E092B913F092BA1383E693E1CC
:106D30000E947F341093C0130093BF13D093B313FA
:106D4000C093B613D701C6018096A11DB11D8093D3
:106D5000B7139093B813A093B913B093BA1383E603
:106D600093E10E947F348FEFC81AD80AE80AF80A24
:106D700085E1C81682E1D806E104F10439F682E122
:106D800090E09093C0138093BF13D093B313C0933C
:106D9000B61384E190E1A0E0B0E08093B713909344
:106DA000B813A093B913B093BA1383E693E1DF91BC
:106DB000CF911F910F91FF90EF90DF90CF90BF90F8
:106DC000AF909F908F900C947F341F920F920FB6CC
:106DD0000F9211240BB60F922F938F939F93EF93E3
:106DE000FF938091130420911204821306C08091B6
:106DF000D1008F7D8093D10012C0E82FF0E0EE5ECD
:106E0000FB4F92818F5F8F779093D600809313040E
:106E10009091D00090649093D000281741F3FF9197
:106E2000EF919F918F912F910F900BBE0F900FBEFE
:106E30000F901F9018951F920F920FB60F9211246A
:106E40000BB60F920F931F932F933F934F935F9324
:106E50006F937F938F939F93AF93BF93CF93DF9362
:106E6000EF93FF93C091D60000913605D091350580
:106E700011E01D0F1F7390911104913108F09FC014
:106E8000E92FF0E08827E85BF84C8F4F0D94D12B69
:106E9000593788379737A637AD37DF37B137DF3700
:106EA000B537B937DF37BD37C137C537CC37DF37EF
:106EB000D737C03229F028F5CA3011F0CD3031F57E
:106EC000011731F0ED2FF0E0EB5CFA4FC283D12FC8
:106ED000D0933505FF91EF91DF91CF91BF91AF91A5
:106EE0009F918F917F916F915F914F913F912F91E2
:106EF0001F910F910F900BBE0F900FBE0F901F9020
:106F00001895CD3481F081E0CE3471F080E10CC071
:106F1000CA3338F4C033A0F6C03291F2CD32B1F7A3
:106F2000CFCFCD3499F782E080931104C9CFC1331C
:106F300059F018F4C03221F2E9CF88E0C433A1F34C
:106F40008BE0C83389F3E2CF83E0EECF84E0C03337
:106F500059F386E0C13341F3D9CF85E0C833B1F6A8
:106F6000E3CF87E0C23391F6DFCF89E0C13371F61A
:106F7000DBCF8AE0C03351F6D7CF8CE0C73331F690
:106F8000D3CF8DE0C63311F6CFCFC03209F498CFFE
:106F90008EE0C33549F2BACF80ED8C0F8A3008F00D
:106FA0008FCF9FE0909311048093100489CFCA3053
:106FB00019F0CD3009F084CF1092110481CFCA307E
:106FC00019F0CD3009F07CCF80911D148823A1F3F6
:106FD000973089F038F4953079F710923C0210928E
:106FE0001F0CEACF9A3059F09F3031F7809110048E
:106FF0000E949E31E1CF81E080930906DDCF81E0E0
:1070000080930806D9CF9091C00095FFFCCF809364
:10701000C6000895CF93DF93EC018991882319F07E
:107020000E940338FACF8DE00E9403388AE0DF9196
:10703000CF910C940338CF92DF92EF92FF92CF93CF
:107040006B017C01C42F4A3069F4F7FE0BC0F09449
:10705000E094D094C094C11CD11CE11CF11C8DE2C1
:107060000E9403384C2FC701B601CF91FF90EF90DB
:10707000DF90CF900C943EAACF93DF93EC01FE01FA
:1070800084912196882319F00E940338F8CFDF916C
:10709000CF910895CF93DF93D0911C118BE59CE1A4
:1070A0000E943C388AE00E94033880919B0C873014
:1070B00009F449C083E08093990C81E080936E02CB
:1070C00080E190E09093C0138093BF1385E080939C
:1070D000B313C2E8C093B61384E190E1A0E0B0E03E
:1070E0008093B7139093B813A093B913B093BA13C6
:1070F00083E693E10E947F3461E070E080E090E0FD
:107100000E94872C81E09AE59093C0138093BF136F
:1071100085E390E09093C2138093C11387E080933E
:10712000B313C093B61384E890E0A0E0B0E080937E
:10713000B7139093B813A093B913B093BA1383E61F
:1071400093E10E947F3480911C11813089F182305B
:1071500061F50E94742B6093A3057093A40580933E
:10716000A5059093A60581E080931C110E94E3FC85
:1071700060939F057093A0058093A1059093A2054D
:10718000D23089F080918C0690918D060196909373
:107190008D0680938C061092AB051092AC05109270
:1071A000AD051092AE0581E004C00E94A62BDBCF96
:1071B00080E0DF91CF910895CF93C82FCB010E943B
:1071C0003C388FEC98E10E943C3880EC98E1CC236D
:1071D00011F085EC98E10E943C388AE0CF910C9444
:1071E0000338CF93DF9300D01F92CDB7DEB784EF83
:1071F00091E0A0E0B0E089839A83AB83BC83BE01B9
:107200006F5F7F4F8CE30E9461338DEE98E10E94A7
:107210003C388CB167EE78E185FB882780F90E94C5
:10722000DC388091030161EE78E1869581700E94DF
:10723000DC3889B16BED78E183FB882780F90E9407
:10724000DC388CB162ED78E1829581700E94DC3887
:107250004B9909C00E949C330F900F900F900F9094
:10726000DF91CF9108950E9481330F900F900F907E
:107270000F90DF91CF91089580911C118130C1F55D
:107280008BE998E10E943C388AE00E94033881E053
:107290009AE59093C0138093BF1387E590E0909395
:1072A000C2138093C11387E08093B31382E8809365
:1072B000B61384E890E0A0E0B0E08093B713909319
:1072C000B813A093B913B093BA1383E693E10E9465
:1072D0007F3482E080931C110E94E3FC6093A70539
:1072E0007093A8058093A9059093AA0581E008955D
:1072F00080E008950F931F930E94E3FC009187069E
:10730000109188062091890630918A060115110591
:107310002105310509F067C020919512222309F457
:107320005FC0E091931221502093951221E02E0F1F
:107330002093931230919612231302C0109293124D
:1073400024E0E29FF0011124E956FD4E00811181F5
:10735000228133810093830610938406209385064F
:1073600030938606600F711F811D911D6093870603
:10737000709388068093890690938A06809185068B
:1073800090918606892B61F11FB7F8948AE898E1FD
:107390000E943C388AE00E94033884E096E0909393
:1073A000C0138093BF1380EA90E89093C213809338
:1073B000C11387E08093B31382E88093B61380EA09
:1073C00090E0A0E0B0E08093B7139093B813A0933F
:1073D000B913B093BA1383E693E10E947F341FBFC1
:1073E0001F910F910895601B710B820B930B97FDFA
:1073F000F7CF40981092870610928806109289065F
:1074000010928A06EDCF0F931F93CF93DF938C01D9
:10741000EB019091951220919612921305C00E9453
:107420007A390E9406C2F5CF8091941234E0839F8E
:10743000F0011124E956FD4E11830083D383C283EA
:107440009F5F909395128F5F281739F08093941265
:10745000DF91CF911F910F91089510929412F8CF60
:10746000CF92DF92EF92FF921F93CF93DF93182F6B
:10747000662351F01092E4041092E0041092E104AB
:107480001092E2041092E3040E94E3FC6B017C0181
:107490008091E0049091E104A091E204B091E304B2
:1074A000A7019601281B390B4A0B5B0BDA01C901B6
:1074B000B7FD3DC02091E40417FD13C0412F012EFC
:1074C000000C550B4C5F5F4F822F022E000C990B66
:1074D0004817590764F184EF91E0A0E0B0E021176C
:1074E00024F488EE93E0A0E0B0E08C0D9D1DAE1D6D
:1074F000BF1D8093E0049093E104A093E204B09355
:10750000E3042170C22F30E0D32F84E28C9FB001BE
:107510008D9F700D7C1B112460597C4F82E390E09D
:107520000E94033A8091E4048F5F8093E404DF912A
:10753000CF911F91FF90EF90DF90CF900895CF9360
:10754000DF9300D01F92CDB7DEB780E198E10E94B3
:107550003C388AE00E94033880919B0C8330D9F13B
:1075600019821A821B821C8260E0CE0101960E9461
:10757000C12B19821A821B821C8261E0CE01019606
:107580000E94C12B81E080936D021092980C809331
:107590006E0281E09AE59093C0138093BF1383E35A
:1075A00090E09093C2138093C11387E08093B3134C
:1075B00082E88093B61384E890E0A0E0B0E0809386
:1075C000B7139093B813A093B913B093BA1383E68B
:1075D00093E10E947F340F900F900F900F90DF91F6
:1075E000CF9108956F927F928F929F92AF92BF92A8
:1075F000CF92DF92EF92FF920F931F93CF93DF937F
:10760000CDB7DEB764970FB6F894DEBF0FBECDBF1F
:107610001092D0008091D00082608093D0001092B0
:10762000D50080E18093D4008091D1008061809367
:10763000D1008091D10088608093D1008091D100E9
:1076400080688093D1008091D1008F7D8093D1009C
:107650008AE58093B4138093641385EA8093B5130D
:1076600080936513E3E0F4E18AE1DF011D928A95DE
:10767000E9F78091970C882309F473C283E090E0C6
:107680009093C0138093BF1385E08093B31382E877
:107690008093B6138FE190E1A0E0B0E08093B71340
:1076A0009093B813A093B913B093BA1383E693E100
:1076B0000E947F3484E690E09093C0138093BF13C0
:1076C00005E00093B31312E81093B61386E090E13F
:1076D000A0E0B0E08093B7139093B813A093B913D0
:1076E000B093BA1383E693E10E947F348BE090E07D
:1076F0009093C0138093BF130093B3131093B613EA
:1077000080E092E1A0E0B0E08093B7139093B813CB
:10771000A093B913B093BA1383E693E10E947F3428
:107720001092C0131092BF130093B3131093B613AB
:1077300084E390E1A0E0B0E08093B7139093B81396
:10774000A093B913B093BA1383E693E10E947F34F8
:107750001092C0131092BF130093B3131093B6137B
:107760008AE390E1A0E0B0E08093B7139093B81360
:10777000A093B913B093BA1383E693E10E947F34C8
:107780008091E3119091E4119093C0138093BF1303
:107790000093B3131093B61386E390E1A0E0B0E03A
:1077A0008093B7139093B813A093B913B093BA13FF
:1077B00083E693E10E947F34809178119091791152
:1077C0009093C0138093BF130093B3131093B61319
:1077D0008CE390E1A0E0B0E08093B7139093B813EE
:1077E000A093B913B093BA1383E693E10E947F3458
:1077F00082E090E09093C0138093BF130093B31383
:107800001093B6138EE190E1A0E0B0E08093B7133F
:107810009093B813A093B913B093BA1383E693E18E
:107820000E947F3481E080936D0270E6C72E70E184
:10783000D72EE12CF12C1092C0131092BF1300939D
:10784000B3131093B613C092B713D092B813E0924B
:10785000B913F092BA1383E693E10E947F34BFEF2D
:10786000CB1ADB0AEB0AFB0AE4E7CE16E0E1DE0600
:10787000E104F10401F7CE0101967C0184E1D70116
:107880001D928A95E9F781E08F9390E99F938F93FA
:107890009CE29F938F939F938DE893E09F938F93A8
:1078A000FF92EF920F94622F20E630E140E050E02B
:1078B0006AE973E083E693E10E94A6E02AE630E1FC
:1078C00040E050E067EA73E083E693E10E94A6E0BF
:1078D00024E730E140E050E0B70183E693E10E9405
:1078E000A6E02EE730E140E050E063EB73E083E692
:1078F00093E10E94A6E01092C0131092BF13009370
:10790000B3131093B6138EE090E1A0E0B0E0809343
:10791000B7139093B813A093B913B093BA1383E637
:1079200093E10E947F341092C0131092BF13009312
:10793000B3131093B6138FE090E1A0E0B0E0809312
:10794000B7139093B813A093B913B093BA1383E607
:1079500093E10E947F340FB6F894DEBF0FBECDBF17
:107960004AE0C42E40E2D42EE12CF12C55E0752ED5
:1079700062E8662E460157010AE010E01092C0133B
:107980001092BF137092B3136092B6138092B71324
:107990009092B813A092B913B092BA1383E693E110
:1079A0000E947F3401501109FFEF8F1A9F0AAF0A1E
:1079B000BF0A0115110511F78AE0C80ED11CE11CA0
:1079C000F11C92EDC91690E2D906E104F10491F69A
:1079D000C12C30E2D32EE12CF12C05E012E81092FC
:1079E000C0131092BF130093B3131093B613C09239
:1079F000B713D092B813E092B913F092BA1383E69A
:107A000093E10E947F341092C0131092BF13009331
:107A1000B3131093B613D701C6018C529F4FAF4FCB
:107A2000BF4F8093B7139093B813A093B913B0933B
:107A3000BA1383E693E10E947F34AFEFCA1ADA0AE1
:107A4000EA0AFA0ABAE0CB16B0E2DB06E104F10476
:107A500031F62EEDC22E20E2D22EE12CF12C05E0E3
:107A600012E81092C0131092BF130093B313109337
:107A7000B613C092B713D092B813E092B913F09234
:107A8000BA1383E693E10E947F34EFEFCE1ADE0A49
:107A9000EE0AFE0AF6EECF16F0E2DF06E104F1048C
:107AA00001F7CC24C39482E1D82EE12CF12C9AE08A
:107AB000A92EB12C05E012E8B092C013A092BF131A
:107AC0000093B3131093B613C092B713D092B813A8
:107AD000E092B913F092BA1383E693E10E947F34E7
:107AE000B092C013A092BF130093B3131093B613B8
:107AF000D701C6018096A11DB11D8093B713909345
:107B0000B813A093B913B093BA1383E693E10E941C
:107B10007F348FEFC81AD80AE80AF80A95E1C91627
:107B200092E1D906E104F10439F686E797E10E9473
:107B30003C388AE00E94033864960FB6F894DEBFA2
:107B40000FBECDBFDF91CF911F910F91FF90EF90AE
:107B5000DF90CF90BF90AF909F908F907F906F906D
:107B6000089582E090E08CCD0E94F23A10927E055A
:107B700081E080936E0288E298E10E943C388AE0BE
:107B80000C9403380F931F93CF938C01C62F84E27C
:107B900094E10E943C38C8010E943C388AE30E946C
:107BA000033880E38C0F0E9403388AE0CF911F9145
:107BB0000F910C94033887EA95E10E943C3860E00D
:107BC00087E995E10E94C23D60E082E895E10E946C
:107BD000C23D61E08BE795E10E94C23D61E080E734
:107BE00095E10E94C23D61E080E695E10E94C23DC0
:107BF00060E087E595E10E94C23D61E08DE495E19A
:107C00000E94C23D61E083E495E10E94C23D61E0D3
:107C10008CE395E10E94C23D61E084E395E10E941E
:107C2000C23D61E086E295E10E94C23D61E088E1EB
:107C300095E10E94C23D60E089E095E10E94C23D6D
:107C400060E08BEF94E10E94C23D60E085EE94E13C
:107C50000E94C23D61E084ED94E10E94C23D61E07A
:107C600085EC94E10E94C23D61E08EEB94E10E94BC
:107C7000C23D60E087EB94E10E94C23D61E08EEA84
:107C800094E10E94C23D61E089E994E10E94C23D15
:107C900061E08BE894E10E94C23D61E088E794E1F5
:107CA0000E94C23D60E08BE694E10E94C23D61E02B
:107CB00086E694E10E94C23D61E089E594E10E947C
:107CC000C23D60E085E494E10E94C23D60E082E351
:107CD00094E10E94C23D60E08CE294E10E94601D4C
:107CE000682F617089E294E10C94C23D80912F0568
:107CF000827149F4809131058C7829F480913205A4
:107D0000837009F475C082E40E943E1E882351F0FE
:107D10000E940C246093460C7093470C8093480C8F
:107D20009093490C83E50E943E1E882351F00E94E7
:107D300092246093760C7093770C8093780C9093D8
:107D4000790C84E50E943E1E882351F00E94922403
:107D500060937A0C70937B0C80937C0C90937D0CD9
:107D600088E50E943E1E882351F00E949224609371
:107D7000D5087093D6088093D7089093D80889E5E2
:107D80000E943E1E882351F00E9492246093D908DD
:107D90007093DA088093DB089093DC088AE50E94F0
:107DA0003E1E8823B1F00E9492246093DD087093F8
:107DB000DE088093DF089093E0082DEC3CEC4CEC5F
:107DC0005DE30F940A25181624F088E99EE00E94CE
:107DD0003C3885E40E943E1E882351F00E94922484
:107DE0006093E1087093E2088093E3089093E408BD
:107DF0000895AF92BF92CF92DF92EF920F931F93AD
:107E0000CF93DF935B01EA016901882309F463C022
:107E100081E99EE00E943C38F50160817181828198
:107E2000938146E00E9446BAE1100BC088E89EE0CC
:107E30000E943C38688179818A819B8146E00E945A
:107E400046BA81E89EE00E943C38F601608171816B
:107E50008281938143E00E9446BA8AE79EE00E94B5
:107E60003C38F801608171818281938143E00E94F6
:107E700046BA81E79EE00E943C38F60120813181BC
:107E800042815381F80160817181828193810F94D5
:107E9000D92B43E00E9446BAEE20F9F08AE00E9416
:107EA00003388CE59EE00E943C38688179818A81A4
:107EB0009B8146E00E9446BA8AE00E9403388AE02D
:107EC000DF91CF911F910F91EF90DF90CF90BF90F6
:107ED000AF900C940338E110E4CFDF91CF911F9164
:107EE0000F91EF90DF90CF90BF90AF9008950F93D8
:107EF0001F93CF938C01C62F89E798E00E943C38EE
:107F0000C8010E943C38CC2331F08AE0CF911F9108
:107F10000F910C940338CF911F910F9108950E94F7
:107F20003BE410921F0C10923C020E94BC3188234B
:107F300051F08091291482FD06C086E898E1909363
:107F40007F0C80937E0C61E08FE798E10E94773F81
:107F50000C944A380F931F93CF93DF938C016F3F9C
:107F600019F410925D1160E020915D11862F062EAC
:107F7000000C990B2817190609F08CF560935D1118
:107F800060E089E498E10E94773FC8010E943C3894
:107F90008AE00E940338C8010F945724800F911F74
:107FA000EC01C01BD10BC034D1053CF00197FC01A2
:107FB0002491207C2038D1F3F3CFDD27AE01B80126
:107FC0008DE191E10F947824C35EDE4E18828DE13D
:107FD00091E1DF91CF911F910F910C944935DF9181
:107FE000CF911F910F91089510921F0C10923C0297
:107FF0008091291480648093291461E087E598E1D9
:108000000E94773F4CE658E164E778E185E00E9402
:10801000C0E260E08EE598E10C94AA3F0F931F93B5
:10802000CF938C01C62F60E083E898E00E94773FF1
:10803000C8010E943C38CC2331F08AE0CF911F91D7
:108040000F910C940338CF911F910F91089561E027
:108050008BE898E00C940E40EF92FF920F931F93E1
:10806000CF937C018B01C42F60E083E898E00E94ED
:10807000773FC7010E943C3880E20E940338C80164
:108080000E943C38CC2319F08C2F0E9403388AE0E0
:10809000CF911F910F91FF90EF900C940338DF92D6
:1080A000EF92FF920F931F93CF93DF93D82E7B0114
:1080B0008A01E9010E942740D092891140E0B7016E
:1080C00084E799E00E942C400115110531F040E051
:1080D000B8018DE699E00E942C40209731F040E0F5
:1080E000BE018DE699E00E942C4061E088E699E0AF
:1080F000DF91CF911F910F91FF90EF90DF900C9443
:108100000E40AF92BF92CF92DF92EF92FF920F9309
:108110001F93CF93DF9386EE97E00E943C38C0E038
:10812000D7E0D15021F080E20E940338FACF8C2FA3
:108130000E94F9E0CF5FC53099F78AE00E940338CA
:1081400008E817E0C0E080E20E9403388C2F0E940C
:10815000F9E05801D5E080E20E940338F501C080C3
:10816000D180E280F380A7019601C701B6010F9488
:10817000CC2E882369F180E20E9403388DE30E94AF
:1081800003388DE30E9403388DE30E9403388DE3AA
:108190000E9403388DE30E940338D150F4E1AF0E02
:1081A000B11CD111D8CF8AE00E940338CF5F0C5F99
:1081B0001F4FC53041F68AE0DF91CF911F910F919B
:1081C000FF90EF90DF90CF90BF90AF900C9403386A
:1081D00020E030E0A901C701B6010F943A2E87FDD7
:1081E00003C08BE20E94033843E0C701B6010E943E
:1081F00046BAD3CF811107C08AEC9EE00E943C387A
:108200008AE00C9403388EEC9EE0F8CFCF93DF9396
:10821000EB010E943C38CE01DF91CF910C94B7E185
:10822000CF93C62F0E943C388C2FCF910C94F9E04D
:10823000CF92DF92EF92FF926A017B010E943C385D
:1082400042E0C701B601FF90EF90DF90CF900C9411
:1082500046BACF92DF92EF92FF926A017B010E94B1
:108260003C384AE0C701B601FF90EF90DF90CF9015
:108270000C941B38CF93DF93EB010E943C38CE0166
:10828000DF91CF910C9400E14F925F926F927F92B9
:108290008F929F92AF92BF92CF92DF92EF92FF9216
:1082A0000F931F93CF93DF9300D000D01F921F92A4
:1082B000CDB7DEB780917D0581110AC480917B0521
:1082C00090917C059C012F5F3F4F30937C0520935C
:1082D0007B058E3E924008F4FBC38091E3119091A0
:1082E000E4119093C0138093BF1305E00093B31380
:1082F00012E81093B61386E390E1A0E0B0E080931B
:10830000B7139093B813A093B913B093BA1383E63D
:1083100093E10E947F34809178119091791190932C
:10832000C0138093BF130093B3131093B6138CE361
:1083300090E1A0E0B0E08093B7139093B813A093BE
:10834000B913B093BA1383E693E10E947F3480910E
:10835000E5119091E6119093C0138093BF130093A1
:10836000B3131093B61384E390E1A0E0B0E08093E0
:10837000B7139093B813A093B913B093BA1383E6CD
:1083800093E10E947F3480917A1190917B119093B8
:10839000C0138093BF130093B3131093B6138AE3F3
:1083A00090E1A0E0B0E08093B7139093B813A0934E
:1083B000B913B093BA1383E693E10E947F3481E04E
:1083C00080937D0510927C0510927B0580919B0C1B
:1083D000882339F10E94F21C811123C080917A0513
:1083E0008F5F80937A0580917A05853620F0109210
:1083F0007A0510929B0CE0919B0CE150E73008F05D
:108400006AC00E2E000CFF0B8827E65FFD4B8F4FD6
:108410000D94D12B144263422F445B449C44D444BA
:10842000674210927A05DFCF0E947F2C882309F4DF
:1084300052C081E080936E0282E098E10E943C3855
:108440008AE00E94033880E190E09093C01380930B
:10845000BF1385E08093B31312E81093B61384E141
:1084600090E1A0E0B0E08093B7139093B813A0938D
:10847000B913B093BA1383E693E10E947F3481E08D
:108480009AE59093C0138093BF1386E390E0909396
:10849000C2138093C11387E08093B3131093B61374
:1084A00084E890E0A0E0B0E08093B7139093B81315
:1084B000A093B913B093BA1383E693E10E947F347B
:1084C00010929B0C08C00E947F2C882321F00E94F0
:1084D000F21C8823A9F380916E02882309F433C724
:1084E00080917E058111C0C284E096E09093C01314
:1084F0008093BF1380EA90E89093C2138093C113D6
:1085000017E01093B31302E80093B61380EA90E0EB
:10851000A0E0B0E08093B7139093B813A093B91381
:10852000B093BA1383E693E10E947F34809169028D
:1085300090916A02A0916B02B0916C020097A10524
:10854000B10509F03FC21092C0131092BF1315E09D
:108550001093B3130093B6138AE890E1A0E0B0E063
:108560008093B7139093B813A093B913B093BA1331
:1085700083E693E10E947F3489E090E09093C013FA
:108580008093BF131093B3130093B6138CE890E15C
:10859000A0E0B0E08093B7139093B813A093B91301
:1085A000B093BA1383E693E10E947F34809169020D
:1085B00090916A02A0916B02B0916C020097F1E079
:1085C000AF07B10508F441C2B093C013A093BF1325
:1085D0009093C2138093C11387E08093B31382E812
:1085E0008093B61388E890E1A0E0B0E08093B713E1
:1085F0009093B813A093B913B093BA1383E693E1A1
:108600000E947F348091690290916A02A0916B026E
:10861000B0916C02BA2FA92F982F8827009721E0DC
:10862000A207B10508F417C2B093C013A093BF13FB
:108630009093C2138093C11387E08093B31312E821
:108640001093B61381EA90E0A0E0B0E08093B713F6
:108650009093B813A093B913B093BA1383E693E140
:108660000E947F348091310C882309F4FAC183E0A1
:1086700090E09093C0138093BF1385E08093B31371
:108680001093B61385E490E1A0E0B0E08093B713B7
:108690009093B813A093B913B093BA1383E693E100
:1086A0000E947F3480917E05875E80937E052091B5
:1086B0007E05822F90E0253608F021C29093C013EA
:1086C0008093BF1385E08093B31382E88093B61341
:1086D00080E090E1A0E0B0E08093B7139093B813EE
:1086E000A093B913B093BA1383E693E10E947F3449
:1086F0000E94F21C811114C20E94BC31811105C07C
:108700009091810591FD0E94F21C9091810580FB62
:1087100091F99093810591FD03C28091291482FD06
:10872000FFC180911C118150823008F4F9C1609121
:108730007A1170917B11072E000C880B990B0F9406
:1087400011256B017C0120E030E0A9010F940A257E
:10875000882309F4BBC66091781170917911072EB6
:10876000000C880B990B0F9411252B013C0120E084
:1087700030E040E050E4C701B6010F94D92BA301CB
:1087800092010F943A2E18160CF4C2C66091E311B0
:108790007091E411072E000C880B990B0F94112592
:1087A0006D837E838F8398876091E5117091E611C8
:1087B000072E000C880B990B0F9411254B015C01BF
:1087C00020E030E040E251E40F94D92B2D813E812E
:1087D0004F8158850F943A2E18160CF499C620E054
:1087E00030E040E050E4C701B6010F94DA2BA3015A
:1087F00092010F940A2587FD10C020E030E040E28E
:1088000051E4C501B4010F94DA2B2D813E814F81D3
:1088100058850F940A2587FF6AC684E190E09093FB
:10882000C0138093BF1385E08093B31382E88093D5
:10883000B61384E190E1A0E0B0E08093B713909389
:10884000B813A093B913B093BA1383E693E10E94CF
:108850007F348091990C81117CC682E07AC684EFC6
:1088600097E10E943C388AE00E94033881E09AE553
:108870009093C0138093BF1380E490E09093C21351
:108880008093C11317E01093B31382E88093B6135B
:1088900084E890E0A0E0B0E08093B7139093B81321
:1088A000A093B913B093BA1383E693E10E947F3487
:1088B00010939B0C10CE8091880C882309F40BCE6A
:1088C0000E947F2C882309F406CE0E94F21C81119D
:1088D00002CE86EE97E10E943C388AE00E9403387F
:1088E0008091890C90E0B0E0A0E0895B9F4FAE4F93
:1088F000B54A21E03AE53093C0132093BF1390931B
:10890000C2138093C11387E08093B31382E88093EE
:10891000B61384E890E0A0E0B0E08093B7139093A2
:10892000B813A093B913B093BA1383E693E10E94EE
:108930007F341092880CC4CD0E947F2C882309F4C8
:10894000CACD0E94F21C8111C6CD81E080936E02D7
:1089500010929B0C88ED97E10E943C388AE00E94BF
:10896000033881E09AE59093C0138093BF138EE49F
:1089700090E09093C2138093C11387E08093B31368
:1089800082E88093B61384E890E0A0E0B0E08093A2
:10899000B7139093B813A093B913B093BA1383E6A7
:1089A00093E10E947F3497CD0E94F21C811193CDF8
:1089B00019821A821B821C8262E0CE0101960E94FB
:1089C00088F47ECD0196A11DB11D35E0B695A79521
:1089D000979587953A95D1F70197A109B109009725
:1089E000E1E0AE07B10548F1B093C013A093BF1307
:1089F0009093C2138093C1131093B31312E8109392
:108A0000B6138AE890E1A0E0B0E08093B7139093AA
:108A1000B813A093B913B093BA1383E693E10E94FD
:108A20007F3488E090E09093C0138093BF1385E07B
:108A30008093B3131093B613A9CD9093C013809372
:108A4000BF1385E08093B313D9CF9093C013809365
:108A5000BF1385E0C2CD9093C0138093BF1385E010
:108A6000ECCD82E090E005CE8A3F08F020CE8EEF7C
:108A700080937E0587EC97E10E943C388AE00E9453
:108A8000033881E080936E0281E09AE59093C013F1
:108A90008093BF138DE290E09093C2138093C11333
:108AA00087E08093B31382E88093B61384E890E064
:108AB000A0E0B0E08093B7139093B813A093B913DC
:108AC000B093BA1383E693E10E947F3410927D0540
:108AD00028960FB6F894DEBF0FBECDBFDF91CF91C1
:108AE0001F910F91FF90EF90DF90CF90BF90AF90CC
:108AF0009F908F907F906F905F904F9008958456D5
:108B000091099093C0138093BF1385E08093B313B2
:108B100082E88093B61381E090E1A0E0B0E0DCCD84
:108B20008CE090E09093C0138093BF1315E01093F6
:108B3000B31382E88093B61384E190E1A0E0B0E043
:108B40008093B7139093B813A093B913B093BA134B
:108B500083E693E10E947F340E94742B20E13EE083
:108B600040E050E00F944E2B2115310581E048077D
:108B7000510508F470C05093C0134093BF13309355
:108B8000C2132093C11387E08093B31312E81093AC
:108B9000B61380E190E1A0E0B0E08093B71390932A
:108BA000B813A093B913B093BA1383E693E10E946C
:108BB0007F340E94742B20E13EE040E050E00F94AF
:108BC0004E2B2CE330E040E050E00F944E2B3093DE
:108BD000C0132093BF1305E00093B3131093B61393
:108BE00082E190E1A0E0B0E08093B7139093B813D6
:108BF000A093B913B093BA1383E693E10E947F3434
:108C00000E94CA31882309F45CC48F5F8093790580
:108C1000E82EF12C833330F5EE0CFF1CF092C013DC
:108C2000E092BF130093B3131093B6138EE090E15C
:108C3000A0E0B0E08093B7139093B813A093B9135A
:108C4000B093BA1383E693E10E947F341092C0136D
:108C50001092BF132BC03093C0132093BF131093F7
:108C6000B31394CF84E690E09093C0138093BF1326
:108C70000093B3131093B6138EE090E1A0E0B0E040
:108C80008093B7139093B813A093B913B093BA130A
:108C900083E693E10E947F34A2E3EA1AA0E8FA0A8D
:108CA000EE0CFF1CF092C013E092BF130093B313BD
:108CB0001093B6138FE090E1A0E0B0E08093B7137B
:108CC0009093B813A093B913B093BA1383E693E1CA
:108CD0000E947F340E94CA3190E09093C013809329
:108CE000BF1385E08093B31382E88093B61386E1C7
:108CF00090E1A0E0B0E08093B7139093B813A093F5
:108D0000B913B093BA1383E693E10E947F3420E055
:108D100030E0A901609178127091791280917A12F5
:108D200090917B120F94DA2B20E030E048EC52E473
:108D30000F9470250F94462D7093C0136093BF134A
:108D400005E00093B31312E81093B61386E290E1A6
:108D5000A0E0B0E08093B7139093B813A093B91339
:108D6000B093BA1383E693E10E947F348091650249
:108D7000909166029093C0138093BF130093B31336
:108D80001093B61380E093E1A0E0B0E08093B713B6
:108D90009093B813A093B913B093BA1383E693E1F9
:108DA0000E947F3420E030E040E251E460914A0CC0
:108DB00070914B0C80914C0C90914D0C0F94702540
:108DC0000F944D2D7093C0136093BF130093B31392
:108DD0001093B61382E492E1A0E0B0E08093B71361
:108DE0009093B813A093B913B093BA1383E693E1A9
:108DF0000E947F3420E030E040E251E460914E0C6C
:108E000070914F0C8091500C9091510C0F947025E3
:108E10000F944D2D7093C0136093BF130093B31341
:108E20001093B61386E492E1A0E0B0E08093B7130C
:108E30009093B813A093B913B093BA1383E693E158
:108E40000E947F3420E030E040E251E46091520C17
:108E50007091530C8091540C9091550C0F94702587
:108E60000F944D2D7093C0136093BF130093B313F1
:108E70001093B6138AE492E1A0E0B0E08093B713B8
:108E80009093B813A093B913B093BA1383E693E108
:108E90000E947F3420E030E040E251E46091560CC3
:108EA0007091570C8091580C9091590C0F9470252B
:108EB0000F944D2D7093C0136093BF130093B313A1
:108EC0001093B6138EE492E1A0E0B0E08093B71364
:108ED0009093B813A093B913B093BA1383E693E1B8
:108EE0000E947F3420E030E048EC52E46091701240
:108EF0007091711280917212909173120F9470257B
:108F00000F94462D7093C0136093BF130093B31357
:108F10001093B61386E392E1A0E0B0E08093B7131C
:108F20009093B813A093B913B093BA1383E693E167
:108F30000E947F3420E030E048EC52E460917412EB
:108F40007091751280917612909177120F9470251E
:108F50000F94462D7093C0136093BF130093B31307
:108F60001093B6138AE392E1A0E0B0E08093B713C8
:108F70009093B813A093B913B093BA1383E693E117
:108F80000E947F3480917502909176029093C01375
:108F90008093BF130093B3131093B61382E592E14D
:108FA000A0E0B0E08093B7139093B813A093B913E7
:108FB000B093BA1383E693E10E947F3480917302E9
:108FC000909174029093C0138093BF130093B313D6
:108FD0001093B61384E592E1A0E0B0E08093B7135C
:108FE0009093B813A093B913B093BA1383E693E1A7
:108FF0000E947F3420E030E040E251E46091E811CB
:109000007091E9118091EA119091EB110F94702504
:109010000F944D2D7093C0136093BF130093B3133F
:109020001093B61386E592E1A0E0B0E08093B71309
:109030009093B813A093B913B093BA1383E693E156
:109040000E947F342CEA35EC47E25EE36091EC113C
:109050007091ED118091EE119091EF110F94D42C3D
:1090600020E030E040E251E40F9470250F944D2D44
:109070007093C0136093BF130093B3131093B61390
:109080008AE592E1A0E0B0E08093B7139093B81323
:10909000A093B913B093BA1383E693E10E947F348F
:1090A0002CEA35EC47E25EE36091F0117091F1112A
:1090B0008091F2119091F3110F94702520E030E02F
:1090C00040E251E40F9470250F944D2D7093C0131E
:1090D0006093BF130093B3131093B6138EE592E120
:1090E000A0E0B0E08093B7139093B813A093B913A6
:1090F000B093BA1383E693E10E947F3420E030E01E
:1091000040E251E460917D1170917E1180917F1158
:10911000909180110F9470250F944D2D7093C01372
:109120006093BF130093B3131093B61382E692E1DA
:10913000A0E0B0E08093B7139093B813A093B91355
:10914000B093BA1383E693E10E947F342CEA35ECA6
:1091500047E25EE3609181117091821180918311E9
:10916000909184110F94D42C20E030E040E251E43F
:109170000F9470250F944D2D7093C0136093BF13FF
:109180000093B3131093B61386E692E1A0E0B0E02B
:109190008093B7139093B813A093B913B093BA13F5
:1091A00083E693E10E947F342CEA35EC47E25EE3EC
:1091B000609185117091861180918711909188112D
:1091C0000F94702520E030E040E251E40F947025C8
:1091D0000F944D2D7093C0136093BF130093B3137E
:1091E0001093B6138AE692E1A0E0B0E08093B71343
:1091F0009093B813A093B913B093BA1383E693E195
:109200000E947F348091920C811105C08091940C52
:10921000882309F46DC06091E3117091E411072E69
:10922000000C880B990B0F94112520E030E048ECDE
:1092300052E40F9470256B017C016091E5117091EF
:10924000E611072E000C880B990B0F9411259B013A
:10925000AC01C701B6010F94D42C0F944D2D653687
:10926000710510F064E670E07093C0136093BF1353
:1092700005E00093B31312E81093B61384E290E173
:10928000A0E0B0E08093B7139093B813A093B91304
:10929000B093BA1383E693E10E947F346091E311A7
:1092A0007091E411072E000C880B990B0F94112577
:1092B0006B017C0120E030E04AE253E40F943A2E47
:1092C000181624F48091920C811146C16091E51129
:1092D0007091E611072E000C880B990B0F94112545
:1092E0009B01AC01C701B6010F943A2E87FFAFC1B5
:1092F0008091880C882339F18091870C91E0980F38
:109300009093870C90E09093C0138093BF1385E0F7
:109310008093B31382E88093B61382E490E1A0E0D7
:10932000B0E08093B7139093B813A093B913B093A0
:10933000BA1383E693E10E947F348091870C8A30D0
:1093400010F01092870C0E940A2C882309F4B5C1F2
:109350006091800C7091810CEE24E394F12C6115E6
:109360007105A9F090E080E00F940F2520E030E037
:1093700040E85EE30F9470250F94B82C20E030E0B5
:1093800040E85FE30F94DA2B0F944D2D7B0101E051
:1093900010E08091820C811102C010E000E0809109
:1093A000A7129091A8128F3F980711F40E949BB3C7
:1093B0009093A8128093A712080F191FB80190E08C
:1093C00080E00F940F2520E030E040E85EE30F944A
:1093D00070250F94B82C4B015C01F092C013E09201
:1093E000BF1305E00093B31312E81093B61380E1A6
:1093F00093E1A0E0B0E08093B7139093B813A093EB
:10940000B913B093BA1383E693E10E947F34C50188
:10941000B4010F944D2D7093C0136093BF1300934C
:10942000B3131093B61382E193E1A0E0B0E0809310
:10943000B7139093B813A093B913B093BA1383E6FC
:1094400093E10E947F3403E014E1AAE1FA2E8091B7
:109450003505909136052091770530917805891B67
:109460008F7309F449C12A3131050CF0DBC19091A9
:109470003505809136054FEF5FEF981749F0E82FDB
:10948000F0E0EB5CFA4F42818F5F8F73809336057B
:10949000F901ED5FFB4E4083809103148A3509F09A
:1094A000B3C162E070E080E090E00E94872C809180
:1094B00077059091780501969093780580937705CC
:1094C000C6CF1092C0131092BF13ACCB6091E511C0
:1094D0007091E611072E000C880B990B0F94112543
:1094E00020E030E0A9010F940A25811134C98CE0F5
:1094F00090E09093C0138093BF1385E08093B313E3
:1095000082E88093B61384E190E1A0E0B0E0F3CB71
:109510008DE090E09093C0138093BF1385E080931B
:10952000B31382E88093B61384E190E1A0E0B0E049
:109530008093B7139093B813A093B913B093BA1351
:1095400083E693E10E947F348091990C811101C0E0
:1095500081E08093990CDBCB1092920C20E030E0FC
:1095600040E251E460918A0C70918B0C80918C0CDC
:1095700090918D0C0F9470250F94462D7093C0130D
:109580006093BF130093B3131093B61384E590E177
:10959000A0E0B0E08093B7139093B813A093B913F1
:1095A000B093BA1383E693E10E947F3420E030E069
:1095B00040E251E460918E0C70918F0C8091900C80
:1095C0009091910C0F9470250F94462D7093C013B9
:1095D0006093BF130093B3131093B61388E590E123
:1095E000A0E0B0E08093B7139093B813A093B913A1
:1095F000B093BA1383E693E10E947F3486EA97E141
:109600000E943C388AE00E94033881E09AE59093FA
:10961000C0138093BF1381E490E09093C2138093B2
:10962000C11387E08093B3131093B61384E890E0DE
:10963000A0E0B0E08093B7139093B813A093B91350
:10964000B093BA1383E693E10E947F3451CE6091C8
:10965000940C662309F44CCE062E000C770B8DE893
:1096600097E10E943A418AE00E9403381092940CDC
:1096700084E090E09093C0138093BF1385E08093C3
:10968000B31312E81093B6138EE890E1A0E0B0E0B7
:109690008093B7139093B813A093B913B093BA13F0
:1096A00083E693E10E947F3481E09AE59093C013B2
:1096B0008093BF1383E590E0B0CF1092C013109257
:1096C000BF1305E00093B31312E81093B61380E1C3
:1096D00093E1A0E0B0E08093B7139093B813A09308
:1096E000B913B093BA1383E693E10E947F341092CA
:1096F000C0131092BF1393CE121613060CF492C02F
:109700008091671390916813A0916913B0916A13C7
:109710008C34E0E19E07A105B10509F4D7C98A346C
:109720009041A105B10509F4D1C920E030E040E243
:1097300051E46091200C7091210C8091220C909149
:10974000230C0F9470250F94462D7093C0136093D3
:10975000BF1305E00093B31312E81093B61388E427
:1097600090E1A0E0B0E08093B7139093B813A0937A
:10977000B913B093BA1383E693E10E947F3420E0DB
:1097800030E040E251E46091240C7091250C80910E
:10979000260C9091270C0F9470250F94462D7093F2
:1097A000C0136093BF130093B3131093B6138AE4EE
:1097B00090E1A0E0B0E08093B7139093B813A0932A
:1097C000B913B093BA1383E693E10E947F3420E08B
:1097D00030E040E251E46091280C7091290C8091B6
:1097E0002A0C90912B0C0F9470250F94462D70939A
:1097F000C0136093BF130093B3131093B6138CE49C
:1098000090E1A0E0B0E056C9121613060CF01FCE8E
:10981000F8012F2D11922A95E9F7109278051092F0
:10982000770515CE9091641380910314981321C08D
:10983000909165138091041498131BC02330310557
:10984000C4F0909105149093631380910614809353
:1098500066139330D1F4982F9D7F9038B1F4909196
:1098600007149F3409F059C0909108149B3409F0F3
:1098700054C0E3E0F4E18AE1DF011D928A95E9F743
:1098800010927805109277053BCF833809F045C0D8
:109890008091071490910814982789279827B0E0A1
:1098A000A0E08093671390936813A0936913B0931B
:1098B0006A13C0900914D12CF12CE12CC0926B13C7
:1098C000D0926C13E0926D13F0926E132AE034E1A3
:1098D00040E050E0BA014C155D056E057F0508F0CB
:1098E0004AC0DB01CA01B695A7959795879506965C
:1098F000880F991FFC01ED59FC4ED9018C911196EE
:109900009C91892798278927918380834E5F5F4F99
:109910006F4F7F4F2E5F3F4FDECF813861F58091D3
:10992000071490E0B0E0A0E0809367139093681371
:10993000A0936913B0936A1380910814482F50E0E4
:1099400070E060E040936B1350936C1360936D1361
:1099500070936E13A9E0B4E1EFE6F3E190E030E03C
:1099600020E08217930739F04D9150E041935193D5
:109970002F5F3F4FF6CFE3E0F4E18AE1DF011D9274
:109980008A95E9F710927805109277050E9493FD69
:10999000B7CE3F924F925F926F927F928F929F923B
:1099A000AF92BF92CF92DF92EF92FF920F931F93ED
:1099B000CF93DF938091310587FD38C080913205C8
:1099C0008370A1F5C0917C12D0917D12488159819C
:1099D0006A817B8187E197E10E9418414C815D811A
:1099E0006E817F818FE49FE20E941841409178123E
:1099F0005091791260917A1270917B128CE49FE2FF
:109A00000E9418418AE0DF91CF911F910F91FF9042
:109A1000EF90DF90CF90BF90AF909F908F907F900E
:109A20006F905F904F903F900C940338609070124D
:109A3000709071128090721290907312A0907412B4
:109A4000B09075120091761210917712C090781232
:109A5000D0907912E0907A12F0907B1288E50E9403
:109A60008C1EC82F882309F49AC00E949224362E97
:109A7000472E582ED92F20E030E046E953EC0F94C2
:109A80003A2E87FD0DC020E030E046E953E4632D17
:109A9000742D852D9D2F0F940A2518160CF081C06A
:109AA0006CE271E084E097E10E943A416CE271E07F
:109AB0008FEF96E10E943A418CEF96E10E943C388C
:109AC000C0E089E50E948C1E882361F10E949224E7
:109AD000362E472E582ED92F20E030E046E953ECA1
:109AE0000F943A2E87FD0DC020E030E046E953E4A4
:109AF000632D742D852D9D2F0F940A2518160CF0BB
:109B000055C06CE271E089EE96E10E943A416CE248
:109B100071E084EE96E10E943A4181EE96E10E9466
:109B20003C38C0E08AE50E948C1E882309F443C0BB
:109B30000E9492246B017C0120E030E040E151EC76
:109B40000F943A2E87FD0AC020E030E040E151E456
:109B5000C701B6010F940A2518166CF567EF7FEF61
:109B60008FEC96E10E943A4169E070E08AEC96E160
:109B70000E943A4187EC96E1DF91CF911F910F91BE
:109B8000FF90EF90DF90CF90BF90AF909F908F901D
:109B90007F906F905F904F903F900C943C38C1E065
:109BA00090CF632C742C852C9D2E8BCFA32CB42CA2
:109BB000052D1D2FB7CFCC23E1F0C301D401809335
:109BC000701290937112A0937212B0937312C50128
:109BD000D8018093741290937512A0937612B0936B
:109BE0007712C0927812D0927912E0927A12F092A3
:109BF0007B12DF91CF911F910F91FF90EF90DF903B
:109C0000CF90BF90AF909F908F907F906F905F901C
:109C10004F903F9008958FED97E00C943C3889ED7C
:109C200097E00C943C3884E690E09093BC058093D8
:109C3000BB051092DC051092DB050C946ADBEF92F9
:109C4000FF920F931F93CF93DF93CDB7DEB7629749
:109C50000FB6F894DEBF0FBECDBF0E940D2A882339
:109C600009F43FC042EE53E082FF02C046EC53E0ED
:109C700022EE33E081FF02C028EC33E080FD2EC0ED
:109C800082EE93E05F934F933F932F939F938F9335
:109C900081E499E19F938F938E010F5F1F4F1F9374
:109CA0000F930F94A1240E940F4EC8010E940A38FE
:109CB000C8010E9403E40FB6F894DEBF0FBECDBF0B
:109CC00081E062960FB6F894DEBF0FBECDBFDF9184
:109CD000CF911F910F91FF90EF9008958AEC93E040
:109CE000D1CF80E0EECFCF92DF92EF92FF928AE564
:109CF0000E948C1E882309F45AC00E94922420E0FE
:109D000030E040E050EC0F940A25C12CD12CE12C1E
:109D100090ECF92E87FD0FC00E94922420E030E0E5
:109D200040E050E40F943A2E18160CF462C00E94E2
:109D300092246B017C012091520C3091530C409184
:109D4000540C5091550CC701B6010F9470250F9417
:109D5000462DCB010E941CFD80E50E943E1E811114
:109D60004EC0A7019601609178127091791280918E
:109D70007A1290917B120F94DA2B60937812709381
:109D8000791280937A1290937B120E940F4E409129
:109D900078125091791260917A1270917B1288EB4F
:109DA00096E10E9418418AE00E94033805C083E5CD
:109DB0000E948C1E8111A1CF8091310587FD24C0A6
:109DC00080913205837001F50E940F4E4091781208
:109DD0005091791260917A1270917B1289EA96E122
:109DE0000E9418418AE0FF90EF90DF90CF900C9492
:109DF0000338C12CD12CE12C80E4F82E9CCF0E949A
:109E00005A248111AECFD8CF82E50E943E1E811127
:109E1000DBCFFF90EF90DF90CF900895CF9384E554
:109E20000E948C1EC0E08823D9F00E943A24C82FDB
:109E30001816B4F40E940F4E8DE40E9403388091EE
:109E40002C0590912D050E94B7E16C2FCC0F770B5C
:109E500088EA9FE00E943A418AE00E940338CFEFEF
:109E60008C2FCF9108954F925F926F927F928F9235
:109E70009F92AF92BF92CF92DF92EF92FF92CF93D9
:109E8000DF93CDB7DEB72C970FB6F894DEBF0FBEC9
:109E9000CDBF4090C8085090C9086090CA08709023
:109EA000CB082091470230914802409149025091DD
:109EB0004A02C301B2010F94DA2B69837A838B8340
:109EC0009C838090CC089090CD08A090CE08B09054
:109ED000CF0820914B0230914C0240914D0250919D
:109EE0004E02C501B4010F94DA2B6D837E838F83FC
:109EF0009887C090D008D090D108E090D208F09018
:109F0000D30820914F02309150024091510250915C
:109F10005202C701B6010F94DA2B69877A878B87C3
:109F20009C872091530230915402409155025091E8
:109F30005602C301B2010F94DA2B2B013C01209190
:109F40005702309158024091590250915A02C5016E
:109F5000B4010F94DA2B4B015C0120915B0230912C
:109F60005C0240915D0250915E02C701B6010F9400
:109F7000DA2B6B017C010E940F4E83EE9EE00E9463
:109F80003C3883E50E943E1E882321F00E945A241B
:109F90008093450280914502811151C08AEC9EE078
:109FA0000E943C388BED9EE00E943C3849815A81EA
:109FB0006B817C818FE09EE10E9418414D815E8122
:109FC0006F8178858FE49FE20E94184149855A8508
:109FD0006B857C858CE49FE20E94184189ED9EE0B0
:109FE0000E943C3881ED9EE00E943C38B301A20102
:109FF0008FE09EE10E941841B501A4018FE49FE229
:10A000000E941841B701A6018CE49FE20E9418410A
:10A010008AE02C960FB6F894DEBF0FBECDBFDF915D
:10A02000CF91FF90EF90DF90CF90BF90AF909F9037
:10A030008F907F906F905F904F900C9403388EECD0
:10A040009EE0AECF5F926F927F928F929F92AF927F
:10A05000BF92CF92DF92EF92FF920F931F93CF9315
:10A06000DF931F92CDB7DEB77C0139018B015B0115
:10A07000A40EB51ED12CC12CA016B10609F450C0F7
:10A08000F70180809180F80151908F015982C401BD
:10A090000F94282B5816B9F1652DC4010F94302B5D
:10A0A000FFEFCF1ADF0AC6018F779927892B21F19D
:10A0B00062E070E080E090E00E94B0FCC4010F9488
:10A0C000282B99818917F9F00E940F4E8FE694E0B2
:10A0D0000E943C3881E00F90DF91CF911F910F914A
:10A0E000FF90EF90DF90CF90BF90AF909F908F90B8
:10A0F0007F906F905F90089562E070E080E090E064
:10A100000E940026DBCFBE016F5F7F4FC3010E941C
:10A110008BE0F70180819181019691838083ACCFA0
:10A1200080E0D9CFDF92EF92FF920F931F93CF93EE
:10A13000DF93CDB7DEB7CA5AD1090FB6F894DEBFA8
:10A140000FBECDBFCF55DF4F188219821A821B82F6
:10A15000C15AD0408091CC039091CD03A091CE0301
:10A16000B091CF03CB55DF4F88839983AA83BB83FC
:10A17000C55AD04084E690E09093BC058093BB051F
:10A180001092DC051092DB051092DD052BED35E019
:10A1900044E050E0BE016B557F4F8BEB95E00E9491
:10A1A00022508091BB059091BC0502969093BC050E
:10A1B0008093BB051092DC051092DB0581E0C6554B
:10A1C000DF4F8883CA5AD040CE0186559F4F0E94E8
:10A1D000B2D12BED35E048E450E066E37CE08BEB58
:10A1E00095E00E9422502BED35E040E150E065ED16
:10A1F00078E08BEB95E00E9422508AE097EDA3EA8D
:10A20000BCE3CF55DF4F88839983AA83BB83C15AB0
:10A21000D040CE018F559F4F0E94A9D18EEF97E07D
:10A220000E94C4D186E292E00E94BBD182E292E019
:10A230000E94A9D18091C4089091C508A091C60838
:10A24000B091C70889839A83AB83BC838E010F5F6B
:10A250001F4FC8010E94A9D1CF55DF4F1882198224
:10A260001A821B82C15AD0407E018DE6E80EF11C95
:10A2700083E0D7018C938983CE018F559F4F0E9435
:10A28000A9D1C7010E94B2D1C8010E94B2D14AE04F
:10A29000D42EDA94DD2031F0CE018F559F4F0E94ED
:10A2A000A9D1F7CF80E792E10E94C4D1CF55DF4F0B
:10A2B000188219821A821B82C15AD0403AE0D32EEA
:10A2C000DA94DD2031F0CE018F559F4F0E94A9D145
:10A2D000F7CF85E0D82ED982F701D082C8010E943D
:10A2E000B2D1C7010E94B2D12BED35E048E050E079
:10A2F0006EEC75E08BEB95E00E9422502BED35E083
:10A3000048E050E066EC75E08BEB95E00E9422504F
:10A310002BED35E044E650E068E877E08BEB95E024
:10A320000E94225019828FEFD7018C93C8010E949E
:10A33000BBD1C7010E94B2D12BED35E044E050E023
:10A3400066EE72E08BEB95E00E94225080919F06B2
:10A350008983C8010E94BBD1198A1A8A1B8A1C8A68
:10A3600080E090E0A0E8BFE38D879E87AF87B88B41
:10A370008091E8119091E911A091EA11B091EB114F
:10A3800089839A83AB83BC832CEA35EC47E25EE396
:10A390006091EC117091ED118091EE119091EF119F
:10A3A0000F94D42C6D837E838F8398872CEA35ECB1
:10A3B00047E25EE36091F0117091F1118091F2112A
:10A3C0009091F3110F94702569877A878B879C870A
:10A3D0002BED35E044E150E0B8018BEB95E00E94B5
:10A3E000225084E190E09A838983C8010E9497D12A
:10A3F00080917D1190917E11A0917F11B09180117B
:10A4000089839A83AB83BC832CEA35EC47E25EE315
:10A4100060918111709182118091831190918411CA
:10A420000F94D42C6D837E838F8398872CEA35EC30
:10A4300047E25EE3609185117091861180918711EA
:10A44000909188110F94702569877A878B879C87F4
:10A45000C8010E94A0D18CE0EDE7F2E0D8010190A4
:10A460000D928A95E1F7C8010E94A0D11982C80116
:10A470000E94B2D18FE790E09A838983C8010E943D
:10A4800097D1E9E8F2E0D80101900D92DA94E1F772
:10A490002BED35E045E050E0B8018BEB95E00E94F4
:10A4A00022508091C5058983C8010E94BBD180E2FA
:10A4B000EEE8F2E0D80101900D928A95E1F72BEDDC
:10A4C00035E040E250E0B8018BEB95E00E9422506D
:10A4D000F7011082C7010E94BBD181EF97E00E9473
:10A4E000BBD18DEE97E00E94A9D1CF55DF4F1882E6
:10A4F00019821A821B82C15AD040CE018F559F4FBC
:10A500000E94A9D180E2D8011D928A95E9F72BED2E
:10A5100035E040E250E0B8018BEB95E00E9422501C
:10A52000FE01F99688E0DF011D928A95E9F744E67D
:10A5300050E060E070E049835A836B837C834D83F5
:10A540005E836F83788783E090E0A0E0B0E0898746
:10A550009A87AB87BC874D875E876F87788B498BDF
:10A560005A8B6B8B7C8B8D8B9E8BAF8BB88F898F2F
:10A570009A8FAB8FBC8F8D8F9E8FAF8FB8A38EE1DC
:10A5800090E0A0E0B0E089A39AA3ABA3BCA38DA305
:10A590009EA3AFA3B8A789A79AA7ABA7BCA78DA76F
:10A5A0009EA7AFA7B8AB89AB9AABABABBCAB8DAB3F
:10A5B0009EABAFABB8AF2BED35E040E450E0B80157
:10A5C0008BEB95E00E94225090E1D92EF8018D2D61
:10A5D00011928A95E9F72BED35E040E150E0B801A2
:10A5E0008BEB95E00E942250D8011D92DA94E9F796
:10A5F0002BED35E040E150E0B8018BEB95E00E9497
:10A600002250CF55DF4F188219821A821B82C15AFD
:10A61000D040CE018F559F4F0E94A9D12CE0D22E61
:10A62000F8018D2D11928A95E9F72BED35E04CE07C
:10A6300050E0B8018BEB95E00E9422508CE6D801E7
:10A640001D928A95E9F72BED35E04CE650E0B80114
:10A650008BEB95E00E9422508FEA95E00E94A0D1FA
:10A660002BED35E048E050E06DEB75E08BEB95E0CD
:10A670000E942250F7011192DA94E9F7C755DF4F93
:10A680001882C95AD04080E090E0A0E4B0E4C356FC
:10A69000DF4F88839983AA83BB83CD59D040C701FC
:10A6A0000E94C4D1CE0187559F4F0E94B2D1CE01E6
:10A6B00083569F4F0E94A9D180E3D7011D928A95AE
:10A6C000E9F78BE89CE10E943C388AE00E9403385D
:10A6D0002BED35E040E350E0B7018BEB95E00E94B5
:10A6E00022508091DD05811128C00091BB05109199
:10A6F000BC058091DB059091DC05F7019183808397
:10A7000084E690E09093BC058093BB052BED35E08B
:10A7100044E050E06AEE72E08BEB95E00E9422503C
:10A72000C7010E9497D191E00536134009F490E0EB
:10A730008091DD05892B8093DD058091DD058111F8
:10A7400005C060E08FEB9CE10E94AA3F8FE99CE18D
:10A750000E943C388AE00E9403389091DD0581E038
:10A760008927C655DF4F0FB6F894DEBF0FBECDBFA9
:10A77000DF91CF911F910F91FF90EF90DF9008959F
:10A78000CF93DF9300D01F92CDB7DEB780918B06B9
:10A790008823C1F083E390E09C838B831A82198223
:10A7A0009E012F5F3F4F40E150E06CE876E0CE0124
:10A7B00003960E9422508FE99CE10E943C388AE077
:10A7C0000E9403380F900F900F900F90DF91CF9160
:10A7D0000895CF92DF92EF92FF92CF93C82F80918E
:10A7E0001C118150823008F069C00E949F3A10927B
:10A7F0001C110E94E3FC6093A7057093A805809349
:10A80000A9059093AA05C090AB05D090AC05E09047
:10A81000AD05F090AE050E94742BAB01BC014093D6
:10A82000AB055093AC056093AD057093AE05809178
:10A83000900690919106A0919206B09193068C1982
:10A840009D09AE09BF09840F951FA61FB71F8093EE
:10A85000900690939106A0939206B0939306C1112F
:10A860000AC0C1E00E94C0538C2FCF91FF90EF909F
:10A87000DF90CF90089580918E0690918F0601967B
:10A8800090938F0680938E060E94742BC09094063E
:10A89000D0909506E0909606F0909706C616D706DB
:10A8A000E806F906F0F60E94742B60939406709304
:10A8B00095068093960690939706D3CFC0E0D2CFAB
:10A8C00081E00C94E9530E94B9BE0E94605480E07C
:10A8D0000E94B2F88091E1068130A1F40E940B4EF3
:10A8E00082E697E00E943C3860E088E597E00E94AD
:10A8F000AA3F6EE571E080E090E00E94002688E0CB
:10A900008093E1060895CF92DF92EF92FF921F931A
:10A91000CF93DF9300D01F92CDB7DEB78EEEC82E57
:10A9200082E0D82EE12CF12CC982DA82EB82FC8203
:10A93000BE016F5F7F4F8AE50E94613381110EC0B7
:10A9400010E0812F0F900F900F900F90DF91CF911B
:10A950001F91FF90EF90DF90CF9008950E94B73342
:10A96000C982DA82EB82FC82BE016F5F7F4F8AE58B
:10A970000E946133182F882319F30E940B4E8CE339
:10A9800098E00E943C380E946354DBCFCF92DF9264
:10A99000EF92FF921F93CF93DF9300D01F92CDB71A
:10A9A000DEB78EEEC82E82E0D82EE12CF12CC982C3
:10A9B000DA82EB82FC82BE016F5F7F4F8AE00E94E9
:10A9C000613381110EC010E0812F0F900F900F9016
:10A9D0000F90DF91CF911F91FF90EF90DF90CF907C
:10A9E00008950E94B7330E9481330E949C330E94D5
:10A9F0008133C982DA82EB82FC82BE016F5F7F4FB6
:10AA00008AE00E946133182F8823E9F20E940B4EDE
:10AA10008FEF97E00E943C380E946354D5CFCF93CC
:10AA2000DF9300D01F921F92CDB7DEB781E08093F5
:10AA30008B0680E1ECE8F6E0DF011D928A95E9F7EC
:10AA40000E94C05386E18D8382E390E09C838B83D8
:10AA50001A8219829E012F5F3F4F41E050E0BE01F4
:10AA60006B5F7F4FCE0103960E9422500F900F9094
:10AA70000F900F900F90DF91CF910895CF93DF93B8
:10AA8000CDB7DEB7A8970FB6F894DEBF0FBECDBF27
:10AA90008C01F42E0E94B9BE0E940B4E88E397E011
:10AAA0000E943C380115110511F40FE217E0809166
:10AAB000810580FD79C08160809381058BE197E0FD
:10AAC0000E943C388AE00E940338CC24C3948AE573
:10AAD000D82ED092C013C092BF138FE090E0909315
:10AAE000C2138093C11397E0792E7092B31322E8BA
:10AAF000E22EE092B61334E8832E912CA12CB12CD7
:10AB00008092B7139092B813A092B913B092BA136F
:10AB100083E693E10E947F34D092C013C092BF13AA
:10AB200088E590E09093C2138093C1137092B313A1
:10AB3000E092B6138092B7139092B813A092B91313
:10AB4000B092BA1383E693E10E947F348AE289834C
:10AB50008A838B838C83F801DE011596BE016F5FBB
:10AB60007F4FCD01861B970B2491319621110CC08C
:10AB7000FB01E80FF91F8AE29F01261B370B2832E1
:10AB8000310524F48193F8CF2D93EBCF20E630E10B
:10AB900040E050E083E693E10E94A6E06AE070E0C6
:10ABA00080E090E00E94872C61E086E297E00E94BE
:10ABB000773F89EE93E030E6019729F0232F2A951D
:10ABC0000000E9F7F9CFF89489EE93E038EE0197A9
:10ABD00029F0232F2A950000E9F7F9CF0E94B9BE8A
:10ABE000FF2031F00E94F81E0E94111FA895FECF91
:10ABF0000E94F61EF9CF8091E006882319F010928A
:10AC0000E006089540E070E060E082EB98E10E9489
:10AC10003E5580919C0C90919D0C2FEF3FEF981723
:10AC200051F0E92FF0E0E456F34F228130E09F5FCE
:10AC30009F7790939D0CC90108951F920F920FB6B4
:10AC40000F9211240F900FBE0F901F9018951F9216
:10AC50000F920FB60F9211240BB60F920F931F9302
:10AC60002F933F934F935F936F937F938F939F9314
:10AC7000AF93BF93CF93DF93EF93FF93C091C60041
:10AC800000919D0CD0919C0C11E01D0F1F779091AD
:10AC90000F04913108F09FC0E92FF0E08827EC5AAB
:10ACA000F94A8F4F0D94D12B65569456A356B25640
:10ACB000B956EB56BD56EB56C156C556EB56C9565E
:10ACC000CD56D156D856EB56E356C03229F028F56A
:10ACD000CA3011F0CD3031F5011731F0ED2FF0E031
:10ACE000E456F34FC283D12FD0939C0CFF91EF9188
:10ACF000DF91CF91BF91AF919F918F917F916F9194
:10AD00005F914F913F912F911F910F910F900BBE2B
:10AD10000F900FBE0F901F901895CD3481F081E0F9
:10AD2000CE3471F080E10CC0CA3338F4C033A0F6E1
:10AD3000C03291F2CD32B1F7CFCFCD3499F782E066
:10AD400080930F04C9CFC13359F018F4C03221F2F7
:10AD5000E9CF88E0C433A1F38BE0C83389F3E2CFB5
:10AD600083E0EECF84E0C03359F386E0C13341F392
:10AD7000D9CF85E0C833B1F6E3CF87E0C23391F68F
:10AD8000DFCF89E0C13371F6DBCF8AE0C03351F603
:10AD9000D7CF8CE0C73331F6D3CF8DE0C63311F671
:10ADA000CFCFC03209F498CF8EE0C33549F2BACF85
:10ADB00080ED8C0F8A3008F08FCF9FE090930F04C6
:10ADC0008093100489CFCA3019F0CD3009F084CFB8
:10ADD00010920F0481CFCA3019F0CD3009F07CCF2A
:10ADE00080911D148823A1F3973089F038F49530B1
:10ADF00079F710923C0210921F0CEACF9A3059F06A
:10AE00009F3031F7809110040E949E31E1CF81E0A4
:10AE100080930906DDCF81E080930806D9CF8EBDEF
:10AE20000DB407FEFDCF08958FEF8EBD0DB407FE64
:10AE3000FDCF8EB50895909164009B7F9093640040
:10AE4000982F906A96959CBD80FD03C091E0863056
:10AE500009F490E09DBD0895CF93DF93EB010E942C
:10AE60003C38CE01DF91CF910C9403AF2F923F92EB
:10AE70004F925F926F927F928F929F92AF92BF920A
:10AE8000CF92DF92EF92FF920F931F93CF93DF93B6
:10AE9000009709F0AAC11092840C1092830C909331
:10AEA000800580937F05BAE0CB2EB0E2DB2EE12C4B
:10AEB000F12C15E002E846015701C4E1D0E0109200
:10AEC0000613109205131093F9120093FC1280924E
:10AED000FD129092FE12A092FF12B092001389EA26
:10AEE00092E10E947F3421972FEF821A920AA20AE0
:10AEF000B20A209721F744E1C40ED11CE11CF11CD9
:10AF00008AE5C81680E2D806E104F104A1F6C12C56
:10AF1000A0E2DA2EE12CF12CD5E0C2E81092061363
:10AF200010920513D093F912C093FC12C092FD1237
:10AF3000D092FE12E092FF12F092001389EA92E1A1
:10AF40000E947F341092061310920513D093F912C9
:10AF5000C093FC12D701C6018C529F4FAF4FBF4F19
:10AF60008093FD129093FE12A093FF12B0930013F2
:10AF700089EA92E10E947F34EFEFCE1ADE0AEE0AF0
:10AF8000FE0AFAE0CF16F0E2DF06E104F10431F642
:10AF9000FEEDCF2EF0E2DF2EE12CF12CD5E0C2E861
:10AFA0001092061310920513D093F912C093FC125D
:10AFB000C092FD12D092FE12E092FF12F0920013A6
:10AFC00089EA92E10E947F342FEFC21AD20AE20A84
:10AFD000F20A46EEC41640E2D406E104F10401F799
:10AFE000CC24C394E2E1DE2EE12CF12C0AE010E047
:10AFF000D5E0C2E81093061300930513D093F9121D
:10B00000C093FC12C092FD12D092FE12E092FF1289
:10B01000F092001389EA92E10E947F3410930613A4
:10B0200000930513D093F912C093FC12D701C60107
:10B030008096A11DB11D8093FD129093FE12A093E6
:10B04000FF12B093001389EA92E10E947F348FEFE0
:10B05000C81AD80AE80AF80AE5E0CE16E2E1DE06E8
:10B06000E104F10439F60091830C1091840C011570
:10B07000110509F0D6C08091820C882309F4E1C043
:10B080002AE030E240E050E060ED73E089EA92E1CE
:10B090000E94A6E0C1E0D0E003E010E0E090830C65
:10B0A000F090840C35E0332E42E8242E44244A9458
:10B0B000542C64E0662E712C7FE1C72E74E0D72EED
:10B0C0008091830C9091840C800F911FE816F906F3
:10B0D00008F0D5C0C7010E94BDE1882309F481C0F2
:10B0E000809197116AE871E1882311F067E971E1B5
:10B0F000FB0101900020E9F7CF010197861B970B18
:10B10000F4E1FC9F9001FD9F300D1124265F3F4D1F
:10B1100050E040E0459710F0FB01128A89EA92E185
:10B120000E94A6E0CE018F5F9D4EB0E0A0E0219688
:10B130004E0124E0880C991C2A95E1F7FDEF8F1A47
:10B14000FFE99F0AB12CA12C2091291424FF7EC075
:10B1500070920613609205133092F9122092FC123D
:10B160008093FD129093FE12A093FF12B0930013F0
:10B1700089EA92E10E947F34D0920613C0920513AF
:10B180003092F9122092FC128092FD129092FE12DF
:10B19000A092FF12B092001389EA92E10E947F34DC
:10B1A000B70187E498E10E9406418091971167E911
:10B1B00071E1811102C06AE871E184E498E10E94C2
:10B1C0002C576FED7BE080E498E10E942C576AE8F1
:10B1D00071E18FE398E10E942C578BE398E10E9484
:10B1E0003C382FEFE21AF20A6BCF2091830C30919A
:10B1F000840CA9014150510960917F05709180052F
:10B200006817790738F42C5F3F4F3093840C2093F4
:10B21000830C45CE4430510508F43DCE245031090D
:10B22000F4CF0430110569F48091820C882331F049
:10B2300083E090E09093840C8093830CD0E0C0E096
:10B240002DCFD0E0C0E004E010E028CF109206132C
:10B25000109205133092F9122092FC128093FD1285
:10B260009093FE12A093FF12B093001389EA92E12B
:10B270000E947F34509206134092051381CFDF91D4
:10B28000CF911F910F91FF90EF90DF90CF90BF90E3
:10B29000AF909F908F907F906F905F904F903F9076
:10B2A0002F900895AF92BF92CF92DF92EF92FF92CC
:10B2B0000F931F93CF93DF93CDB7DEB7E6970FB60B
:10B2C000F894DEBF0FBECDBF009133051091340559
:10B2D000F80101900020E9F731976F01C01AD10AF7
:10B2E000F801CF01801B910B8C159D053CF48191D9
:10B2F0008F32B9F7DF0111971C92F3CF8BE1E9E4AC
:10B30000F4E1DE015C9601900D928A95E1F7F12C53
:10B31000E12CEC14FD040CF05DC0F801EE0DFF1DF6
:10B320008081811103C08FEFE81AF80A5801AE0C32
:10B33000BF1CF5018081882309F44CC0FFEFEF1A90
:10B34000FF0AF801EE0DFF1D7F01E01AF10A81915D
:10B350008111FACFCE014C960E9496B38BE1FE018B
:10B360007C96DE01119601900D928A95E1F7B50168
:10B37000CE0101960E94A4ABCE0101960E948B2FB4
:10B380008FE20E9403388091971181113BC08DEDAF
:10B3900093E00E9403AF8091291484FF1BC019829F
:10B3A0001C8221E0A501BE01645E7F4FCE010196A3
:10B3B0000E94D8B5811129C08AE00E9403380E94FA
:10B3C0000F4EB50186E297E10E942C57CE010196FF
:10B3D0000E948B2F8AE00E940338CE014C960E9477
:10B3E0008B2FE6960FB6F894DEBF0FBECDBFDF9170
:10B3F000CF911F910F91FF90EF90DF90CF90BF9072
:10B40000AF90089587E991E1C4CFCE014C960E9498
:10B4100005B38BE1FE013196DE015C9601900D9241
:10B420008A95E1F7CE0101960E948B2F72CF2F9261
:10B430003F924F925F926F927F928F929F92AF92C4
:10B44000BF92CF92DF92EF92FF920F931F93CF9311
:10B45000DF9300D000D000D01F921F92CDB7DEB78F
:10B46000B82E8091890D843008F0D1C10E94E3FC90
:10B470006B017C018091890D811108C080919C0C29
:10B4800090919D0C891B8F7709F4A4C681E6A82EA4
:10B4900013C08A3019F08D3009F0F6C01092840D77
:10B4A0008091220D9091230DFC01E25EF24F1682F5
:10B4B000892BF1F40E9406C28091890D843008F036
:10B4C000ECC080919C0C90919D0C891B8F7709F4A6
:10B4D000E4C00E94095697FFDCCF0E940B4E85EB1B
:10B4E00095E00E943C3880919C0C80939D0CE4CFA9
:10B4F0001092230D1092220D04E21DE0F8018191BB
:10B50000803209F446C08E3409F0A9C060EB75E0C2
:10B51000C8010F9487244C01892B41F06EE470E040
:10B52000C80104960F94282F009709F4C8014AE037
:10B5300050E070E060E001960F94F7212B013C0190
:10B5400080911E0D90911F0DA091200DB091210DA5
:10B550000196A11DB11D481659066A067B0629F001
:10B5600060E08DE795E0892851F16AE270E0C8015A
:10B570000F94572F9C01009729F1982F901B912C25
:10B58000992349F09150F801E90FF11D8081982627
:10B59000F7CF8F01B3CF4AE050E070E060E0C9011F
:10B5A00001960F94F721292D30E050E040E062171A
:10B5B00073078407950751F060E08EE595E00E94DF
:10B5C00038E77ACF60E084E395E0F9CF40921E0D32
:10B5D00050921F0D6092200D7092210D8091E10616
:10B5E0008130E1F067E470E0C8010F94282F0097E4
:10B5F000A9F04AE050E070E060E001960F94F72176
:10B60000643071058105910548F483E994E00E9456
:10B610003C3860E089E894E00E94AA3FC09280072D
:10B62000D0928107E0928207F09283078091240DE7
:10B630008B3309F441CF8091890D843008F03CCFE1
:10B6400080918B0D8A9DC001112464E27DE08457B6
:10B65000924F0F94332F80E00E94F2E62DCF80911D
:10B66000291480FFBBCF62E77DE2C8010F948724D5
:10B67000009731F0FC01838180538A3008F0AECF0F
:10B6800060E08AE095E09BCF22E23DE044E25DE0AD
:10B6900064E87DE00E940C1D0FCF8091291482FF89
:10B6A000B6C01A82198271E6F72EE0E1EE2EF9E6B5
:10B6B000DF2E8091890D843008F0A9C00E94441DBE
:10B6C0008111A5C041E050E0BE016B5F7F4F8DE866
:10B6D00095E10E9458B10D8110E0019711F00FEF34
:10B6E0001FEF8091951590919615A0919715B091A7
:10B6F00098158093251490932614A0932714B09343
:10B7000028140E94441D0F3F100749F4811107C0FF
:10B710000E940B4E83ED95E00E943C38CACF4091C9
:10B720008B0D242F30E00A3061F00D3051F088236A
:10B7300009F45FC089819A81009719F001969A8374
:10B7400089831092960489819A81F29EF001F39E7A
:10B75000F00D1124E757F24FE80FF91F1382892BE0
:10B7600069F50E9406C20E94441D882309F4A1CFF6
:10B770000E947B618DE895E10E9405B380912014C1
:10B78000882391F18150809320148D9DC001112454
:10B7900062E0875E994F0E945AB8E091201424E03D
:10B7A000E29FF0011124EB5EF94F6081718182818B
:10B7B00093810E945D220E940DAB7BCF1A82198279
:10B7C00081E00E94F2E68091251490912614A091C8
:10B7D0002714B09128148093850D9093860DA09323
:10B7E000870DB093880DBFCF0E940EB3E092E106A3
:10B7F00060CF4F9DA00111244457524F9E012F5FEF
:10B800003F4F66E974E0802F0E940C1D52CF0E94CA
:10B81000E3FC6B017C01B11004C080911B118823F3
:10B8200051F0C0926E11D0926F11E0927011F092AF
:10B830007111BB24B39480910B0590910C05A091DC
:10B840000D05B0910E050097A105B105B1F040912D
:10B850006E1150916F116091701170917111840F80
:10B86000951FA61FB71FA7019601281B390B4A0B6E
:10B870005B0BDA01C901B7FF92C18091130290916D
:10B880001402A0911502B0911602892B8A2B8B2BE2
:10B8900009F099C10E94E3FC4B015C0180911F0CEF
:10B8A000811108C0209181129091821281E02913A8
:10B8B00001C080E02091E3113091E41191E08927EB
:10B8C0002A3A31050CF480E091E040919B045091BC
:10B8D0009C0460919D0470919E04452B462B472B40
:10B8E00009F490E0981789F0882309F4BDC1D501C7
:10B8F000C40180569444A24FBF4F80939B04909301
:10B900009C04A0939D04B0939E0440902C0C5090F6
:10B910002D0C60902E0C70902F0C2091970430917C
:10B9200098044091990450919A04C301B2010F9474
:10B930000A25882319F180919B0490919C04A09181
:10B940009D04B0919E044092970450929804609296
:10B95000990470929A04892B8A2B8B2B09F449C085
:10B96000D501C40180569444A24FBF4F80939B04DD
:10B9700090939C04A0939D04B0939E0480919B049B
:10B9800090919C04A0919D04B0919E040097A10504
:10B99000B10579F1881A990AAA0ABB0AB7FC29C02D
:10B9A00010929B0410929C0410929D0410929E048D
:10B9B00083E396E00E943C3860E08FE196E00E94CD
:10B9C000AA3F8091E5119091E6111816190624F40A
:10B9D00090E080E00E94141F80917A1190917B1179
:10B9E0001816190634F410927B1110927A110E94E5
:10B9F0008CBE8091A3049091A404A091A504B09161
:10BA0000A60446015701881A990AAA0ABB0AD50159
:10BA1000C401B7FDB9C12091811290918212409169
:10BA20002D0280912C02291323C19091F908899F3E
:10BA3000C0011124880F892F881F990B91958D8340
:10BA40008091FA08489FC0011124880F892F881F10
:10BA5000990B91958E830E94E3FC69837A838B8393
:10BA60009C8340E0BE016F5F7F4FCE0105960E9430
:10BA70005E1C6D8170E089E00E94DAFB41E0BE014E
:10BA80006F5F7F4FCE0105960E945E1C6E8170E055
:10BA900087E00E94DAFB80911406882309F467C1CD
:10BAA0000091200210912102C80102972091E51116
:10BAB0003091E611281739070CF459C18090821291
:10BAC0008F82188619861A861B86809181129F8024
:10BAD000891509F4E7C0892D90E03CE5A32EA89EC6
:10BAE000F001A99EF00D1124E250F74F45895689C7
:10BAF0006789708D452B462B472B81F4418D528DE4
:10BB0000638D748D452B462B472B41F4458D568D07
:10BB1000678D70A1452B462B472BE1F12CE5B22E0A
:10BB2000B89E9001B99E300D1124A9014250574F83
:10BB30001A01FA0161817281838194810F94882EA8
:10BB40004B015C01F10161A172A183A194A10F9449
:10BB50000F252B013C01F10165A176A187A190A5DC
:10BB60000F940F259B01AC01C301B2010F94D42C9B
:10BB7000A50194010F9470254B015C01288539853E
:10BB80004A855B850F943A2E181624F48886998688
:10BB9000AA86BB868F818F5F87708F8396CF0E9426
:10BBA0000B4E60917E0770917F0782EE95E00E94B8
:10BBB0002C578AE00E94033840E070E060E090E09B
:10BBC00080E00E943E5590918112809182129817D8
:10BBD00049F0C0926E11D0926F11E0927011F09204
:10BBE000711158CEBB2019F01092A70453CE0E94B9
:10BBF000E3FC00916E1110916F1120917011309142
:10BC000071118090130290901402A0901502B090D0
:10BC10001602080D191D2A1D3B1D601B710B820B9E
:10BC2000930B97FDE1CF8091A704811133CE81E082
:10BC30008093A7045F9A8091300C8E7F8093300CA4
:10BC40008A9A8091300C8D7F8093300C809108010E
:10BC500080958170809306018091300C8B7F80935A
:10BC6000300C0E94F61E16CE80E090E0DC0145CE3E
:10BC7000209182125CE5259F900111242250374FBC
:10BC8000F901EA5AFF4F9081899FC0011124880F62
:10BC9000892F881F990B91958D83295A3F4FF90160
:10BCA0008081D0CE20911A0230911B0240911C025B
:10BCB00050911D02688579858A859B850F94702532
:10BCC0004B015C01B801012E000C880B990B0F94FD
:10BCD00011259B01AC01C501B4010F94DA2B6983D6
:10BCE0007A838B839C8340911E0250911F02B8017E
:10BCF000CE0101960E94C4C189809A80AB80BC802D
:10BD000040909F045090A0046090A1047090A20401
:10BD1000A3019201C501B4010F940A2587FF16C043
:10BD200028E431EE4AE75FE3C301B2010F947025C6
:10BD300020E037ED43EA5CE30F94DA2BA501940190
:10BD40000F94702569837A838B839C8369817A81C0
:10BD50008B819C8160939F047093A0048093A104C5
:10BD60009093A2040F94462DCB010E94141FF4E679
:10BD7000CF0ED11CE11CF11CC092A304D092A404EC
:10BD8000E092A504F092A6040E9406C28091E1060A
:10BD9000882309F4E0C180912602882309F4A3C016
:10BDA0008091E50481119FC080911B11811108C011
:10BDB00080911C11813021F08091291482FF93C061
:10BDC000F894649B10C08091220290912302A0916C
:10BDD0002402B09125028093E2059093E305A0939D
:10BDE000E405B093E5056091E2057091E30580916B
:10BDF000E4059091E505789420E030E0A9010F94E6
:10BE00000A2587FF70C001E00093E50480911B11B3
:10BE1000811167C088E496E00E943C388AE00E9465
:10BE2000033884E08093990C82E08093850C81E054
:10BE30009AE59093C0138093BF138EE490E09093A3
:10BE4000C2138093C11387E08093B31382E8809379
:10BE5000B61384E890E0A0E0B0E08093B71390932D
:10BE6000B813A093B913B093BA1383E693E10E9479
:10BE70007F340E9427400093891140E36CE876E00C
:10BE800084E799E00E942C4061E088E699E00E94F6
:10BE90000E4010910F0560E010278CE399E069F4E3
:10BEA0008AE796E00E94773F80E30E9403388AE0A9
:10BEB0000E94033860E08DE596E00E94773F88E6B7
:10BEC00096E00E943C3880E30E9403388AE00E949A
:10BED0000338112331F083E696E090937F0C809332
:10BEE0007E0C0E947B6190910901892F8095817061
:10BEF000109100021817C9F0209129142062209394
:10BF000029148093000290FD3FC164EF71E080E04E
:10BF100090E00E9400260E9430B38091291483FD96
:10BF20007CC1111133C10E94D1350E94E3FC6B0129
:10BF30007C01109117021123F1F0809110058823E4
:10BF4000D1F04091A8045091A9046091AA04709185
:10BF5000AB0446015701841A950AA60AB70AB5012F
:10BF6000A40177FD1AC0833009F42FC10CF01EC163
:10BF700081300CF023C1212F30E0A8EEB3E00F9404
:10BF8000A22BC60ED71EE81EF91EC092A804D0929E
:10BF9000A904E092AA04F092AB0480911C118130B4
:10BFA00009F073C00E94E3FC6B017C018091B00436
:10BFB0009091B104A091B204B091B304A70196018D
:10BFC000281B390B4A0B5B0BDA01C901B7FD3AC0DC
:10BFD000D701C601805F984DAF4FBF4F8093B0042B
:10BFE0009093B104A093B204B093B3048090AB05D6
:10BFF0009090AC05A090AD05B090AE050E94742B5A
:10C00000AB01BC014093AB055093AC056093AD050B
:10C010007093AE058091900690919106A091920642
:10C02000B091930688199909AA09BB09840F951F35
:10C03000A61FB71F8093900690939106A093920637
:10C04000B09393068091AC049091AD04A091AE049E
:10C05000B091AF0446015701881A990AAA0ABB0A8F
:10C06000D501C401B7FD11C020E8C20E2EEED21ECC
:10C0700026E3E21EF11CC092AC04D092AD04E09223
:10C08000AE04F092AF040E94C0530E947A390E941D
:10C09000444180910A05882379F10E94E3FC6B01F9
:10C0A0007C018091060590910705A0910805B0914B
:10C0B000090546015701881A990AAA0ABB0AD5013F
:10C0C000C401B7FD19C020910A0530E0A8EEB3E025
:10C0D0000F94A22BC60ED71EE81EF91EC0920605AD
:10C0E000D0920705E0920805F092090580E00E94D1
:10C0F000EABA8AE00E94033880910505882359F145
:10C100000E94E3FC6B017C01809101059091020586
:10C11000A0910305B0910405A7019601281B390BD6
:10C120004A0B5B0BDA01C901B7FD15C0209105056B
:10C1300030E0A8EEB3E00F94A22BC60ED71EE81E87
:10C14000F91EC0920105D0920205E0920305F0921B
:10C1500004050E94CBAA2B960FB6F894DEBF0FBE43
:10C16000CDBFDF91CF911F910F91FF90EF90DF90A6
:10C17000CF90BF90AF909F908F907F906F905F9087
:10C180004F903F902F9008950E941FB3123008F0F7
:10C19000CCCE0E94D13560E085EC96E050C083EDB6
:10C1A00096E090937F0C80937E0CBFCE843009F094
:10C1B000E2CE0E940F4E8AED96E004C00E940F4E20
:10C1C00089E097E00E943C38D6CE0E940F4E82EF65
:10C1D00096E0F8CF8091800790918107A091820727
:10C1E000B0918307A7019601281B390B4A0B5B0B03
:10C1F000DA01C901885E9340A109B109B7FD46C9BA
:10C200008DEC95E00E943C38C0928007D092810767
:10C21000E0928207F092830739C9123098F48DE9D1
:10C2200096E00E943C388AE00E9403380E94A22CCB
:10C2300090E080E00E94365760E086EB96E00E9436
:10C24000AA3F73CE123009F070CE0E948AB78823BD
:10C2500079F081E00E9460B742EB50E06AE078E05C
:10C260008EE294E10E9458B18EE294E10E9405B3FF
:10C270000E94792F811193CF0E94632F0E9406B8EC
:10C280000E945BB752CECF93DF9380918112909141
:10C290008212891B8095877019F40E94175AF5CF76
:10C2A000809181128F5F8770A09181129CE5A99F78
:10C2B000D0011124FD01E250F74FEF0119929A9538
:10C2C000E9F798E09083AD5EB64F90E1E3E8F2E1E4
:10C2D00001900D929A95E1F720918112909182122E
:10C2E000291303C094E690937E1280938112DF910C
:10C2F000CF910C94912F909181128091821298137A
:10C3000006C08091FC089091FD08892B21F080E007
:10C310000E94175AF0CF0895FC012081318142819B
:10C3200053816091560C7091570C8091580C9091EC
:10C33000590C0F9470250F94472E60938F127093B1
:10C340009012809391129093921290918112809109
:10C35000821298130C9443610E947B610E94002A10
:10C3600040918F125091901260919112709192129F
:10C3700040930406509305066093060670930706E3
:10C3800081110C94912F08954F925F926F927F923A
:10C390008F929F92AF92BF92CF92DF92EF92FF92D5
:10C3A0000F931F93CF93DF93EC018B015A01F90197
:10C3B0002091560C3091570C4091580C5091590CCB
:10C3C00060817181828193810F9470250F94472E33
:10C3D0006B017C012091520C3091530C4091540C14
:10C3E0005091550CF50160817181828193810F9488
:10C3F00070250F94472E4B015C0120914E0C30911B
:10C400004F0C4091500C5091510CF801608171819A
:10C41000828193810F9470250F94472E2B013C014C
:10C4200020914A0C30914B0C40914C0C50914D0C8A
:10C43000688179818A819B810F9470250F94472EA2
:10C440006093831270938412809385129093861266
:10C4500040928712509288126092891270928A12CA
:10C4600080928B1290928C12A0928D12B0928E12AA
:10C47000C0928F12D0929012E0929112F09292128A
:10C480009091811280918212981791F0DF91CF9153
:10C490001F910F91FF90EF90DF90CF90BF90AF90E2
:10C4A0009F908F907F906F905F904F900C9443611E
:10C4B0000E947B610E94002A40918B1250918C1245
:10C4C00060918D1270918E120091871210918812D6
:10C4D0002091891230918A12C0908312D0908412D8
:10C4E000E0908512F0908612C092F805D092F9057E
:10C4F000E092FA05F092FB050093FC051093FD0510
:10C500002093FE053093FF054093000650930106EB
:10C51000609302067093030640918F12509190121F
:10C520006091911270919212409304065093050607
:10C530006093060670930706882391F0DF91CF91F0
:10C540001F910F91FF90EF90DF90CF90BF90AF9031
:10C550009F908F907F906F905F904F900C94912F51
:10C56000DF91CF911F910F91FF90EF90DF90CF90CF
:10C57000BF90AF909F908F907F906F905F904F9003
:10C5800008953F924F925F926F927F928F929F9207
:10C59000AF92BF92CF92DF92EF92FF920F931F93D1
:10C5A000CF93DF93CDB7DEB768970FB6F894DEBFB1
:10C5B0000FBECDBFD82E2A013B01480159013E2CA8
:10C5C00020E030E0A901C501B8010F940A258111CE
:10C5D00010C081E08D1508F0B6C060E070E080E723
:10C5E00093E420E030E040E752E40F94D42C4B0178
:10C5F0005C018D8A9E8AAF8AB88E0D2D10E0F801FD
:10C60000E456F64EE491BB24B3941E160CF4B12C00
:10C61000CC24C39420E030E0A901C301B2010F94FF
:10C620003A2E18160CF0C12CBC1471F092E0D912FD
:10C630000BC0332049F081E00E94B2F869E170E05C
:10C6400080E090E00E94002680E00E94972F69839E
:10C650007A838B839C8381E00E94972F6D837E83F6
:10C660008F83988782E00E94972F69877A878B87CC
:10C670009C8783E00E94972F6D877E878F87988B9A
:10C68000000F111F000F111FE1E0F0E0EC0FFD1F84
:10C690000E0F1F1FF80110821182128213829E0159
:10C6A000235F3F4FAE01475F5F4FBE016B5F7F4F20
:10C6B000CE0101960E94C461F801408251826282DB
:10C6C0007382198A1A8A1B8A1C8A8091FC089091AD
:10C6D000FD08892B91F4CE0141967C018E010B5E01
:10C6E0001F4F9E01235F3F4FAE01475F5F4FBE016B
:10C6F0006B5F7F4F40970E945CE70E947B61BC1498
:10C7000051F092E0D91205C0332019F080E00E9468
:10C71000B2F80E94FB5568960FB6F894DEBF0FBEC4
:10C72000CDBFDF91CF911F910F91FF90EF90DF90E0
:10C73000CF90BF90AF909F908F907F906F905F90C1
:10C740004F903F90089560E070E88BE395E449CF07
:10C750004F925F926F927F928F929F92AF92BF9211
:10C76000CF92DF92EF92FF920F931F93CF93DF93BD
:10C77000CDB7DEB72C970FB6F894DEBF0FBECDBF96
:10C780002B013C0129873A874B875C874701580179
:10C79000F601E080F1800281138120E030E0A90100
:10C7A000B701C8010F940A25882309F488C05E2DBB
:10C7B0004F2D302F212F852F942FA32FB22F898318
:10C7C0009A83AB83BC8320E030E0A901B701C801A4
:10C7D0000F940A25811108C0E0903D02F0903E02BE
:10C7E00000913F0210914002C701D8018D839E83C2
:10C7F000AF83B887A50194016091280C7091290C32
:10C8000080912A0C90912B0C0F940A2587FF0CC065
:10C810008092280C9092290CA0922A0CB0922B0C9A
:10C82000CE0101960E94DB2A4092200C5092210CEE
:10C830006092220C7092230C89859A85AB85BC8509
:10C840008093240C9093250CA093260CB093270C76
:10C85000CE0105960E94DB2AA50194016091280C67
:10C860007091290C80912A0C90912B0C0F943A2EE8
:10C87000181664F48092280C9092290CA0922A0C2D
:10C88000B0922B0CCE0101960E94DB2A0E947B61A4
:10C890002C960FB6F894DEBF0FBECDBFDF91CF91BF
:10C8A0001F910F91FF90EF90DF90CF90BF90AF90CE
:10C8B0009F908F907F906F905F904F90089550E081
:10C8C00040E030E820E477CFCF92DF92EF92FF9202
:10C8D0000F931F936A01E090280CF090290C0091AF
:10C8E0002A0C10912B0CFB01208131814281538154
:10C8F000FC0160817181828193810E94A8631F91F4
:10C900000F91FF90EF90DF90CF900895CF92DF923C
:10C91000EF92FF920F931F936B01FC01E080F18077
:10C9200002811381E0E2FCE0248135814681578158
:10C9300060817181828193810E94A8631F910F9110
:10C94000FF90EF90DF90CF9008950F931F93CF93B8
:10C95000DF93EC018B0181E00E94B2F869E170E0A5
:10C9600080E090E00E940026B801CE010E9486641B
:10C97000C091E00680E00E94B2F81092E00682E0EA
:10C980000E94C12F0E94F62AC2FBCC27C0F981E089
:10C990008C27DF91CF911F910F910895AF92BF9295
:10C9A000CF92DF92EF92FF920F931F93CF93DF937B
:10C9B00000D01F92CDB7DEB7FC01E080F18002818C
:10C9C0001381611112C0A090280CB090290CC09066
:10C9D0002A0CD0902B0C9501A601B701C8010F9429
:10C9E0000A2587FF02C07501860120E030E048EC8F
:10C9F00053E4B701C8010F940A2587FD04C0E12C58
:10CA0000F12C08EC13E4C701D80189839A83AB8326
:10CA1000BC8362EE72E0CE0101960E9486640F90A4
:10CA20000F900F900F90DF91CF911F910F91FF907A
:10CA3000EF90DF90CF90BF90AF9008953F924F92CC
:10CA40005F926F927F928F929F92AF92BF92CF929E
:10CA5000DF92EF92FF920F931F93CF93DF9300D05B
:10CA60001F92CDB7DEB7382E80E090E0A0E2B1E4AF
:10CA700089839A83AB83BC83C0907812D09079125B
:10CA8000E0907A12F0907B1220E030E0A901C7011B
:10CA9000B6010F940A2587FF0CC0A701960160E03C
:10CAA00070E080E291E40F94D92B69837A838B83C1
:10CAB0009C8360E0CE0101960E94CE644090200CE1
:10CAC0005090210C6090220C7090230C8090240CCC
:10CAD0009090250CA090260CB090270C332089F163
:10CAE0000E94C65419821A821B821C82E090280C74
:10CAF000F090290C00912A0C10912B0CCE0101967C
:10CB00006C01A5019401C301B2010E94A863309297
:10CB10007C070E94652B0F900F900F900F90DF9174
:10CB2000CF911F910F91FF90EF90DF90CF90BF902A
:10CB3000AF909F908F907F906F905F904F903F90BD
:10CB400008950E948354CECF80917C07882319F0EA
:10CB500080E00E941E6580E008952F923F924F92E0
:10CB60005F926F927F928F929F92AF92BF92CF927D
:10CB7000DF92EF92FF920F931F93CF93DF93CDB786
:10CB8000DEB766970FB6F894DEBF0FBECDBFF82EA6
:10CB9000282E312CF101E456F64ED49022E0821377
:10CBA00035C080917C07811103C081E00E941E6521
:10CBB0000E94C654811139C188E999E10E947D1D06
:10CBC00020E030E0A9010F940A258823F9F06D2DAB
:10CBD000DD0C770B880B990B0F9411252B013C0171
:10CBE00088E999E10E947D1D4B015C0120E030E065
:10CBF00040EA50E40F940A2511E087FF1CC0812C05
:10CC0000912C90EAA92E90E4B92E15C06D2DDD0C63
:10CC1000770B880B990B0F9411252B013C01C10157
:10CC2000880F991F880F991F8057964E0E947D1D6F
:10CC30004B015C0110E0A3019201C501B4010F9406
:10CC400070254B015C016101CC0CDD1CCC0CDD1CA2
:10CC5000C6018C57964E0E947D1DEE24E394E1267A
:10CC600020E030E040EC5FE30F947025A3019201D7
:10CC70000F947025AB01BC0100E010E098018F2DEE
:10CC80000E94C16220E030E0A901C501B4010F9407
:10CC90000A25F601E858F64EFA8BE98B882309F449
:10CCA0004DC0F2E000E010E020E431E4FF1619F09E
:10CCB00000E010E09801B501A4017058E12C8F2D1F
:10CCC0000E94C162A5019401C501B4010F94DA2B41
:10CCD0006B8B7C8B8D8B9E8B22E0F216E9F0F10141
:10CCE000EB58F64E6491611107C00E940F4E83E528
:10CCF00099E10E943C386AE070E090E080E00F9497
:10CD00000F259B01AC0160E070E088E492E40F9491
:10CD1000D42C8B019C0104C000E010E020EC30E436
:10CD2000EE24E3944B895C896D897E898F2D0E9466
:10CD3000C16232E0F312D0C00E94835481E090E0DF
:10CD4000A0E0B0E00F2C04C0880F991FAA1FBB1FE2
:10CD50000A94D2F72091300C282B2093300C20918C
:10CD60009605822B8093960589899A890E947D1D5C
:10CD7000F601E05EF34F608371838283938382E0E8
:10CD8000F8121AC0209178123091791240917A12DB
:10CD900050917B126091280C7091290C80912A0C83
:10CDA00090912B0C0F94D92B6093280C7093290C25
:10CDB00080932A0C90932B0CF601EE50F84F1082C2
:10CDC0001182128213828F2D0E949A1C0E94F62AD1
:10CDD000F601E05EF34F80819181A281B381F6017B
:10CDE000E459F84F80839183A283B38392E0F916CC
:10CDF000A9F18CE0EEEAF2E0DE01119601900D92CD
:10CE00008A95E1F7E1E0F0E0EC0FFD1FEC0DFD1D70
:10CE100080809180A280B38020E030E0A901C5012C
:10CE2000B4010F940A2581111EC066960FB6F894BE
:10CE3000DEBF0FBECDBFDF91CF911F910F91FF904D
:10CE4000EF90DF90CF90BF90AF909F908F907F90AA
:10CE50006F905F904F903F902F9008950E94A4652F
:10CE60008111E3CFC6CF20E030E0A901C501B401B4
:10CE70000F943A2E87FF04C0B7FAB094B7F8B09475
:10CE8000F601E05EF34F6F01A3019201C501B40109
:10CE90000F9470259B01AC01F60160817181828144
:10CEA00093810F94D92BF6016083718382839383DE
:10CEB000F2E080E090E0A0E4B1E4FF1621F080E031
:10CEC00090E0A8E4B2E48D879E87AF87B88BCE014F
:10CED0000D960E94DB2AA9CF81E090E0A0E0B0E0AF
:10CEE0000F2C04C0880F991FAA1FBB1F0A94D2F7EA
:10CEF0002091300C282B2093300C20919605822B0A
:10CF00008093960589899A890E947D1DF601E05ECD
:10CF1000F34F60837183828393834ECFCF93DF93EC
:10CF200000D01F92CDB7DEB780E090E0A0EAB0E479
:10CF300089839A83AB83BC8361E0CE0101960E9412
:10CF4000CE640F900F900F900F90DF91CF910895C6
:10CF50008F929F92AF92BF92CF92DF92EF92FF9209
:10CF60000F931F93CF93DF93CDB7DEB72C970FB6F8
:10CF7000F894DEBF0FBECDBF8B0140E050E068E407
:10CF800072E44D835E836F83788740E050E060EA0F
:10CF900070E449875A876B877C878130B9F182308A
:10CFA00009F459C020E030E040E050E46091280CE2
:10CFB0007091290C80912A0C90912B0C0F94DA2BF4
:10CFC0004B017C0120E030E048EC53E40F943A2E12
:10CFD000181634F4812C912C88ECE82E93E4F92E69
:10CFE000F801A084B184C284D3849401A701B5015F
:10CFF000C6010F943A2E181614F054016701C501AA
:10D00000D60189839A83AB83BC8348C0BE01675F26
:10D010007F4FC80108960E948664B8016C5F7F4FFD
:10D02000AE014B5F5F4FC8010E9464640E94913063
:10D030002C960FB6F894DEBF0FBECDBFDF91CF9117
:10D040001F910F91FF90EF90DF90CF90BF90AF9026
:10D050009F908F900895F8012085318542855385F2
:10D060006091280C7091290C80912A0C90912B0CC6
:10D070000F94DA2B6B017C0120E030E048EC53E4A4
:10D080000F940A2587FD06C0C12CD12C28ECE22E76
:10D0900023E4F22EC982DA82EB82FC82BE01675F52
:10D0A0007F4FCE010196B7CFEF92FF920F931F9360
:10D0B000CF93DF937C018B010E948B31C0E2DCE0D7
:10D0C00020916102309162024091630250916402AA
:10D0D000F70160817181828193810F94D42C2C851A
:10D0E0003D854E855F850F94DA2B6C877D878E8713
:10D0F0009F87C8010E94DB2ADF91CF911F910F917A
:10D10000FF90EF900C947B614F925F926F927F92B1
:10D11000AF92BF92CF92DF92EF92FF920F931F9345
:10D12000CF93DF9300D000D01F921F92CDB7DEB710
:10D130005C0180E090E0A0E7B2E489839A83AB834E
:10D14000BC8380E090E0A0E8B0EC8D839E83AF8349
:10D15000B887BE016F5F7F4FCE0105960E9454686D
:10D1600068E873E180E090E00E940026C12CD12C99
:10D1700088ECE82E81E4F82EC982DA82EB82FC8208
:10D1800080E090E0A0E8B0E48D839E83AF83B88711
:10D19000BE016F5F7F4FCE0105960E94546806E383
:10D1A0001CE0F80140AC51AC62AC73ACC0AED1AE87
:10D1B000E2AEF3AE80E090E0A0EAB1E489839A8326
:10D1C000AB83BC83F50180819181A281B3818D8382
:10D1D0009E83AF83B887BE016F5F7F4FCE010596F8
:10D1E0000E945468F80140AE51AE62AE73AE129A1E
:10D1F00064E670E080E090E00E94002681E02896DE
:10D200000FB6F894DEBF0FBECDBFDF91CF911F9157
:10D210000F91FF90EF90DF90CF90BF90AF907F90F5
:10D220006F905F904F9008951F93CF93DF93CDB78A
:10D23000DEB72C970FB6F894DEBF0FBECDBF182F08
:10D24000882379F020E030E0A9016091CE0570914B
:10D25000CF058091D0059091D1050F940A258823A0
:10D26000F9F08091310C8117D9F00E947B618CE03C
:10D27000EAEBF2E0DE01119601900D928A95E1F75A
:10D28000CE0101960E94291F8091310C882391F0D4
:10D2900080E29CE00E9402271092310C0E94F62A44
:10D2A0002C960FB6F894DEBF0FBECDBFDF91CF91A5
:10D2B0001F91089581E08093310C80E29CE00E94F0
:10D2C0001621ECCF2F923F924F925F926F927F92F6
:10D2D0008F929F92AF92BF92CF92DF92EF92FF9286
:10D2E0000F931F93CF93DF93CDB7DEB7CB54D10904
:10D2F0000FB6F894DEBF0FBECDBF2DB73EB739AF26
:10D3000028AF87E00E941F4E81110BC061E086E5C7
:10D310000E944E248DA3853060F087E39EE00E943A
:10D320003C38A8ADB9AD0FB6F894BEBF0FBEADBFC7
:10D3300040C33DA1332321F087E19EE00E943C38A9
:10D340006AE080E50E944E24182F8CEF810F8F3207
:10D3500018F083EF9DE0E3CF60E085E40E946A244B
:10D36000882309F448C081E08FABE0907C12F090F4
:10D370007D12D7012D913D914D915C916091200CD2
:10D380007091210C8091220C9091230C0F94DA2B38
:10D39000AB01BC0188E50E94BC2469877A878B8732
:10D3A0009C87F70124813581468157816091240C47
:10D3B0007091250C8091260C9091270C0F94DA2BFC
:10D3C000AB01BC0189E50E94BC246D877E878F87F5
:10D3D000988BBE01635F7F4FCE0109960E94302E6D
:10D3E000382E81110BC063E68FED9DE00E94AA3FAD
:10D3F00087EC9DE094CF92E09FABB7CF8CE40E9486
:10D400003E1E082F882309F431C10E943A248EA3BE
:10D41000803118F080EA9DE082CFFEA1F13009F45E
:10D4200027C160E083E50E946A248AAF882321F047
:10D43000011102C037E03EA38DA1833020F086E8C1
:10D440009DE00E943C389091310C9DAF80E00E949D
:10D4500014690E94D31C1D8A1E8A1F8A188E198E79
:10D460001A8E1B8E1C8E83EF9FE4A3ECB7E48D8F86
:10D470009E8FAF8FB8A383EF9FE4A3ECB7EC89A393
:10D480009AA3ABA3BCA3A12FB0E0BCA7ABA7EDB7F9
:10D49000FEB724E0129FE019F10911240FB6F894A9
:10D4A000FEBF0FBEEDBF8DB79EB701969CAF8BAF91
:10D4B0002DA14FA9BE01635F7F4FCE0109960E9447
:10D4C00041F99B01AC010F94CC2E811162C20E94E4
:10D4D000E3FC611571058105910511F00F94902011
:10D4E000212C1BAA1CAA1DAA1EAAAEA1A150BB0BCF
:10D4F0002C96BFAFAEAF2C97E22DF0E0F8A7EFA3CC
:10D500002BA53CA5E217F3070CF074C23196FEA7D9
:10D51000EDA73F932F93FF93EF9382E79DE09F93B7
:10D520008F938CE79DE09F938F931F920E94D0F87A
:10D530008DB79EB709960FB6F8949EBF0FBE8DBFEC
:10D540009EA1992309F458C10F9441202AE030E0AC
:10D5500040E050E00F94702B0F94112520E030E054
:10D5600040EA50E40F943A2E0FEF1FEF181614F014
:10D5700001E010E00F94412028E631E040E050E067
:10D580000F94702B0F9411252B013C010F94412017
:10D5900020E230E040E050E00F94702B6B5F7F4F53
:10D5A0008F4F9F4F0F9411254B015C01ADA1A4300B
:10D5B000D1F4BC01A40184E69DE00E941841B301AE
:10D5C000A2018CE59DE00E94184186E59DE00E9445
:10D5D0003C380130110519F483E40E94033882E5D8
:10D5E0009DE00E943C38312CC801110FAA0BBB0BE7
:10D5F0002A968CAF9DAFAEAFBFAF2A972C96AEAD3B
:10D60000BFAD2C973A161B060CF0F6C02A966CADEF
:10D610007DAD8EAD9FAD2A970F9411256B017C01D6
:10D62000BAADBB2341F1AC019B010F94DA2B20E092
:10D6300030E040E952E40F9470259B01AC01C30136
:10D64000B2010F94DA2B2B013C0120E030E044EBD7
:10D6500053E40F943A2E1816FCF420E030E044EB2B
:10D6600053E4C301B2010F94D92BEDCF1EA2D9CE42
:10D6700022E02EA3D6CE0F94412024E130E040E0FA
:10D6800050E00F94702B675E7F4F8F4F9F4F0F942A
:10D690001125A7019601CFCF20E030E0A901C301F9
:10D6A000B2010F940A2587FF0BC020E030E044EB65
:10D6B00053E4C301B2010F94DA2B2B013C01ECCFF0
:10D6C00000917C1210917D12F801248135814681F0
:10D6D00057816D857E858F8598890F94D92B2296E9
:10D6E0006CAF7DAF8EAF9FAF22972BED3FE049E44B
:10D6F00050E4C301B2010F94702520E030E044E310
:10D7000053E40F94D42C6B017C010F94CF2C6FA7A2
:10D7100078AB89AB9AABD8012D913D914D915C913D
:10D7200069857A858B859C850F94D92B26966CAF5D
:10D730007DAF8EAF9FAF2697A50194016FA578A905
:10D7400089A99AA90F9470259B01AC0126966CAD0E
:10D750007DAD8EAD9FAD26970F94DA2B69837A83CA
:10D760008B839C83C701B6010F947A2EA501940187
:10D770000F94702522962CAD3DAD4EAD5FAD229736
:10D780000F94DA2B6D837E838F8398874BE351E070
:10D7900070E060E0CE0101960E94C4C146E351E012
:10D7A00070E060E0CE0105960E94C4C1BDA1B43016
:10D7B00099F449815A816B817C8186E49DE00E94C5
:10D7C00018414D815E816F8178858FE49FE20E94D0
:10D7D00018418AE00E940338198A1A8A1B8A1C8A17
:10D7E000AE014F5E5F4FBE016B5F7F4FCE01019672
:10D7F0000E946464339402CF20E04FA9BE01635FAE
:10D800007F4FCE0109960E9441F94B015C01312CFA
:10D81000AC019B010F94CC2E811102C033243394B0
:10D82000A5019401C501B4010F94CC2E8111E2C071
:10D83000EFA1F8A5EE0FFF1FEE0FFF1F2BAD3CADC4
:10D84000E20FF31F80829182A282B382A50194012C
:10D850006D8D7E8D8F8D98A10F943A2E181624F41D
:10D860008D8E9E8EAF8EB8A2A501940169A17AA17A
:10D870008BA19CA10F940A2587FF04C089A29AA2BC
:10D88000ABA2BCA2A50194016BA97CA98DA99EA9FC
:10D890000F94DA2B6BAB7CAB8DAB9EABADA5BEA56D
:10D8A000BD01BB0F880B990B0F9411256FA378A7AF
:10D8B00089A79AA79B01AC016BA97CA98DA99EA9F8
:10D8C0000F94D42C2B013C014D8A5E8A6F8A788E8E
:10D8D000EBADFCADF8ABEFA710E0C12CD12C76017D
:10D8E000AFA5B8A96D917D918D919D91B8ABAFA772
:10D8F000A30192010F94D92B9B01AC010F947025C9
:10D900009B01AC01C701B6010F94DA2B6B017C01BE
:10D910001F5F211628F72FA138A549A55AA50F94F6
:10D92000D42C0F94882E698F7A8F8B8F9C8FBDA1FA
:10D93000B23068F18DA59EA50E9400E16BA57CA583
:10D9400081E49DE00E943A418BE39DE00E943C38D7
:10D9500043E0C501B4010E9446BA80E20E94033848
:10D9600081E0EDA1E3300CF480E0E12C8E010F5D4D
:10D970001F4F9E01235E3F4FAE01475E5F4FBE01CA
:10D980006B5E7F4F0E94F93E8AE00E940338239429
:10D99000B3CD0E94A4650E94BA1C8DAD0E9414698B
:10D9A0000E94913088AD99AD0FB6F8949EBF0FBE1E
:10D9B0008DBFE8ADF9AD0FB6F894FEBF0FBEEDBF59
:10D9C000C55BDF4F0FB6F894DEBF0FBECDBFDF9152
:10D9D000CF911F910F91FF90EF90DF90CF90BF906C
:10D9E000AF909F908F907F906F905F904F903F90FF
:10D9F0002F9008950E94A465332069F280E39DE092
:10DA00000E943C3881E0FDA11F160CF080E0EE245E
:10DA1000E3948E010F5D1F4F9E01235E3F4FAE01C9
:10DA2000475E5F4FBE016B5E7F4F0E94F93E698D7E
:10DA30007A8D8B8D9C8D0052110926E042E00F9467
:10DA4000D71F9F938F938FE19DE09F938F9389E2E0
:10DA50009DE09F938F931F920E94D0F82DB73EB701
:10DA6000295F3F4F0FB6F8943EBF0FBE2DBF93CF37
:10DA70002F923F924F925F926F927F928F929F92DE
:10DA8000AF92BF92CF92DF92EF92FF920F931F93CC
:10DA9000CF93DF93CDB7DEB76A970FB6F894DEBFAA
:10DAA0000FBECDBF83E50E943E1E182F3090310C73
:10DAB000882319F00E945A24382E4090200C509050
:10DAC000210C6090220C7090230C8091240C90917A
:10DAD000250CA091260CB091270C8B8B9C8BAD8BC9
:10DAE000BE8B8091280C9091290CA0912A0CB091AA
:10DAF0002B0C8F8B988FA98FBA8F112329F031109F
:10DB000003C080E00E94146986E50E943E1E8A8B55
:10DB100020E030E0A9016091CE057091CF058091A1
:10DB2000D0059091D1050F940A25882309F4C9C026
:10DB300083E40E943E1E882309F49DC00E94922423
:10DB40006B017C01A8E8B7E0B987A887BF83AE83E3
:10DB5000F5E0FD831D861E8628EC2F8702EC1A86D1
:10DB6000212C88EC8B8792E49C87AE81BF81B98B96
:10DB7000A88B15E0E889F98981909190A190B190E6
:10DB8000F98BE88B2A85322D4B855C85C501B40164
:10DB90000F940A2587FF04C08A86292CAB86BC8691
:10DBA0002D853E854F85502FC501B4010F943A2E27
:10DBB000181624F48D869E86AF860B2D1150D1F653
:10DBC000FD81F150FD838E819F8144969F838E83DA
:10DBD000F111CBCF2D853E854F85502F6A85722D53
:10DBE0008B859C850F94DA2B20E030E040E05FE3EA
:10DBF0000F947025A70196010F94DA2B4B015C015D
:10DC00002DEB37E346E855EB0F943A2E87FD0AC01B
:10DC10002DEB37E346E855E3C501B4010F940A251F
:10DC200018164CF580E00E94146910E0E884F9842D
:10DC300000E0D7016D917D918D919D917D016D01E8
:10DC4000B4E0CB1AD108A50194010F94D92BF601A9
:10DC50006083718382839383602F812F0E94A5F755
:10DC60000F5F053031F71F5F888599854496998746
:10DC700088871530D9F6AA89AA2381F020E030E000
:10DC8000A9016091CE057091CF058091D00590914A
:10DC9000D1050F940A2581110E9481408AE50E94D6
:10DCA0003E1E882351F00E94922469837A838B83DD
:10DCB0009C83CE0101960E946DF6832D0E9414690B
:10DCC0000BC0311003C09A89992341F30E940F4E73
:10DCD00080E69CE00E943C38332051F08091310C6A
:10DCE000811106C00E940B4E81E49CE00E943C38EA
:10DCF0000E940F4E83E39CE00E943C388091310CDF
:10DD00000E94FA400E940F4E86E29CE00E943C383E
:10DD1000C090C408D090C508E090C608F090C7082D
:10DD200020E030E0A901C701B6010F943A2E181681
:10DD30000CF053C042E0C701B6010E9446BA8DE024
:10DD40000E9403388AE00E940338A3019201609187
:10DD5000200C7091210C8091220C9091230C0F9437
:10DD60000A2581111FC02B893C894D895E896091EC
:10DD7000240C7091250C8091260C9091270C0F9407
:10DD80000A2581110FC02F89388D498D5A8D6091D8
:10DD9000280C7091290C80912A0C90912B0C0F94D7
:10DDA0000A2581110E9491306A960FB6F894DEBF61
:10DDB0000FBECDBFDF91CF911F910F91FF90EF90DC
:10DDC000DF90CF90BF90AF909F908F907F906F909B
:10DDD0005F904F903F902F90089581E29CE00E94C9
:10DDE0003C38B3CF8F929F92AF92BF92EF92FF9247
:10DDF0000F931F93CF93DF9380E00E9414691092DA
:10DE0000CA051092CB051092CC051092CD05109248
:10DE1000C6051092C7051092C8051092C905109248
:10DE2000D2051092D3051092D4051092D505109208
:10DE3000CE051092CF051092D0051092D10508E8BA
:10DE400017E0C0E0812C912C80ECA82E8FE7B82E33
:10DE50007801D0E0F70181929192A192B1927F0175
:10DE60006D2F8C2F0E94A5F7DF5FD53099F7CF5F1C
:10DE70000C5E1F4FC53061F7DF91CF911F910F915D
:10DE8000FF90EF90BF90AF909F908F9008959091EA
:10DE9000811280918212981308C08091FC089091A1
:10DEA000FD08892B11F40C94F81E80E00E94175A8B
:10DEB000EECF83E50E948C1E8823E9F00E94E3FCEC
:10DEC00060936E1170936F11809370119093711124
:10DED0000E94922420E030E04AE754E40F94702539
:10DEE0000F944D2D609313027093140280931502CA
:10DEF00090931602089580912F0584FD0AC08091A9
:10DF0000310587FD06C080913205837011F40C94B1
:10DF1000476F0E947B6188E50E943E1E882331F096
:10DF20005F9A8091300C8E7F8093300C89E50E943F
:10DF30003E1E882331F08A9A8091300C8D7F809329
:10DF4000300C8AE50E943E1E882359F0809108011A
:10DF500080958170809306018091300C8B7F809337
:10DF6000300C85E40E943E1E81110C94F61E08952B
:10DF70002F923F924F925F926F927F928F929F92D9
:10DF8000AF92BF92CF92DF92EF92FF920F931F93C7
:10DF9000CF93DF93CDB7DEB7A6970FB6F894DEBF69
:10DFA0000FBECDBF8CE697E00E94232A8091DE0B46
:10DFB00083FD7EC020912C0C30912D0C40912E0CB5
:10DFC00050912F0C609178077091790780917A07B2
:10DFD00090917B070F940A25882309F469C010915A
:10DFE000FB08111161C080915F029091600201975E
:10DFF0002091E3113091E411281739073CF40E9475
:10E000000F4E86E299E10E943C3811E020912C0CE1
:10E0100030912D0C40912E0C50912F0C609178076F
:10E020007091790780917A0790917B070F94D92B93
:10E030006B017C0120E030E0A9010F943A2E87FFAC
:10E0400004C0F7FAF094F7F8F0942091610230914F
:10E0500062024091630250916402C701B6010F94BD
:10E06000702520E030E84BE354E40F943A2E181664
:10E07000ECF40E940F4E87E099E10E943C388091B9
:10E08000780790917907A0917A07B0917B078093E8
:10E090002C0C90932D0CA0932E0CB0932F0C88E792
:10E0A00097E00E948C6104C010E0B0CF1111E7CF5F
:10E0B0002AE037ED43E25CE3609141027091420255
:10E0C00080914302909144020F9470256B017C0172
:10E0D0006091670270916802072E000C880B990B03
:10E0E0000F9411259B01AC01C701B6010F94702557
:10E0F000698B7A8B8B8B9C8B8091310C882309F1F7
:10E100008090C4089090C508A090C608B090C70839
:10E11000C0907407D0907507E0907607F09077076D
:10E1200020E030E0A901C501B4010F940A2588233D
:10E13000D1F1A7019601C501B4010F943A2E18162A
:10E1400094F1C12CD12C76018E010F5E1F4F28E770
:10E1500037E044E757E060E777E08CE697E00E941D
:10E1600026F480E1ECE6F7E0A0E2BCE001900D923D
:10E170008A95E1F7A6960FB6F894DEBF0FBECDBF25
:10E18000DF91CF911F910F91FF90EF90DF90CF9093
:10E19000BF90AF909F908F907F906F905F904F90C7
:10E1A0003F902F9008952091200C3091210C4091A8
:10E1B000220C5091230C60916C0770916D07809137
:10E1C0006E0790916F070F94D92B6D8B7E8B8F8B81
:10E1D000988F2091240C3091250C4091260C509161
:10E1E000270C609170077091710780917207909170
:10E1F00073070F94D92B698F7A8F8B8F9C8F209107
:10E20000280C3091290C40912A0C50912B0CC701FD
:10E21000B6010F94D92B6D8F7E8F8F8F98A320918D
:10E220002C0C30912D0C40912E0C50912F0C6091A4
:10E2300078077091790780917A0790917B070F9406
:10E24000D92B6B017C0120E030E0A9016D897E892A
:10E250008F89988D0F940A2581110CC020E030E041
:10E26000A901698D7A8D8B8D9C8D0F940A25882349
:10E2700009F467CF2D893E894F89588DCA01B901AC
:10E280000F9470254B015C01298D3A8D4B8D5C8D6F
:10E29000CA01B9010F9470259B01AC01C501B401FD
:10E2A0000F94DA2B4B015C012D8D3E8D4F8D58A1C3
:10E2B000CA01B9010F9470259B01AC01C501B401DD
:10E2C0000F94DA2B4B015C01A7019601C701B6013F
:10E2D0000F9470259B01AC01C501B4010F94DA2B9A
:10E2E0000F94882E4B015C012DEB37E346E855E394
:10E2F0000F940A2587FF0FC020E030E0A901C70175
:10E30000B6010F943A2E4601570187FF04C0B7FAB1
:10E31000B094B7F8B0942DEB37E346E855E3C50168
:10E32000B4010F940A2587FD1CCF20E030E040EABD
:10E3300051E4C501B4010F94D42C0F944D2D1B0151
:10E34000672B19F422242394312CB10190E080E052
:10E350000F940F259B01AC0160E070E080E89FE323
:10E360000F94D42C2B013C01AC019B01C501B401DD
:10E370000F9470254B015C01A30192016D897E8988
:10E380008F89988D0F9470256D8B7E8B8F8B988FD6
:10E39000A3019201698D7A8D8B8D9C8D0F947025D0
:10E3A000698F7A8F8B8F9C8FA30192016D8D7E8DEB
:10E3B0008F8D98A10F9470256D8F7E8F8F8F98A36E
:10E3C000A3019201C701B6010F94702569A37AA336
:10E3D0008BA39CA380E1E0E2FCE08E010F5F1F4F66
:10E3E000D80101900D928A95E1F70E94E3FC2B0180
:10E3F0003C0128EC420E511C611C711C0DA31EA394
:10E4000081E0281A310809F460C00E94E3FC8B0106
:10E410009C01041915092609370937FD59C02B013C
:10E420003C0128EC420E511C611C711C80E00E94D2
:10E43000175A2D893E894F89588D69817A818B8140
:10E440009C810F94DA2B69837A838B839C83298D3B
:10E450003A8D4B8D5C8D6D817E818F8198850F9477
:10E46000DA2B6D837E838F8398872D8D3E8D4F8D24
:10E4700058A169857A858B859C850F94DA2B6987ED
:10E480007A878B879C8729A13AA14BA15CA16D85D6
:10E490007E858F8598890F94DA2B6D877E878F878D
:10E4A000988B750164018E010F5E1F4F9E01235FE3
:10E4B0003F4FAE01475F5F4FBE016B5F7F4F8DA146
:10E4C0009EA10E9426F481119BCF750164013CCE70
:10E4D0000E9406C2AECF8F929F92AF92BF92CF9210
:10E4E000DF92EF92FF92CF93DF9380904102909062
:10E4F0004202A0904302B0904402FC01C080D1804F
:10E50000E280F38020E030E0A901C701B6010F945A
:10E510000A25882341F0C0924102D0924202E09243
:10E520004302F0924402C0916702D091680284E6EF
:10E5300090E09093680280936702C0906102D0904F
:10E540006202E0906302F090640280E090E0A0E854
:10E55000BFE38093610290936202A0936302B09341
:10E5600064020E94B86F8092410290924202A0928F
:10E570004302B0924402D0936802C0936702C092F3
:10E580006102D0926202E0926302F0926402DF9133
:10E59000CF91FF90EF90DF90CF90BF90AF909F9082
:10E5A0008F9008950F931F93CF93DF9300D01F9206
:10E5B000CDB7DEB79C010CE617E090E1E0E2FCE0AD
:10E5C000D80101900D929A95E1F7F90120813181EE
:10E5D00042815381F80160857185828593850F940E
:10E5E000DA2BF801608771878287938780E090E05B
:10E5F000A0EAB0E489839A83AB83BC83CE01019601
:10E600000E946B720F900F900F900F90DF91CF913F
:10E610001F910F9108952F923F924F925F926F92A8
:10E620007F928F929F92AF92BF92CF92DF92EF92A2
:10E63000FF921F93CF93DF93CDB7DEB72C970FB622
:10E64000F894DEBF0FBECDBF7A011901DC012D9118
:10E650003D914D915C912D833E834F835887FB0103
:10E6600040805180628073808090200C9090210CBB
:10E67000A090220CB090230CA50194016D817E81A5
:10E680008F8198850F940A2581110EC011E0A30196
:10E6900092016091240C7091250C8091260C909130
:10E6A000270C0F940A25811110E0D1012D913D9185
:10E6B0004D915C9129873A874B875C87F701C08031
:10E6C000D180E280F38020910B0230910C024091C6
:10E6D0000D0250910E02C701B6010F940A2588233E
:10E6E00009F44EC0C0920B02D0920C02E0920D02CF
:10E6F000F0920E0280912C0C90912D0CA0912E0C7A
:10E70000B0912F0C4091240C5091250C6091260C57
:10E710007091270C80926C0790926D07A0926E0703
:10E72000B0926F0740937007509371076093720720
:10E7300070937307C0927407D0927507E0927607C2
:10E74000F09277078093780790937907A0937A07E0
:10E75000B0937B0720E030E040E05FE36091620C23
:10E760007091630C8091640C9091650C0F947025EE
:10E7700069837A838B839C83CE0101960E946B729E
:10E780002D813E814F81588520936C0730936D0712
:10E7900040936E0750936F07409270075092710735
:10E7A0006092720770927307D1012D913D914D9146
:10E7B0005C91609178077091790780917A079091C8
:10E7C0007B070F94DA2B6093780770937907809317
:10E7D0007A0790937B0711112FC020E030E0A90148
:10E7E00069857A858B859C850F940A25811133C0B4
:10E7F00060E070E088EC92E469837A838B839C8389
:10E80000CE0101960E946B722C960FB6F894DEBF73
:10E810000FBECDBFDF91CF911F91FF90EF90DF90A2
:10E82000CF90BF90AF909F908F907F906F905F90B0
:10E830004F903F902F9008952AEF3EE74AE25FE322
:10E840006091660C7091670C8091680C9091690CD6
:10E850000F947025D1CF60E070E080EA91E4CCCFD6
:10E860000F931F93CF93DF9300D000D01F921F927E
:10E87000CDB7DEB78B01FC0123A5211102C00E9498
:10E880002EFB1D821E821F82188620E030E040E0B1
:10E890005FE36091280C7091290C80912A0C909173
:10E8A0002B0C0F94DA2B69837A838B839C839E01D4
:10E8B0002B5F3F4FAE014F5F5F4F64E27CE080E231
:10E8C0009CE00E940B731D821E821F82188620E02E
:10E8D00030E040E05FE3F8016085718582859385D3
:10E8E0000F94DA2B69837A838B839C83B8016C5FE6
:10E8F0007F4F9E012B5F3F4FAE014F5F5F4FC801BF
:10E900000E940B7328960FB6F894DEBF0FBECDBFE2
:10E91000DF91CF911F910F9108959B01AC01485F4A
:10E920005F4FBC016C5F7F4F0C940B732F923F9233
:10E930004F925F926F927F928F929F92AF92BF920F
:10E94000CF92DF92EF92FF920F931F93CF93DF93BB
:10E95000CDB7DEB7A6970FB6F894DEBF0FBECDBF1A
:10E960008C011B015A8749874090200C5090210C44
:10E970006090220C7090230C8090240C9090250CB9
:10E98000A090260CB090270CDB018D919D910D90ED
:10E99000BC91A02D8B8B9C8BAD8BBE8B9C01AD0154
:10E9A000C301B2010F94D92B6B017C01D1011496E4
:10E9B0008D919D910D90BC91A02D8F8B988FA98FDB
:10E9C000BA8F9C01AD01C501B4010F94D92B6B8F97
:10E9D0007C8F8D8F9E8FA985BA858D919D910D908D
:10E9E000BC91A02D8B879C87AD87BE879C01AD0114
:10E9F000C301B2010F94D92B6F8F78A389A39AA377
:10EA0000A985BA8514968D919D910D90BC91A02DEC
:10EA10008F87988BA98BBA8B9C01AD01C501B4017E
:10EA20000F94D92B6BA37CA38DA39EA3A701960162
:10EA3000C701B6010F9470256B017C012B8D3C8DB5
:10EA40004D8D5E8DCA01B9010F9470259B01AC01FB
:10EA5000C701B6010F94DA2B4B015C012B893C896D
:10EA60004D895E896B857C858D859E850F94D92B1C
:10EA70002B013C012F89388D498D5A8D6F857889FE
:10EA800089899A890F94D92B6B017C01A30192018A
:10EA9000C301B2010F9470252B013C01A70196011F
:10EAA000C701B6010F9470259B01AC01C301B201EF
:10EAB0000F94DA2B0F94882E6B017C012F8D38A1D7
:10EAC00049A15AA1CA01B9010F9470252B013C013B
:10EAD0002BA13CA14DA15EA1CA01B9010F947025E3
:10EAE0009B01AC01C301B2010F94DA2B9B01AC0175
:10EAF000C501B4010F943A2E1816B4F520E030E0A9
:10EB0000A901C701B6010F943A2E87FF2AC0C70199
:10EB1000B601905820E030E040EA50E40F943A2EDD
:10EB2000181614F5A10169857A85C8010E949674AA
:10EB3000A6960FB6F894DEBF0FBECDBFDF91CF9182
:10EB40001F910F91FF90EF90DF90CF90BF90AF900B
:10EB50009F908F907F906F905F904F903F902F90FD
:10EB60000895C701B601D6CF20E030E040E050E480
:10EB7000C501B4010F943A2E181624F4B101C8014E
:10EB80000E94307419821A821B821C82BE016F5F40
:10EB90007F4FC1010E948D742DEC3CEC4CEC5CE38A
:10EBA000C701B6010F9470259B01AC01F80160818B
:10EBB0007181828193810F9470256D837E838F8311
:10EBC0009887D8019B968C919B978823C9F02AE956
:10EBD00039E949E95FE314966D917D918D919C919E
:10EBE00017970F94702569837A838B839C83BE016A
:10EBF0006F5F7F4F8CE697E00E948D74F80113A63B
:10EC0000BE016B5F7F4F89859A850E948D7490CF7E
:10EC10003F924F925F926F927F928F929F92AF92AC
:10EC2000BF92CF92DF92EF92FF920F931F93CF93F9
:10EC3000DF93CDB7DEB76C970FB6F894DEBF0FBE8B
:10EC4000CDBFDB010C91142F100F153008F067C1F8
:10EC50001196DC90C22ECD0CB4E0BC1508F45FC157
:10EC6000ED2DF0E0EA50FB4F8080912CB12CA12CCF
:10EC7000002E04C0B694A794979487940A94D2F770
:10EC800080FE4DC1EC2DF0E0EA50FB4F8080912CCE
:10EC9000B12CA12C012E04C0B694A794979487940C
:10ECA0000A94D2F780FE3BC1322E642F7C01409043
:10ECB000C6055090C7056090C8057090C905809141
:10ECC000CE059091CF05A091D005B091D105898F47
:10ECD0009A8FAB8FBC8F660F770B072E000C880BBB
:10ECE000990B0F9411254B015C01602F000F770BDE
:10ECF000880B990B0F941125298D3A8D4B8D5C8DC6
:10ED00000F947025A30192010F94DA2BA5019401B1
:10ED10000F94DA2B6D877E878F87988B612F110F69
:10ED2000770B880B990B0F941125298D3A8D4B8DFC
:10ED30005C8D0F947025A30192010F94DA2BA5012D
:10ED400094010F94D92B69837A838B839C834090A1
:10ED5000CA055090CB056090CC057090CD05809190
:10ED6000D2059091D305A091D405B091D505898F96
:10ED70009A8FAB8FBC8F632D660F770B072E000C1D
:10ED8000880B990B0F9411254B015C016D2DDD0C47
:10ED9000770B880B990B0F941125298D3A8D4B8D8C
:10EDA0005C8D0F947025A30192010F94DA2BA501BD
:10EDB00094010F94DA2B698B7A8B8B8B9C8B6C2D47
:10EDC000CC0C770B880B990B0F941125298D3A8D5C
:10EDD0004B8D5C8D0F947025A30192010F94DA2B5B
:10EDE000A50194010F94D92B6D837E838F8398871F
:10EDF000F70180859185A285B38589879A87AB873E
:10EE0000BC878D8B9E8BAF8BB88F45E351E061E063
:10EE100070E0CE0141960E94C4C145E351E061E03B
:10EE200070E0CE0105960E94C4C14AE351E061E062
:10EE300070E0CE010D960E94C4C14AE351E061E04A
:10EE400070E0CE0101960E94C4C189889A88AB887F
:10EE5000BC8827E137EB41ED58EBC501B4010F94B5
:10EE60003A2E87FD5CC023E030E04BE953E4C50156
:10EE7000B4010F940A2518160CF451C08D849E8499
:10EE8000AF84B88827E137EB41ED58EBC501B401F9
:10EE90000F943A2E87FD43C023E030E84DE953E458
:10EEA000C501B4010F940A251816CCF18D809E80FF
:10EEB000AF80B88427E137EB41ED58EBC501B401D1
:10EEC0000F943A2E87FD2BC023E030E04BE953E44A
:10EED000C501B4010F940A2518160CF189809A8097
:10EEE000AB80BC8027E137EB41ED58EBC501B401A5
:10EEF0000F943A2E87FD13C023E030E84DE953E428
:10EF0000C501B4010F940A2518164CF0AE014F5FED
:10EF10005F4FBE01635F7F4FC7010E9496746C967E
:10EF20000FB6F894DEBF0FBECDBFDF91CF911F911A
:10EF30000F91FF90EF90DF90CF90BF90AF909F9098
:10EF40008F907F906F905F904F903F9008952F9299
:10EF50003F924F925F926F927F928F929F92AF9269
:10EF6000BF92CF92DF92EF92FF920F931F93CF93B6
:10EF7000DF93CDB7DEB7CC58D1090FB6F894DEBF1A
:10EF80000FBECDBF80E19CE00E943C3887E00E942C
:10EF90001F4E81116EC084E50E948C1E882329F0CB
:10EFA0000E947F2481110E9434BA80E090E0A0E8A2
:10EFB000BFE389839A83AB83BC838D839E83AF83B6
:10EFC000B8878DEC9CECACE4BEE389879A87AB876D
:10EFD000BC8780E090E0A0E2B1E48D879E87AF8798
:10EFE000B88B8CE390E09A8B898B8DEC90E09C8BB6
:10EFF0008B8B8DEC9CECACECBEE38D8B9E8BAF8B46
:10F00000B88F80E090E0A0EEBFE3898F9A8FAB8F3E
:10F01000BC8F1BA61CA64AE959E969E97EE38FE487
:10F020000E94BC246D8F7E8F8F8F98A360E083E455
:10F030000E946A2489A360E08BE40E946A248AA368
:10F0400082E40E948C1E882381F10E947F24009715
:10F0500061F19C01285231092536310520F16CE817
:10F0600070E082EE9BE00E943A418DED9BE00E94B1
:10F070003C38C457DF4F0FB6F894DEBF0FBECDBF8C
:10F08000DF91CF911F910F91FF90EF90DF90CF9084
:10F09000BF90AF909F908F907F906F905F904F90B8
:10F0A0003F902F9008959A8B898B8CE40E948C1E40
:10F0B0008823E1F00E9492246B017C01C986DA86E4
:10F0C000EB86FC8620E030E0A9010F943A2E87FD04
:10F0D0000AC020E030E040E050E4C701B6010F94E0
:10F0E0000A2518161CF485EB9BE0C1CF81E50E9430
:10F0F0003E1E882331F18091FF0490910005892BF9
:10F10000E9F00E9492246B017C01CD82DE82EF82C5
:10F11000F8862DEC3CEC4CE45DE30F943A2E87FD31
:10F120000AC020E030E040E751E4C701B6010F9487
:10F130000A25181634F484E89BE099CF89E59BE012
:10F1400096CF83E50E948C1E8823E9F00E949224CA
:10F150006B017C01CD8ADE8AEF8AF88E2DEC3CECC7
:10F160004CEC5DE30F943A2E87FD0AC020E030E0BE
:10F1700040E050E4C701B6010F940A2518161CF4AC
:10F1800082E39BE074CF80E50E943E1E882341F11C
:10F190008091FF0490910005892B19F48AEF9AE081
:10F1A00066CF8BA58F5F8BA70E9492246B017C0199
:10F1B000CD86DE86EF86F88A20E030E0A9010F9444
:10F1C0003A2E87FD0AC020E030E048EC51E4C70148
:10F1D000B6010F940A2518161CF482ED9AE047CF69
:10F1E00086E40E948C1E8823E9F00E9492246B0121
:10F1F0007C01C98EDA8EEB8EFC8E20E030E040E898
:10F200005FE30F943A2E87FD0AC020E030E040E82B
:10F2100050E4C701B6010F940A2518161CF489EAB8
:10F220009AE025CFC98CDA8CEB8CFC8C8D889E887B
:10F23000AF88B88CA7019601C701B6010F9470255D
:10F240009B01AC0160E070E084E490E40F94D42C66
:10F2500029813A814B815C810F9470252B013C01FF
:10F26000A5019401C501B4010F947025A701960171
:10F270000F9470252CEE31E548EB5DE30F94D42C10
:10F280009B01AC01C301B2010F94702569837A839D
:10F290008B839C8388E40E948C1E882379F00E94D3
:10F2A0007F24009759F09C01255A310928383105EF
:10F2B00018F08BE79AE0DBCE9C8B8B8B85E50E9468
:10F2C0003E1E8823C9F00E94E3FC6115710581058B
:10F2D000910511F00F9490208091FF04909100050A
:10F2E000892B91F00E9492246093FB047093FC049C
:10F2F0008093FD049093FE0482E50E943E1E8111DE
:10F3000008C087E49AE0B3CE60E070E088E492E45D
:10F31000EBCF8091FF0490910005892B61F00E9452
:10F320007F24AD969FAF8EAFAD97181619064CF09F
:10F3300083E19AE09CCE2AE130E0AD963FAF2EAF5C
:10F34000AD9789E50E948C1E882381F10E9492244A
:10F350002091CC083091CD084091CE085091CF0833
:10F360000F94D92B6B017C0188E50E948C1E8823A9
:10F3700031F10E9492242091C8083091C90840912F
:10F38000CA085091CB080F94D92B6BA37CA38DA3F3
:10F390009EA3CFA2D8A6E9A6FAA6CE0183960E9484
:10F3A000FD1D811115C089EE99E061CEC090240C3D
:10F3B000D090250CE090260CF090270CD5CF6091D2
:10F3C000200C7091210C8091220C9091230CDDCFA8
:10F3D00084E40E943E1E91E089270E94146980E027
:10F3E00090E0A0EAB0E48DA79EA7AFA7B8AB60E01D
:10F3F000CE018D960E94CE643091F107CD57DF4F3C
:10F400003883C358D0401092F1070E94F71B88EC54
:10F4100099E00E943C3889899A898A3191050CF0DB
:10F4200044C08B899C890E94141F61E080E00E9487
:10F43000D4BC811142C06FEF8DED99E00E94AA3FCC
:10F440008CA5811104C0CE0101960E942EFB80E0A4
:10F4500090E0A0EAB0E48093740790937507A093BE
:10F460007607B09377071DA61EA61FA618AABE0191
:10F47000635D7F4F8CE697E00E948D74CD57DF4F20
:10F480005881C358D0405093F1070E94F71B8AA1BE
:10F490008111EFCD10927B1110927A110E948CBED7
:10F4A00090E080E00E94141FE4CD0E94522281E08F
:10F4B0000E945DBB8111B5CFBECF10922C0C109273
:10F4C0002D0C10922E0C10922F0C8CE29CE00E94BE
:10F4D0008C618BA5882309F452C020E030E040E71E
:10F4E00051E46091660C7091670C8091680C90916A
:10F4F000690C0F94D42C6DA77EA78FA798AB80E1E1
:10F50000E0E2FCE0ACE6B7E001900D928A95E1F70D
:10F510002D853E854F8558896091780770917907D0
:10F5200080917A0790917B070F94DA2B609378078C
:10F530007093790780937A0790937B07CE018D961D
:10F540000E946B722D853E854F85588960917807A2
:10F550007091790780917A0790917B070F94D92B4E
:10F56000609378077093790780937A0790937B076D
:10F570008CA5811104C0CE0101960E942EFBE6EFFE
:10F58000F4E085E0DF011D928A95E9F780E1E0E291
:10F59000FCE0ACE6B7E001900D928A95E1F7898531
:10F5A0009A85AB85BC858093740790937507A0936B
:10F5B0007607B09377071DA61EA61FA618AABE0140
:10F5C000635D7F4F8CE697E00E948D74BE01635EA1
:10F5D0007F4F8CE697E00E948D7489A1882309F4FF
:10F5E0001CC42091200C3091210C4091220C509190
:10F5F000230CE5962CAF3DAF4EAF5FAFE597809102
:10F60000240C9091250CA091260CB091270CE1962A
:10F610008CAF9DAFAEAFBFAFE197312C212C9FEFE8
:10F62000A4969FAFA497AFEFA896AFAFA897BFEFF0
:10F63000C158DF4FB883CF57D040EFE4C058DF4FF9
:10F64000E883C058D040F3ECCF57DF4FF883C15860
:10F65000D04027E4CE57DF4F2883C258D04081E006
:10F6600090E0A0E0B0E0022C04C0880F991FAA1F10
:10F67000BB1F0A94D2F7CC57DF4F88839983AA83A4
:10F68000BB83C458D040A6EFB4E0E796BFAFAEAF9F
:10F69000E79710E000E09101032C000C440B550BA0
:10F6A000C857DF4F288339834A835B83C858D040CB
:10F6B000C457DF4F2882CC58D040E796AEADBFADDF
:10F6C000E7978D91E796BFAFAEAFE79790E0B0E0D8
:10F6D000A0E0CC57DF4F288139814A815B81C45833
:10F6E000D04082239323A423B523892B8A2B8B2BF1
:10F6F00009F024C1C857DF4F688179818A819B81D5
:10F70000C858D0400F9411252091CE053091CF05D7
:10F710004091D0055091D1050F9470252091C605D8
:10F720003091C7054091C8055091C9050F94DA2B57
:10F73000EB966CAF7DAF8EAF9FAFEB97B801012E0C
:10F74000000C880B990B0F9411252091D205309154
:10F75000D3054091D4055091D5050F947025209183
:10F76000CA053091CB054091CC055091CD050F9441
:10F77000DA2B6B017C01EB962CAD3DAD4EAD5FAD50
:10F78000EB97E5966CAD7DAD8EAD9FADE5970F9493
:10F79000D92B2B013C01A7019601E1966CAD7DAD03
:10F7A0008EAD9FADE1970F94D92B4B015C01A30166
:10F7B0009201C301B2010F9470252B013C01A501F8
:10F7C0009401C501B4010F9470259B01AC01C301E4
:10F7D000B2010F94DA2B0F94882E4B015C01EB964B
:10F7E0002CAD3DAD4EAD5FADEB976BA17CA18DA176
:10F7F0009EA10F94D92B2B013C01A70196016FA16B
:10F8000078A589A59AA50F94D92B6B017C01A3013A
:10F810009201C301B2010F9470252B013C01A70195
:10F820009601C701B6010F9470259B01AC01C3017D
:10F83000B2010F94DA2B0F94882E20E030E040E7DD
:10F8400051E40F94D42CA50194010F94DA2B6B0191
:10F850007C018090FB049090FC04A090FD04B0908B
:10F86000FE0420E030E040E85FE3C501B4010F94FE
:10F870003A2E1816F4F4C501B4010F94462D4B012D
:10F880005C0160E070E0CB01181419041A041B0439
:10F8900034F40F944120A50194010F94702B0F9420
:10F8A00011259B01AC01B601C7010F94DA2B6B0146
:10F8B0007C01C158DF4F2881CF57D040C058DF4F5F
:10F8C0003881C058D040CF57DF4F4881C158D04011
:10F8D000CE57DF4F5881C258D040B601C7010F94B0
:10F8E0000A2587FF2BC0A4960FAFA497C457DF4FFC
:10F8F0003881CC58D040A8963FAFA897EC96CFAEB1
:10F90000EC97ED96DFAEED97EE96EFAEEE97EF96B5
:10F91000FFAEEF97C158DF4FC882CF57D040C058D5
:10F92000DF4FD882C058D040CF57DF4FE882C15850
:10F93000D040CE57DF4FF882C258D0400F5F1F4FE4
:10F940000530110509F0B9CE4FEF241A340A55E0FD
:10F950002516310409F083CEA4968FADA497E82F25
:10F96000F0E0EA50FB4F208181E090E0A0E0B0E0C1
:10F97000A8960FACA89704C0880F991FAA1FBB1F99
:10F980000A94D2F7822B8083A8969FADA8976A9697
:10F990009FAF6A97A496AFADA4976B96AFAF6B97E6
:10F9A000EC968FADEC97ED969FADED97EE96AFADE3
:10F9B000EE97EF96BFADEF976F968CAF9DAFAEAF62
:10F9C000BFAF6F97A896BFADA897BF3F09F409C214
:10F9D000A496EFADA497EF3F09F403C26B2FBB0FC2
:10F9E000770B880B990B0F9411252091CE05309140
:10F9F000CF054091D0055091D1050F9470252091ED
:10FA0000C6053091C7054091C8055091C9050F94AE
:10FA1000DA2B162F072F382E292E862F902FA32D65
:10FA2000B22D65968CAF9DAFAEAFBFAF6597A49674
:10FA3000FFADA4976F2FFF0F770B880B990B0F94D7
:10FA400011252091D2053091D3054091D4055091D4
:10FA5000D5050F9470252091CA053091CB054091B2
:10FA6000CC055091CD050F94DA2B6B017C01699682
:10FA7000CCAEDDAEEEAEFFAE6997CE018F5A9F4F92
:10FA80000E94FD1D882309F4B0C120E030E040EA67
:10FA900050E4612F702F832D922D0F94DA2B4B01A0
:10FAA0005C01CB01D50121968CAF9DAFAEAFBFAF4E
:10FAB00021972596CCAEDDAEEEAEFFAE2597A8968B
:10FAC0002FADA8972111E3C1A4963FADA4973111A2
:10FAD000B3C120E030E040EA50E4C701B6010F9422
:10FAE000DA2B6B017C01A4964FADA497442309F453
:10FAF000C5C1A4968FADA49784300CF0BFC122ED90
:10FB0000422E23E5522E2BE7622E21E4722E2196FF
:10FB10008CAC9DACAEACBFAC219725968CAD9DADA9
:10FB2000AEADBFAD2597A7968CAF9DAFAEAFBFAFC3
:10FB3000A7979C01AD0169966CAD7DAD8EAD9FAD73
:10FB400069970F94D92BAB966CAF7DAF8EAF9FAFFB
:10FB5000AB97A501940165966CAD7DAD8EAD9FAD63
:10FB600065970F94D92B2D966CAF7DAF8EAF9FAF5D
:10FB70002D97AB962CAD3DAD4EAD5FADAB9761967D
:10FB80002CAF3DAF4EAF5FAF6197A501940160917F
:10FB9000200C7091210C8091220C9091230C0F94D9
:10FBA000D92B4B015C01A7962CAD3DAD4EAD5FADA1
:10FBB000A7976091240C7091250C8091260C909150
:10FBC000270C0F94D92BA7966CAF7DAF8EAF9FAF4C
:10FBD000A797812F902FA32DB22D8DA79EA7AFA7FA
:10FBE000B8ABC9AADAAAEBAAFCAAC984DA84EB8466
:10FBF000FC84CDAADEAAEFAAF8AE2DEC3CEC4CECCE
:10FC00005CE3C301B2010F94702529813A814B81D5
:10FC10005C810F94702520912C0C30912D0C40911B
:10FC20002E0C50912F0C0F94DA2B69AF7AAF8BAF5B
:10FC30009CAFA5019401C501B4010F9470254B013F
:10FC40005C01A7962CAD3DAD4EAD5FADA797CA0147
:10FC5000B9010F9470259B01AC01C501B4010F944B
:10FC6000DA2B20E030E040E050E40F943A2E1816F2
:10FC7000ACF420E030E040E05FE3C701B6010F9450
:10FC8000DA2B29966CAF7DAF8EAF9FAF2997BE015F
:10FC9000635C7F4FCE0101960E94307489859A85FE
:10FCA000AB85BC8529968CAF9DAFAEAFBFAF299712
:10FCB000A3961CAE1DAE1EAE1FAEA397BE01615A29
:10FCC0007F4FCE01CD960E948D748CA58823C1F004
:10FCD0002AE939E949E95FE36D817E818F81988561
:10FCE0000F947025A3966CAF7DAF8EAF9FAFA39797
:10FCF000BE01615A7F4F8CE697E00E948D741CA66E
:10FD0000E0905E0CF0905F0C0091600C1091610C23
:10FD1000A0905A0CB0905B0CC0905C0CD0905D0C25
:10FD20009501A601B701C8010F943A2E181614F4D4
:10FD3000750186018090410290904202A09043029A
:10FD4000B09044022DEC3CEC4CEC5DE3B701C801F3
:10FD50000F94702560934102709342028093430296
:10FD60009093440240E0BE01675B7F4FCE018D96C9
:10FD70000F94421480E1E0E2FCE0ACE6B7E00190D1
:10FD80000D928A95E1F78092410290924202A092F0
:10FD90004302B092440220E04FEFBE01675A7F4F0A
:10FDA000CE0101960E94087620E041E0BE01675A2C
:10FDB0007F4FCE0101960E9408762FEF40E0BE01F2
:10FDC000675A7F4FCE0101960E94087621E040E0FD
:10FDD000BE01675A7F4FCE0101960E9408760E94AD
:10FDE0007B6180919C0C80939D0CAD964EAD5FAD78
:10FDF000AD9741505109AD965FAF4EAFAD97452BD2
:10FE000009F419CB6A968FAD6A9787FD14CB6B9670
:10FE10008FAD6B9787FFE1CB0ECB2BA13CA14DA102
:10FE20005EA1E5962CAF3DAF4EAF5FAFE5978FA1DA
:10FE300098A5A9A5BAA5EBCB812F902FA32DB22D04
:10FE400021968CAF9DAFAEAFBFAF219720E030E0E1
:10FE500040EA50E4C701B6010F94D92B25966CAF48
:10FE60007DAF8EAF9FAF2597A4965FADA49754301A
:10FE70000CF42FCE182D092D3A2C2B2C92ED492E57
:10FE800093E5592E9BEF692E90E4792E40CEA896EB
:10FE90009FADA89794300CF452C0A496AFADA49730
:10FEA000A4300CF120E030E040EA50E4612F702FE4
:10FEB000832D922D0F94D92B21966CAF7DAF8EAFF1
:10FEC0009FAF219720E030E040EA50E4C701B6013F
:10FED0000F94D92B6B017C01A496EFADA497E4306D
:10FEE0000CF40DCECBCF812F902FA32DB22D2196C8
:10FEF0008CAF9DAFAEAFBFAF219720E030E040EABE
:10FF000050E4C701B6010F94DA2B25966CAF7DAF94
:10FF10008EAF9FAF2597A496BFADA497B111D2CF56
:10FF200020E030E040EA50E4612F702F832D922DC5
:10FF30000F94D92B162F072F382E292E9FCFA4963A
:10FF4000FFADA497F1110DC020E030E040E251E494
:10FF5000B401C5010F94D92B162F072F382E292E47
:10FF6000CECDA4962FADA49724309CF020E030E0B5
:10FF700040E251E4B401C5010F94D92B21966CAF36
:10FF80007DAF8EAF9FAF2197182D092D3A2C2B2CCA
:10FF9000B6CD182D092D3A2C2B2C82ED482E83E559
:10FFA000582E8BEF682E81E4782EB1CD2F923F92A0
:10FFB0004F925F926F927F928F929F92AF92BF9279
:10FFC000CF92DF92EF92FF920F931F93CF93DF9325
:10FFD000CDB7DEB7EE970FB6F894DEBF0FBECDBF3C
:10FFE0008091310C888B87E50E943E1E882309F49E
:10FFF00023C120E030E0A9016091CE057091CF05CA
:020000021000EC
:100000008091D0059091D1050F940A25811108C0E7
:100010000E940B4E8DE09DE00E943C3810E01FC115
:100020008AE50E948C1E882339F10E949224209137
:10003000D0083091D1084091D2085091D3080F9444
:10004000D92B6B017C0120E030E040E251ECC7018C
:10005000B6010F943A2E87FD0AC020E030E040E25E
:1000600051E4C701B6010F940A25181674F40E94D2
:100070000B4E80E09DE0D0CFC090280CD090290C92
:10008000E0902A0CF0902B0CDECF40E050E060ECCA
:100090007FE788E50E94BC242091C8083091C908F8
:1000A0004091CA085091CB080F94D92B2B013C01E9
:1000B00040E050E060EC7FE789E50E94BC2420919D
:1000C000CC083091CD084091CE085091CF080F94C4
:1000D000D92B4B015C016FEF89E40E944E24182F4D
:1000E0006FEF8AE40E944E24082FA3019201C301FE
:1000F000B2010F94CC2E81116EC0A5019401C501EF
:10010000B4010F94CC2E811166C08BA19CA1ADA12E
:10011000BEA18BAB9CABADABBEAB2091C605309105
:10012000C7054091C8055091C905C301B2010F949C
:10013000D92B2B013C0120E030E040E05FE36BA9CC
:100140007CA98DA99EA90F9470259B01AC01C301C8
:10015000B2010F94DA2B2BA93CA94DA95EA90F94EB
:10016000D42C0F94462D162F4FA058A469A47AA41E
:100170002091CA053091CB054091CC055091CD0519
:10018000C501B4010F94D92B4B015C0120E030E094
:1001900040E05FE3C301B2010F9470259B01AC0105
:1001A000C501B4010F94DA2BA30192010F94D42C52
:1001B0000F94462D062F812F012E000C990B97FDD1
:1001C00033C005979CF5802F002E000C990B97FDEE
:1001D0002FC005977CF5153008F020CF053008F0CA
:1001E0001DCF80E00E94146995E01902F0011124EE
:1001F000E00FF11D07FDFA95EE0FFF1FEE0FFF1F39
:10020000E857F84FC082D182E282F382602F812FBB
:100210000E94A5F788890E9414698889882309F4B7
:10022000FDCE0E949130FACE10E0CDCF14E0CBCFBE
:1002300000E0D1CF04E0CFCF8AE40E943E1E182F09
:10024000811127C070E060E086E50E9483249A83D4
:100250008983059708F18BED9CE00E943C38812F43
:10026000EE960FB6F894DEBF0FBECDBFDF91CF91F3
:100270001F910F91FF90EF90DF90CF90BF90AF90C4
:100280009F908F907F906F905F904F903F902F90B6
:1002900008950E94F26EC2CE60E084E40E946A2457
:1002A0008F8740E050E0BA018AE50E94BC246BA72A
:1002B0007CA78DA79EA740E050E86BE376E483E53A
:1002C0000E94BC2420E030E040E752E40F94D42C9C
:1002D00060933D0270933E0280933F0290934002F0
:1002E000E0907C12F0907D12D7018D909D90AD90A2
:1002F000BC9020E030E0A901C501B4010F94DA2BD5
:100300006BAF7CAF8DAF9EAF20E030E040E450E4B7
:100310000F940A2587FF06C01BAE1CAEB0E4BDAF2C
:10032000E0E4EEAF20E030E84DE953E4C501B4016C
:100330000F94DA2B662E7BAB8FAB98AF20E030E8C2
:1003400044E953E40F943A2E18163CF4612CF0E87B
:10035000FBAB24E92FAB33E438AFD70114968D9073
:100360009D90AD90BC90179720E030E0A901C501A9
:10037000B4010F94DA2BD62EE72EF82E092F20E0A9
:1003800030E040E551E40F940A2587FF05C0D12CE9
:10039000E12CA0E5FA2E01E420E030E04BE953E443
:1003A000C501B4010F94DA2BB62EC72E89AF9AAFD0
:1003B00020E030E84FE853E40F943A2E18163CF44E
:1003C000B12CF0E8CF2EBFE8B9AFE3E4EAAF88E4A0
:1003D0000E943E1E882309F416C20E9492240F94A4
:1003E000462D1B0177FF02C06F5F7F4F75956795A4
:1003F0007195619571096A567F4F072E000C880B25
:10040000990B0F941125762E872E982EA92E2D2D1F
:100410003E2D4F2D502F0F943A2E18161CF4D72C2A
:1004200074010A2D2BAD3CAD4DAD5EAD672D782D21
:10043000892D9A2D0F943A2E181624F07BAC8CAC93
:100440009DACAEAC872D982DA92DBA2D8B8B9C8B96
:10045000AD8BBE8B8D2D9E2DAF2DB02F8F8B988F9A
:10046000A98FBA8FB101330C880B990B0F9411250A
:100470001B012C01AC019B016D2D7E2D8F2D902F2A
:100480000F94DA2BD62EE72EF82E092F2B2D3C2D8C
:1004900049AD5AAD0F940A2587FF04C0BD2CCE2C60
:1004A000F9AE0AAFA2019101672D782D892D9A2D01
:1004B0000F94DA2BD62EE72EF82E092F262D3BA9E6
:1004C0004FA958AD0F940A2587FF04C06D2CEBAAE5
:1004D000FFAA08AF862D9BA9AFA9B8AD8B8F9C8FC3
:1004E000AD8FBE8F8B2D9C2DA9ADBAAD8F8F98A3EC
:1004F000A9A3BAA3BE01695E7F4FCE0143960E94B5
:10050000302E882309F4B0C1BE01615E7F4FCE0159
:100510004B960E94302EE82E882309F4A5C12F891E
:10052000388D498D5A8D6F8D78A189A19AA10F942C
:10053000D92B20E030E040E85EE30F9470254B01BA
:100540005C012B893C894D895E896B8D7C8D8D8DFD
:100550009E8D0F94D92B20E030E040E85EE30F94AD
:1005600070256BA37CA38DA39EA38FA298A6A9A69A
:10057000BAA689819A811816190674F489EA9CE052
:100580000E943C388F85882321F08FE99CE00E94EF
:100590003C388AE00E9403380E947B610E94D31C91
:1005A00080E00E94146980E090E0A0E2B1E48FA7AF
:1005B00098ABA9ABBAAB60E0CE018F960E94CE6437
:1005C0002091CE053091CF054091D0055091D105B5
:1005D0006BA17CA18DA19EA10F940A25811130C031
:1005E0002091D2053091D3054091D4055091D50585
:1005F0006FA178A589A59AA50F940A25811120C01D
:100600002091C6053091C7054091C8055091C90594
:100610006B897C898D899E890F940A25811110C070
:100620002091CA053091CB054091CC055091CD0564
:100630006F89788D898D9A8D0F940A258823A9F06A
:100640000E94F26E88E0FE01B396AEECB5E0019038
:100650000D928A95E1F788E0FE017396A6ECB5E06D
:1006600001900D928A95E1F7188A60E085E40E9476
:100670006A24882309F4FBC0F1E0FBAB1B861C86CF
:100680001D861E861A8A9E2C4FE6C42E4CE0D42E60
:100690005DE7A52E5CE0B52E1A8915300CF0F7C089
:1006A0006B857C858D859E859B01AC010F94CC2E3E
:1006B0008111EDC0992009F4DDC031E03FAB35E098
:1006C000232E91E09926F12EFF0CFF0CF10EF394EE
:1006D000898B19896A89121509F4D5C0062E000C78
:1006E000770B880B990B0F9411252FA138A549A5DD
:1006F0005AA50F9470252F89388D498D5A8D0F94E6
:10070000DA2B2B013C01612F110F770B880B990B12
:100710000F9411252BA13CA14DA15EA10F94702532
:100720002B893C894D895E890F94DA2B6B837C83FE
:100730008D839E834F82588669867A8689819A81C5
:10074000892B79F06F2D8BE89CE00E94104169E1C4
:1007500070E089E89CE00E943A4186E89CE00E94B3
:100760003C381F9299E19F931F92FF92DF92CF92A4
:10077000BF92AF921F920E94D0F829814BA9BE016F
:10078000695F7F4FCE0103960E9441F92B013C0126
:100790004B865C866D867E860FB6F894DEBF0FBEF4
:1007A000CDBFAC019B010F94CC2E811169C089880B
:1007B0003A8825E0382D320380011124030D111DE4
:1007C00037FC1A95000F111F000F111F0857184F03
:1007D000A30192016BA57CA58DA59EA50F94DA2B94
:1007E000D8016D937D938D939C931397632D882DE2
:1007F0000E94A5F7188A81E00E94175AF39489890C
:10080000BFA98B0F65CF4D2D5E2D6F2D702F86E408
:100810000E94BC241B012C014BAD5CAD6DAD7EADC7
:100820008CE40E94BC246B8B7C8B8D8B9E8B2F8ADF
:10083000388E498E5A8E4B2D5C2D69AD7AAD82E48F
:100840000E94BC246B017C01462D5BA96FA978AD89
:1008500082E50E94BC246B8F7C8F8D8F9E8FCF8E04
:10086000D8A2E9A2FAA246CE8FEB9CE0F6CC22E019
:100870002BAB04CF8FEF8FAB22242A9484E021CFBF
:1008800088890E9414698A898F5F8A8B05CF0E94AC
:100890003BE40E94A465882359F088890E9414696A
:1008A00080E090E0A0ECBFE78B879C87AD87BE8798
:1008B0006B857C858D859E859B01AC010F94CC2E2C
:1008C000811159C08F85811126C082E0F82E02E087
:1008D00094E0C92E12E0DC2CD11A21E041E0612F16
:1008E000802F0E946B2221E04FEF612F8F2D0E94FD
:1008F0006B222FEF41E06D2D802F0E946B222FEF96
:100900004FEF6D2D8F2D0E946B22115020F701505B
:10091000F3940F3FF9F60E9481400E94991E8F8543
:10092000811124C088E29CE00E94831D4B015C0180
:1009300080E29CE00E94291F9B01AC01C501B4012B
:100940000F9470259B01AC016091280C7091290CCB
:1009500080912A0C90912B0C0F94D92B6093280C2A
:100960007093290C80932A0C90932B0C8F85811106
:10097000E888E092310C0E94BA1C8091310C811100
:100980000E94F62A0E948E670E9491306B857C85BA
:100990008D859E8511E09B01AC010F94CC2E8111B9
:1009A0005ECC3CCB8F929F92AF92BF92CF92DF9260
:1009B000EF92FF920F931F93CF93DF9300D01F927C
:1009C000CDB7DEB75C016B017A01122F0023E1F194
:1009D0000E940F4E88E999E00E943C3861E0812F27
:1009E0000E94303A9090100583E08093100581E0DA
:1009F00080931F0C0E94274082E08093891140E37E
:100A000068E879E084E799E00E942C4040E069E1E1
:100A100071E18DE699E00E942C4061E088E699E062
:100A20000E940E408AE799E00E94272280911F0CC5
:100A3000882341F060E0812F0E94303A81E00E94DB
:100A4000175AF4CF9092100520E030E0A901F5018B
:100A500060817181828193810F940A25882371F0CE
:100A600080E090E0A0ECB0E489839A83AB83BC8300
:100A7000BE016F5F7F4FC5010E94546820E030E0E7
:100A8000A901F60160817181828193810F940A2509
:100A9000882351F180906E0C90906F0CA090700C98
:100AA000B090710C80E090E0A0E7B1E480936E0C10
:100AB00090936F0CA093700CB093710C80E090E059
:100AC000A0EAB1E489839A83AB83BC83BE016F5FE4
:100AD0007F4FC6010E94546880926E0C90926F0CFA
:100AE000A092700CB092710C20E030E0A901F701E7
:100AF00060817181828193810F943A2E181674F46B
:100B000080E090E0A0E4B0E489839A83AB83BC8367
:100B1000BE016F5F7F4FC7010E9454688091E5045A
:100B200029E131E1882311F029E439E047E559E072
:100B300061E679E081E00E944F400E94274081E019
:100B40000F900F900F900F90DF91CF911F910F9109
:100B5000FF90EF90DF90CF90BF90AF909F908F90DD
:100B60000895CF93C82F8091DE0B83FD14C0809130
:100B7000FB08811110C080915F02909160029C017E
:100B8000215031094091E5115091E6114217530768
:100B900014F40E94141FCC2329F061E080E0CF916F
:100BA0000C94D4BC8091FB0891E0892780933C028F
:100BB00080913C02882389F08091E3119091E411A7
:100BC0002091E5113091E611821B930B97FF03C032
:100BD000919581959109029744F410923C0280917D
:100BE000DE0B83FF06C0C1E01AC080E00E94175AE6
:100BF000DFCFC091FB08C11112C080915F029091BC
:100C0000600201972091E5113091E611281739070C
:100C100054F70E940F4E8BE299E00E943C388C2FD3
:100C2000CF910895AF92BF92CF92DF92EF92FF9251
:100C30000F931F93CF93DF93CDB7DEB764970FB6B3
:100C4000F894DEBF0FBECDBF0E940E4F87FDAFC030
:100C50008AE50E948C1E882309F4BAC040E050E067
:100C6000BA018AE50E94BC247B018C012091280CEA
:100C70003091290C40912A0C50912B0C60E070E0CF
:100C800088EC93E40F94D92B5B016C019701A801C8
:100C90000F943A2E181614F07501860120E030E00A
:100CA000A901B701C8010F943A2E181624F4E12CBB
:100CB000F12C00E010E0B701C8010F94462D072E7B
:100CC000000C880B990B0F941125698B7A8B8B8BF9
:100CD0009C8B20E030E0A9010F940A25882321F0A5
:100CE000CE0141960E94D27280E090E0A0EAB1E489
:100CF0008D879E87AF87B88B19861A861B861C86C0
:100D00008CE40E943E1E882309F467C00E9492244E
:100D10006B017C0120E030E0A901C701B6010F940E
:100D20003A2E87FF04C0F7FAF094F7F8F094CD82DA
:100D3000DE82EF82F8862091E5113091E6112430B1
:100D4000310574F08091E3119091E411821B930BB3
:100D500097FF03C091958195910901E004970CF4E8
:100D600000E080E00E94B185882359F022E0AE01C6
:100D7000435F5F4FBE016B5F7F4FCE0109960E94BC
:100D8000D28469897A898B899C898B019C0130582E
:100D900009831A832B833C8320E030E0A9010F9460
:100DA0000A25882321F0CE0101960E94D272649612
:100DB0000FB6F894DEBF0FBECDBFDF91CF911F916C
:100DC0000F91FF90EF90DF90CF90BF90AF9008957C
:100DD000E12CF12C00E211E449CFC090C105D09084
:100DE000C205E090C305F090C40594CF7F928F9226
:100DF0009F92AF92BF92CF92DF92EF92FF920F93AA
:100E00001F93CF93DF9300D000D01F921F92CDB7D6
:100E1000DEB76C015B014A01722E780100910E066B
:100E20000E94201F8091E5119091E6118E159F057B
:100E30001CF4C7010E94141F80E00E94B185882322
:100E400031F0272DA401B501C6010E94D2841E14E1
:100E50001F043CF4C7010E94141F60E080E00E9460
:100E6000D4BC81E00E94B18580E090E0A0E7B2E4CC
:100E700089839A83AB83BC8380E090E0A0E8B0ECE8
:100E80008D839E83AF83B887BE016F5F7F4FCE0196
:100E900005960E94546887E00E940D2A811158C06F
:100EA0008091280C9091290CA0912A0CB0912B0CC8
:100EB0004091EA045091EB046091EC047091ED04D0
:100EC000C090E604D090E704E090E804F090E904D4
:100ED000C0926C07D0926D07E0926E07F0926F0798
:100EE0004093700750937107609372077093730774
:100EF0008093740790937507A0937607B093770754
:100F000080E090E0A8E4B2E489839A83AB83BC8359
:100F1000CE0101960E946B728091EE049091EF04D5
:100F2000A091F004B091F104809374079093750739
:100F3000A0937607B093770780E090E0A0EAB0E452
:100F400089839A83AB83BC83CE0101960E946B7226
:100F5000C12CD12C80E7E82E82E4F82EC982DA82F7
:100F6000EB82FC8280E090E0A0E8B0E48D839E8379
:100F7000AF83B887BE016F5F7F4FCE0105960E9499
:100F8000546820E030E0A9016091F2047091F3040C
:100F90008091F4049091F5040F940A2587FF0BC00B
:100FA000C982DA82EB82FC82BE016F5F7F4F82EFE3
:100FB00094E00E9454688091F2049091F304A0910F
:100FC000F404B091F50480932C0C90932D0CA09315
:100FD0002E0CB0932F0C8093780790937907A093F1
:100FE0007A07B0937B0788E797E00E948C61809135
:100FF000C50581110E94EBF661E087EB99E00E9444
:10100000773F80911B11815080931B114CE658E172
:101010006FEB79E085E00E94C0E280911B1188238C
:1010200039F00E940DAB80911B11815080931B11F0
:1010300080E00E94B2F80E948B3180911C118230B6
:1010400011F40E944A380E943BE428960FB6F894A7
:10105000DEBF0FBECDBFDF91CF911F910F91FF90EB
:10106000EF90DF90CF90BF90AF909F908F907F9048
:101070000895CF92DF92EF92FF920F931F93CF9339
:10108000DF9300D01F92CDB7DEB77C016B018A01E0
:1010900061E08CE399E00E94773F4CE658E163E41D
:1010A00079E085E00E94C0E290911B1181E0890FF8
:1010B00080931B118091291482FF06C08B7F80933F
:1010C00029149E5F90931B110E943C3980E1E0E25D
:1010D000FCE0A6EEB4E001900D928A95E1F70E9443
:1010E0007B6181E00E94B2F820E030E0A901F701C5
:1010F00060817181828193810F940A258823F1F0A8
:101100008091FB0881110CC080915F029091600278
:1011100001972091E3113091E4112817390774F0F9
:1011200080E090E0A0E7B2E489839A83AB83BC833C
:10113000BE016F5F7F4FC7010E94546887E00E9425
:101140000D2A811103C0B6010E94A86720E030E09B
:10115000A901F80160817181828193810F940A2530
:10116000882341F080E00E94B185882319F0C801EE
:101170000E948468129A64E670E080E090E00E9429
:10118000002681E00F900F900F900F90DF91CF918C
:101190001F910F91FF90EF90DF90CF900895CF9225
:1011A000DF92EF92FF92CF93DF936B017C01D42FFC
:1011B000C091100583E08093100581E080931F0C9F
:1011C000C114D104E104F10431F00E94E3FCC60E25
:1011D000D71EE81EF91E80911F0C882389F0C114C8
:1011E000D104E104F10421F48D2F0E94175AF3CFAA
:1011F0000E94E3FC6C197D098E099F0997FDF4CFCD
:1012000010921F0CC0931005DF91CF91FF90EF90CB
:10121000DF90CF9008950F931F93CF93DF93C82F44
:10122000162F0E940F4EC11194C0CFE8D8E0CE0116
:101230000E943C3861E0812F0E94303A0E94E3FC1A
:10124000685370458F4F9F4F60930A0670930B064B
:1012500080930C0690930D0610920E0600911005D7
:1012600083E08093100530E020E049E151E16DE139
:1012700079E082E00E944F408DE199E00E942722B0
:1012800081E080931F0C80911F0C882309F464C0B7
:1012900060E0812F0E94303A80910E06882309F485
:1012A00054C00E940F4E83E099E00E943C3830E029
:1012B00020E04DEE58E064EF78E082E00E944F407D
:1012C00084EF98E00E94272241E060E070E0CB01CB
:1012D0000E94CF8830E020E050E040E060EE78E00F
:1012E00085E00E944F4080EE98E00E9492350E9477
:1012F000201F80E00E94B1850E940F4ECE010E9407
:101300003C380E94E3FC685370458F4F9F4F6093B9
:101310000A0670930B0680930C0690930D061092AC
:101320000E0630E020E049E151E164ED78E082E032
:101330000E944F4083EC98E00E94272281E0809336
:101340001F0C61E0812F0E94303A81E00E94175A01
:101350009ACFC4EAD8E06BCF00931005DF91CF910C
:101360001F910F910895CF92DF92EF92FF920F930A
:101370001F93CF93DF93CDB7DEB7A0970FB6F89446
:10138000DEBF0FBECDBF0E940E4F87FDCCC085E4EF
:101390000E943E1E882309F4D5C00E9492246B014E
:1013A0007C0120E030E0A9010F943A2E87FF04C0B1
:1013B000F7FAF094F7F8F094F7FAF094F7F8F0945D
:1013C000CD8EDE8EEF8EF8A28CE0E6ECF2E0DE0150
:1013D000119601900D928A95E1F78AE50E948C1E84
:1013E000882351F040E050E0BA018AE50E94BC2415
:1013F00069877A878B879C8788E50E948C1E882363
:1014000051F040E050E0BA0188E50E94BC246983B5
:101410007A838B839C8389E50E948C1E882351F0FC
:1014200040E050E0BA0189E50E94BC246D837E83D0
:101430008F83988785E50E943E1E882309F489C022
:101440000E9492246B017C0120E030E0A901C701D9
:10145000B6010F943A2E87FF04C0F7FAF094F7F81C
:10146000F094F7FAF094F7F8F094C98EDA8EEB8ED8
:10147000FC8E1D8A1E8A1F8A188E8CE40E943E1ED6
:10148000882309F46FC00E9492246B017C0120E044
:1014900030E0A901C701B6010F943A2E87FF04C0BE
:1014A000F7FAF094F7F8F094C98ADA8AEB8AFC8AA2
:1014B00062E070E082E40E948324F82E80911B1188
:1014C000811131C021E0AE01475E5F4FBE016F5F09
:1014D0007F4FCE014D960E943988882321F16F2DD0
:1014E00081E00E940B8982E50E948C1E882309F40A
:1014F00042C00E947F2440E050E060EA71E44D87E2
:101500005E876F87788B20911B11222361F08C01FD
:101510002F2DAE01435F5F4FBE016F5E7F4FCE0147
:1015200045960E94F686A0960FB6F894DEBF0FBED1
:10153000CDBFDF91CF911F910F91FF90EF90DF9082
:10154000CF900895C12CD12C80E8E82E80E4F82EAD
:1015500033CFC090BD05D090BE05E090BF05F090A0
:10156000C00572CFC090C105D090C205E090C30500
:10157000F090C4058CCF90E080E0BDCFCF92DF9299
:10158000EF92FF920F931F93CF93DF93CDB7DEB708
:101590006C970FB6F894DEBF0FBECDBF8CE40E94EF
:1015A0003E1E882309F4B0C00E9492246B017C0186
:1015B00020E030E0A9010F943A2E87FF04C0F7FA2B
:1015C000F094F7F8F094F7FAF094F7F8F094C98EE5
:1015D000DA8EEB8EFC8E8CE0E6ECF2E0DE0111960A
:1015E00001900D928A95E1F788E50E948C1E882370
:1015F000A1F040E050E0BA0188E50E94BC242091AF
:10160000C8083091C9084091CA085091CB080F947E
:10161000D92B69837A838B839C8389E50E948C1EF6
:101620008823A1F040E050E0BA0189E50E94BC2483
:101630002091C8083091C9084091CA085091CB0840
:101640000F94D92B6D837E838F8398878AE50E94C0
:101650008C1E882351F040E050E0BA018AE50E94D8
:10166000BC2469877A878B879C871D861E861F8688
:10167000188A80911B11811138C020E0AE01435FB0
:101680005F4FBE016F5F7F4FCE0149960E94398840
:10169000882359F18091C50581110E94EBF660E025
:1016A00080E00E940B89898D9A8DAB8DBC8DB058DE
:1016B0008D8B9E8BAF8BB88F198A1A8A1B8A1C8AD6
:1016C0001D861E861F86188A80911B11882369F04B
:1016D00010E000E020E0AE014B5E5F4FBE016F5EA8
:1016E0007F4FCE010D960E94F6866C960FB6F89449
:1016F000DEBF0FBECDBFDF91CF911F910F91FF9045
:10170000EF90DF90CF900895C12CD12C80E8E82E87
:1017100080E4F82E58CF2F923F924F925F926F92B3
:101720007F928F929F92AF92BF92CF92DF92EF9271
:10173000FF920F931F93CF93DF93CDB7DEB7E5975B
:101740000FB6F894DEBF0FBECDBF8DAB2091100554
:101750002CAB21E02093100580912E058D3409F4E7
:1017600005C6843511F40C94DEA0873409F091C1CC
:1017700080912C0590912D058B31910509F4DDC1E7
:1017800008F079C18430910508F030C12091E1065C
:101790008230910508F48EC1213009F091C111E029
:1017A000029709F010E00E94D32419821A821B824A
:1017B0001C821D821E821F82188682E50E948C1E5A
:1017C000882309F490C10E9492246B017C0120E0DF
:1017D00030E0A9010F940A25882309F4EAC040905B
:1017E000200C5090210C6090220C7090230C809162
:1017F000240C9091250CA091260CB091270C8CA75D
:101800009DA7AEA7BFA780906C0790906D07A09092
:101810006E07B0906F078091700790917107A0914B
:101820007207B091730788AB99ABAAABBBABA501AC
:101830009401C301B2010F940A2581110DC028A99A
:1018400039A94AA95BA96CA57DA58EA59FA50F9472
:101850000A25882309F4ADC0A3019201C501B40192
:101860000F94D92B20E030E040E05FE30F94702527
:1018700068A779A78AA79BA72CA53DA54EA55FA51C
:1018800068A979A98AA99BA90F94D92B20E030E0F7
:1018900040E05FE30F9470252B013C0120E030E035
:1018A000A901C701B6010F940A25881F8827881F40
:1018B000181709F40FC180E090E0A0E8BFEB8CA7F7
:1018C0009DA7AEA7BFA728A539A54AA55BA5CA01B4
:1018D000B9010F9470254B015C01A3019201C30172
:1018E000B2010F9470259B01AC01C501B4010F94A6
:1018F000DA2B0F94882E4B015C01AC019B01C701D0
:10190000B6010F94D92B68AB79AB8AAB9BABA50121
:101910009401C701B6010F94DA2B9B01AC0168A9B1
:1019200079A98AA99BA90F9470256B017C0120E0FD
:1019300030E0A9010F943A2E87FDD1C0C701B6014E
:101940000F94882E6B017C01C301B2019058A50150
:1019500094010F94D42C2CA53DA54EA55FA50F9402
:101960007025A70196010F94702528A539A54AA5D1
:101970005BA50F94DA2B69837A838B839C83A50103
:10198000940168A579A58AA59BA50F94D42C2CA5B4
:101990003DA54EA55FA50F947025A70196010F9454
:1019A0007025A30192010F94DA2B6D837E838F83C0
:1019B000988720E030E0A90169817A818B819C8140
:1019C0000F940A258111A3C020E030E0A9016D81A8
:1019D0007E818F8198850F940A25811198C00E947D
:1019E0000B4E8BEB9FE00E943C386AC0853191051D
:1019F00009F466C08A31910509F49CC0049709F086
:101A000048C080E50E948C1EC12CD12C7601882311
:101A100021F00E940C246B017C0183E50E948C1E46
:101A2000882361F00E94922420E030E04AE754E4E9
:101A30000F9470250F944D2D6B017C010E947B61EA
:101A400080911D11811105C060E081ED9FE00E9431
:101A5000AA3F0E94E3FCC60ED71EE81EF91E0E9494
:101A6000E3FC6C197D098E099F0997FF29C080E06E
:101A70000E94175AF4CF8A32910509F4ECC260F43F
:101A80008D31910509F415C208F470C04E9709F420
:101A900068C20E9404F914C08B35910509F4BEC3D5
:101AA0008C35910509F4BEC38A35910591F71092E2
:101AB000EC0706C0213021F40E94D3240E94B86FA5
:101AC0003DA9311102C00F94EF138CA9809310052A
:101AD0000C943F9980E090E0A0E8BFE3F0CEC12CE9
:101AE000D12C760131CF89E40E948C1E882331F0FD
:101AF0000E94922469837A838B839C838AE40E9468
:101B00008C1E882309F455CF0E9492244ECF412F7A
:101B1000BE016F5F7F4F8CE697E00F9442140E94E6
:101B2000E3FC60936E1170936F118093701190932A
:101B30007111C6CF0E94A777C3CF87E00E941F4EC6
:101B40008111BECF8CE0E2EDF2E0DE011196019052
:101B50000D928A95E1F770E060E080E50E942C2408
:101B6000BE016F5F7F4F0E94A867AACF87E00E94E7
:101B70000D2A811106C060E08FE40E946A24811161
:101B80009FCF0E947B61109246026091310C8CE4E1
:101B90000E946A24E82E80E00E9414690E94E3FCFF
:101BA00060936E1170936F11809370119093711107
:101BB0000E94D31C81E080939D060E94652B8AE5DC
:101BC0000E943E1EF82E882369F081E00E940D2AB3
:101BD000182F82E00E940D2A11110C9401A111E02E
:101BE000811101C010E088E50E943E1E81110C9415
:101BF000F3A0111145C189E50E943E1E082F8113F3
:101C000007C0012FF11204C011E001E0FF24F3949A
